:100000000C943F2B0C94392E0C94642E0C948F2E50
:100010000C94BA2E0C94E52E0C94102F0C943B2FBC
:100020000C94662F0C94702B0C94702B0C94702BEA
:100030000C94702B0C94702B0C94702B0C94702BD4
:100040000C94702B0C9442AF0C94702B0C94702B6E
:100050000C94702B0C94702B0C94F2A20C94722BB9
:100060000C94702B0C944B910C94F7910C94702B76
:100070000C94702B0C94702B0C94702B0C94702B94
:100080000C94702B0C94702B0C94702B0C94702B84
:100090000C94702B0C94702B0C94702B0C94702B74
:1000A0000C94702B0C94702B0C94702B0C94702B64
:1000B0000C94702B0C94702B0C94702B0C94702B54
:1000C0000C94702B0C94702B0C94702B0C94702B44
:1000D0000C94702B0C94702B0C94702B0C94702B34
:1000E0000C94702BAF2CB42CB92CC32CCD2C462DDA
:1000F000D72CDF2CE72CF12CFB2C052D142D1E2DDD
:10010000462D282D322D3C2D6A2D6D2D5C2D602D18
:10011000662DA42D712D752D7B2D7F2D832D892D81
:100120008D2D912DA42D972D9B2D9F2D975D775D66
:100130007D5D7A5D805D835D865D925D895DA45D98
:100140008C5D8F5D868E848EA88EA58EA38EDA8EB2
:10015000D78ED58E338F018FFE8EFC8E7E9184914B
:100160009591A091A891BD91AC91BD91B091B491A0
:10017000BD91BA91084AD73B3BCE016E84BCBFFD0E
:10018000C12F3D6C74319ABD56833DDA3D00C77F67
:1001900011BED9E4BB4C3E916BAAAABE0000008000
:1001A0003F05A84CCDB2D44EB93836A9020C50B98F
:1001B000918688083CA6AAAA2ABE000000803F00BB
:1001C0000D941B320D945E110D94312D4E414E490C
:1001D0004E495459494E46CDCCCC3D0AD7233C1705
:1001E000B7D13877CC2B329595E6241FB14F0A0052
:1001F0000020410000C84200401C4620BCBE4CCA42
:100200001B0E5AAEC59D7400000A0B02090C0D0EA0
:1002100008070304010000000000000000000000C7
:1002200000000000000000000000000000000000CE
:10023000000000121110000000000000000000008B
:10024000000000000000000000000000000102109B
:1002500020200808102040102040800201020108E0
:100260000402010102040810204080804020100890
:1002700004020180040201804020100804020108E9
:100280000402010102040810204080010204081049
:100290002040800505050507050808080802020238
:1002A000020A0A0808040404040101010101010111
:1002B000010303030303030303040707070C0C0CE8
:1002C0000C0C0C0C0C0202020206060606060606C0
:1002D000060B0B0B0B0B0B0B0B0000200023002657
:1002E0000029002C002F003200000100000301064D
:1002F00001090100002200250028002B002E0031FA
:1003000000340002010000050108010B010000217A
:1003100000240027002A002D0030003300010100D6
:1003200000040107010A0101060D00FE0901660231
:10033000D620FFFE0BFE0AFE0D00602219698080A8
:1003400080808080800080183363A0A0A00357675E
:100350005050F850F850500259692078A0A07028E9
:1003600028F02002596948A85010204050A8900257
:10037000586840A0A040A0989068281363808080AF
:10038000113B6B2040408080808080404020113BAA
:100390006B80404020202020204040800655652072
:1003A000A870A8200455652020F820201133636030
:1003B0004080065161F811336340E04002596908FA
:1003C0000810102040408080025969205088888899
:1003D000888850200259692060A02020202020F821
:1003E0000259697088880810204080F8025969F81D
:1003F0000810207008088870025969101030505099
:1004000090F81010025969F88080B0C80808887008
:1004100002596970888080F088888870025969F86C
:100420000810102020404040025969708888887068
:100430008888887002596970888888780808887068
:1004400011386840E040000040E04011386840E06A
:100450004000006040800259690810204080402020
:100460001008045464F80000F80259698040201014
:1004700008102040800259697088880810202000E8
:100480002002596970888898A8A8B08078025969B4
:100490002050888888F8888888025969F048484838
:1004A00070484848F0025969708880808080808850
:1004B00070025969F048484848484848F00259696C
:1004C000F8808080F0808080F8025969F880808010
:1004D000F080808080025969708880808098888848
:1004E0007002596988888888F888888888123969EC
:1004F000E040404040404040E00259693810101050
:100500001010109060025969888890A0C0A090884F
:10051000880259698080808080808080F8025969D3
:100520008888D8A8A88888888802596988C8C8A8EF
:10053000A8989888880259697088888888888888E7
:1005400070025969F0888888F080808080015A6A3A
:1005500070888888888888A87008025969F0888817
:1005600088F0A09088880259697088808070080897
:100570008870025969F8202020202020202002596C
:1005800069888888888888888870025969888888F6
:1005900088505050202002596988888888A8A8A8C7
:1005A000A8500259698888505020505088880259B4
:1005B00069888850502020202020025969F80810AE
:1005C0001020404080F8113B6BE08080808080806C
:1005D000808080E002596980804040201010080827
:1005E000113B6BE0202020202020202020E0085319
:1005F00063205088015161F82A22628040025666C9
:10060000700878889868025969808080F0888888A6
:1006100088F00256667088808088700259690808E0
:10062000087888888888780256667088F88088708C
:1006300002596930484040F04040404000586870DE
:1006400088888878088870025969808080B0C88856
:100650008888881238684000C040404040E0004A26
:100660006A1000301010101090906002596980805C
:100670008090A0C0A09088123969C040404040409E
:100680004040E0025666D0A8A8A8A888025666B0E6
:10069000C88888888802566670888888887000585C
:1006A00068F0888888F0808080005868788888881A
:1006B00078080808025666B0C880808080025666B6
:1006C0007088601088700258684040F04040404890
:1006D00030025666888888889868025666888888B6
:1006E0005050200256668888A8A8A85002566688EE
:1006F000502020508800586888888898680888703A
:10070000025666F810204080F8015B6B182020200C
:1007100020C02020202018221969808080808080BD
:10072000808080015B6BC0202020201820202020AA
:10073000C008536348A890FFFFFFFFFFFFFFFFFFC4
:10074000FFFFFFFFFFFFFFFFFFFFFFFFFFFFFFFFB9
:10075000FFFFFFFFFFFFFFFF0D0060221969800010
:10076000808080808080800358682070A8A0A0A826
:10077000702002596930484040E0404048B003567C
:100780006688705050708802596988885050F820E7
:10079000F82020221969808080800080808080126B
:1007A0004A6A609080609090601090601A3262A0F7
:1007B000A00359697088A8D8C8D8A888700457675A
:1007C000700878887800F80356662850A0A0502852
:1007D000045363F80808163161E00359697088E82A
:1007E000D8D8E8D888700A5161F8174464609090AE
:1007F000600357672020F8202000F807356540A0E7
:100800002040E007356540A04020C02A2262408099
:100810000058688888888898E8808002596978E854
:10082000E8E8E868282828262161C0202262408064
:1008300007356540C04040E004576770888888707D
:1008400000F8035666A050282850A0025A6A40C0FB
:100850004040E00818283808025A6A40C04040E08A
:100860001028081038025A6A40A04020A0481828D2
:100870003808025969200020204080888870025A78
:100880006A40200020508888F88888025A6A102020
:100890000020508888F88888025A6A304800205022
:1008A0008888F88888025A6A28500020508888F87A
:1008B0008888025A6A50500020508888F888880238
:1008C0005A6A20502020508888F888880259695830
:1008D000A0A0A0B0E0A0A0B8005B6B708880808072
:1008E000808088702040025A6A402000F88080F0A2
:1008F0008080F8025A6A102000F88080F08080F82A
:10090000025A6A304800F88080F08080F8025A6A03
:10091000505000F88080F08080F8123A6A804000E1
:10092000E04040404040E0123A6A204000E0404051
:10093000404040E0124A6A609000E0404040404041
:10094000E0123A6AA0A000E04040404040E0025976
:1009500069F0484848E8484848F0025A6A28500078
:100960008888C8A8988888025A6A402000708888B9
:1009700088888870025A6A10200070888888888861
:1009800070025A6A30480070888888888870025AD5
:100990006A28500070888888888870025A6A505087
:1009A0000070888888888870035565885020508832
:1009B000015B6B08709898A8A8A8C8C87080025AF4
:1009C0006A40200088888888888870025A6A1020C7
:1009D0000088888888888870025A6A304800888829
:1009E0008888888870025A6A505000888888888869
:1009F0008870025A6A102000888850202020200227
:100A0000596980F0888888F08080800259696090F8
:100A100090A0A0908888B0025969402000700878A2
:100A200088986802596910200070087888986802D0
:100A300059693048007008788898680259692850C8
:100A400000700878889868025969505000700878DA
:100A5000889868025A6A3048300070087888986828
:100A6000025666702870A0A8500058687088808070
:100A7000887020400259694020007088F880887092
:100A80000259691020007088F88088700259693016
:100A900048007088F880887002596950500070884A
:100AA000F8808870123969804000C040404040E0C2
:100AB000123969204000C040404040E0124969605E
:100AC0009000C040404040E0123969A0A000C04002
:100AD000404040E0025A6A50206010708888888840
:100AE00070025969285000B0C888888888025969FE
:100AF0004020007088888888700259691020007032
:100B00008888888870025969304800708888888889
:100B10007002596928500070888888887002596965
:100B2000505000708888888870035767202000F82C
:100B3000002020015868087098A8A8C87080025941
:100B400069402000888888889868025969102000C8
:100B50008888888898680259693048008888888819
:100B60009868025969505000888888889868005BA6
:100B70006B1020008888889868088870005A6A80FE
:100B800080B0C88888C8B08080005B6B50500088F7
:100B90008888986808887001050700FE0500FB0139
:100BA000F220FFFE05FE05FE0200400215258080B2
:100BB000800080053242A0A002556550F850F850E0
:100BC0000146562070C030E020025565901020404C
:100BD0004802556560806890680512228080022571
:100BE000354080808040022535804040408004337D
:100BF00043A040A003334340E04001223240800440
:100C00003141E00211218002556508102040800228
:100C100045556090909060022535C04040404002AC
:100C20004555E0106080F0024555E0106010E0028C
:100C300045552060A0F020024555F080E010E0020C
:100C400045556080E09060024555F010204040021C
:100C5000455560906090600245556090701060034B
:100C600013238000800214248000808002354520F8
:100C700040804020033343E000E0023545804020BF
:100C80004080024555E0106000400255657088B80C
:100C9000A870024555609090F090024555E090E0B4
:100CA00090E00235456080808060024555E090907C
:100CB00090E0023545E080E080E0023545E080E0EC
:100CC00080800245557080B090700245559090F03C
:100CD0009090023545E0404040E00245553010100C
:100CE000906002455590A0C0A0900235458080805C
:100CF00080E002556588D8A8888802455590D0B014
:100D000090900245556090909060024555E090901B
:100D1000E080014656609090906010024555E0904A
:100D200090E09002455570806010E0023545E0404B
:100D300040404002455590909090600245559090FB
:100D4000A0A04002556588A8A8A8500245559090DB
:100D50006090900245559090701060023545E020FB
:100D60004080E0022535C0808080C002556580400B
:100D7000201008022535C0404040C005324240A046
:100D8000024151F00522328040024454709090702C
:100D900002455580E09090E002344460808060021B
:100DA0004555107090907002445460B0C060023598
:100DB000452040E040400046567090907010600220
:100DC000455580E09090900215258000808080003D
:100DD0002737400040404040800245558090A0E0C9
:100DE000900215258080808080025464F0A8A8A815
:100DF000024454E090909002445460909060004609
:100E000056E09090E08080004656709090701010F0
:100E1000023444A0C0808002445470C030E00235E7
:100E20004540E04040200244549090907002445469
:100E30009090A040025464A8A85050023444A040AE
:100E400040A0004656909090701060024454F020EC
:100E500040F002354560408040600215258080806A
:100E60008080023545C0402040C005425250A0FF5E
:100E7000FFFFFFFFFFFFFFFFFFFFFFFFFFFFFFFF82
:100E8000FFFFFFFFFFFFFFFFFFFFFFFFFFFFFFFF72
:100E9000020040FFFFFFFFFFFFFFFFFFFFFFFFFF1D
:100EA000FFFFFFFFFFFFFFFFFFFFFFFFFFFFFFFF52
:100EB000FFFFFFFFFFFFFFFFFFFFFFFFFFFFFFFF42
:100EC000FFFFFFFFFFFFFFFFFFFFFFFFFFFFFFFF32
:100ED000FFFFFFFFFFFFFFFFFFFFFFFFFFFFFFFF22
:100EE000FFFFFFFFFFFFFFFFFFFFFFFFFFFFFFFF12
:100EF000FFFF01050800FF060121023520FFFF0763
:100F0000FF06FF0900502216568080808000801561
:100F10003353A0A0A00257575050F850F850500239
:100F200057572070A07028702013355580A040A01E
:100F30002002475740A0A040A0A050251353808016
:100F40008012265640808080804012265680404085
:100F50004040800245559060F06090025555202039
:100F6000F82020113353604080044151F011335375
:100F700040E0400246561010204080801236564015
:100F8000A0A0A0A04012365640C0404040E002461B
:100F9000566090106080F0024656F020601090601D
:100FA0000246562060A0F02020024656F080E01055
:100FB00090600246566080E0909060024656F010C5
:100FC0002020404002465660906090906002465655
:100FD000609090701060122555C0C000C0C01136DE
:100FE000566060006040801236562040808040206D
:100FF000034353F000F01236568040202040801208
:10100000365640A020400040015858304898A8A8C3
:10101000904030024656609090F09090024656E024
:1010200090E09090E002465660908080906002468A
:1010300056E090909090E0024656F080E08080F07C
:10104000024656F080E0808080024656609080B074
:1010500090600246569090F0909090123656E04084
:10106000404040E002465670202020A040024656F4
:1010700090A0C0A0A0900246568080808080F002A0
:10108000465690F0F090909002465690D0F0B0B056
:1010900090024656609090909060024656E0909084
:1010A000E08080014757609090D0B06010024656B3
:1010B000E09090E090900246566090402090601240
:1010C0003656E04040404040024656909090909006
:1010D00060024656909090906060024656909090C4
:1010E000F0F09002465690906060909002565688BC
:1010F0008850202020024656F010204080F0123602
:1011000056E080808080E0024656808040201010AB
:10111000123656E020202020E016325240A0014135
:1011200051F0162252804002445470909070024652
:10113000568080E09090E0123454608080600246D7
:101140005610107090907002445460B0C060024617
:1011500056205040E04040014555609070106002BC
:1011600046568080E09090901236564000C0404035
:10117000E01137572000202020A0400246568080F2
:1011800090E09090123656C040404040E0025454E7
:10119000D0A8A8A8024454E09090900244546090D3
:1011A0009060014555E090E0808001455570907059
:1011B0001010024454A0D0808012345460C020C06B
:1011C0000246564040E040502002445490909070B7
:1011D000123454A0A0A04002545488A8A85002443D
:1011E0005490606090014555909070906002445416
:1011F000F02040F0024757304020C02040302216F7
:1012000056808080808080024757C0204030402038
:10121000C006425250A0FFFFFFFFFFFFFFFFFFFF8E
:10122000FFFFFFFFFFFFFFFFFFFFFFFFFFFFFFFFCE
:10123000FFFFFFFFFFFFFF090050221656800080CE
:101240008080800146562070A0A070200246562063
:1012500050E04050A0025555887050708802565694
:101260008850F820F82022175780808000808080E6
:101270000247577080E0907010E0173151A002567D
:101280005670A8C8C8A87014355560A06000E00367
:10129000435350A050123353E02020143151E00248
:1012A000565670E8D8E8D870173151E015335340DE
:1012B000A04012355540E04000E014355540A020D4
:1012C00040E0143555C020C020C016225240800195
:1012D0004555909090E08002565678E8E8682828B6
:1012E00024115180112252408014355540C0404095
:1012F000E014355540A04000E0034353A050A00245
:101300004757808080A060F0200247578080A0D09F
:1013100010207002475780408060A0F0201236569F
:1013200040004080A04002475740206090F09090DD
:1013300002475720406090F09090024757609060BD
:1013400090F0909002475750A06090F09090024724
:101350005790006090F0909002475760906090F036
:10136000909002465670A0A0F0A0B0014757609040
:1013700080809060400247574020F080E080F0027B
:1013800047572040F080E080F00247576090F0809F
:10139000E080F00247579000F080E080F01237576D
:1013A0008040E0404040E01237572040E04040405D
:1013B000E012375740A0E0404040E0123757A0000D
:1013C000E0404040E00256567048E8484870024706
:1013D0005750A090D0B09090024757402060909016
:1013E000906002475720406090909060024757609D
:1013F00090609090906002475750A06090909060ED
:1014000002475790006090909060123353A040A024
:1014100002465670B0B0D0D0E002475740209090BE
:1014200090906002475720409090909060024757FC
:1014300060909090909060024757900090909090AC
:10144000600257571020885020202002465680E026
:101450009090E0800246566090A0A090A00247576E
:10146000402000709090700247572040007090908C
:10147000700247572050007090907002475750A05C
:101480000070909070024656500070909070024725
:101490005760906070909070025454F068B078116A
:1014A0003555608080604002475740200060B0C0E2
:1014B0006002475720400060B0C06002475760900C
:1014C0000060B0C060024656500060B0C060123785
:1014D00057804000C04040E0123757204000C040D5
:1014E00040E012375740A000C04040E0123656A0FE
:1014F00000C04040E0024757A040A010709060023A
:10150000475750A000E0909090024757402000605D
:1015100090906002475720400060909060024757CB
:101520006090006090906002475750A000609090DB
:10153000600246569000609090601235554000E081
:10154000004002445470B0D0E00247574020009061
:10155000909070024757204000909090700247573B
:10156000609000909090700246569000909090701D
:10157000014858204000909070906001475780804B
:10158000E090E0808001475790009090709060203C
:10159000202020002020202020200025753A253002
:1015A000327500253032753A253032750025756464
:1015B00020253032753A25303275003FFFF0380073
:1015C000703186302387102787902F87D02F03D044
:1015D0002030102078102078102030102F03D02FCA
:1015E00087D02787902387103186303800703FFFDF
:1015F000F03FFFF038007030FC3020FC10207810F5
:101600002030102C00D02E31D02F7BD02F7BD02E2D
:1016100031D02C00D020301020781020FC1030FC6D
:10162000303800703FFFF00410400208200208200C
:101630000410400820801041001041000820800460
:1016400010400000001FFFF81FFFF81FFFF81FFFEA
:10165000F81FE02010201020101020102020102053
:101660001030300840048003001FE03FF03FF03F9F
:10167000F01FE01FE03FF03FF03FF00FC007800396
:10168000004572723A207574663820666F6E742059
:101690006E6F7420696E697469616C697A65642E15
:1016A000004572723A207574663820666F6E742039
:1016B0006E6F7420696E697469616C697A65642EF5
:1016C000004572723A207574663820666F6E742019
:1016D0006E6F7420696E697469616C697A65642ED5
:1016E00000506C65617365207265736574005052BB
:1016F000494E5445522048414C544544007F80FF98
:10170000C0FFC0FFC07F807F80FFC0FFC0FFC03F21
:10171000001E000C00FFFFFF0E000E000E000E006A
:101720000E000E000E000E007FC03F801F000E0056
:10173000040004000E001F003F807FC00E000E005A
:101740000E000E000E000E000E000E0000FE000344
:10175000FF800783C00E01C00E00E01C00E07F0088
:10176000E03E00E01C00E00800E00000E00001C0F6
:101770000E01C00F078007FF0001FC0003F8000FF7
:10178000FE001E0F00380700380380700380700FC2
:10179000E07007C070038070010070000038000026
:1017A0003807001E0F000FFE0003F80000060C00B3
:1017B000FE07022603BC017FFE08FE08FE0508089E
:1017C00006000040F0C888889878100508080600D0
:1017D00000C0F88888888888F8050505060001207B
:1017E00030F830200508080600002070F82020207E
:1017F00020E00509090600FF2070A8A8B8888870B5
:1018000020050606060001E08CEA8C8A0A05090913
:101810000600FFF8A88888888888A8F8050A0A06BC
:1018200000FE205050505088A8A88870030303067B
:10183000000340A040FFFFFFFFFFFFFFFFFFFFFF90
:10184000FFFFFFFFFFFFFFFFFFFFFF000000060598
:10185000FF0107070602008080808080008003036C
:1018600003060105A0A0A005060606000050F850DA
:1018700050F8500509090600FF2070A8A07028A89C
:101880007020050707060000C8C81020409898057A
:10189000070706000040A0A040A8906801030306C7
:1018A00002058080800309090601FF2040408080F6
:1018B000804040200309090601FF8040402020208D
:1018C00040408005070706000020A8702070A8206F
:1018D0000505050600012020F8202002030306016B
:1018E000FFC04080050101060003F8020202060164
:1018F00000C0C00507070600000810102040408007
:10190000050707060000708898A8C88870030707B5
:1019100006010040C040404040E0050707060000C7
:10192000708808102040F8050707060000F8081026
:101930003008887005070706000010305090F81036
:1019400010050707060000F880F0080888700507F2
:1019500007060000304080F0888870050707060001
:1019600000F80810102020200507070600007088E6
:1019700088708888700507070600007088887808D6
:101980001060020505060100C0C000C0C0020606C6
:101990000601FFC0C000C04080030505060101200C
:1019A00040804020050303060002F800F803050507
:1019B000060101804020408005070706000070886E
:1019C00010202000200507070600007088B8A8B87E
:1019D0008070050707060000708888F888888805E9
:1019E0000707060000F04848704848F0050707065A
:1019F000000070888080808870050707060000F06E
:101A00004848484848F0050707060000F88080F07D
:101A10008080F8050707060000F88080F08080804D
:101A20000507070600007088808098887005070702
:101A3000060000888888F888888803070706010060
:101A4000E04040404040E005070706000038101025
:101A5000101090600507070600008890A0C0A090B5
:101A600088050707060000808080808080F80507D1
:101A70000706000088D8A888888888050707060018
:101A8000008888C8A898888805070706000070881D
:101A90008888888870050707060000F08888F0802D
:101AA000808005070706000070888888A890680570
:101AB0000707060000F08888F0A090880507070651
:101AC000000070888070088870050707060000F81D
:101AD000202020202020050707060000888888880D
:101AE000888870050707060000888888885050207D
:101AF00005070706000088888888A8A850050707FA
:101B000006000088885020508888050707060000D6
:101B100088885020202020050707060000F80810BC
:101B2000204080F80309090601FFE0808080808062
:101B30008080E00507070600008040402010100864
:101B40000309090601FFE020202020202020E005D5
:101B500003030600052050880501010600FEF80376
:101B600003030601058040200505050600007008F6
:101B70007888780507070600008080F0888888F05C
:101B800005050506000070808088700507070600BF
:101B900000080878888888780505050600007088A0
:101BA000F08070050707060000304840E0404040E4
:101BB0000507070600FE7088888878087005070703
:101BC0000600008080F088888888030707060100E7
:101BD0004000C0404040E00409090601FE1000300A
:101BE0001010101090600507070600008080889094
:101BF000E09088030707060100C04040404040E0F5
:101C0000050505060000D0A8A8A8A805050506003A
:101C100000B0C88888880505050600007088888897
:101C2000700507070600FEF0888888F080800507A9
:101C3000070600FE788888887808080505050600EC
:101C400000B0C88080800505050600007880700817
:101C5000F00507070600002020F8202020180505C1
:101C60000506000088888898680505050600008834
:101C7000888850200505050600008888A8A850051A
:101C8000050506000088502050880507070600FE5D
:101C900088888850204080050505060000F810203F
:101CA00040F80309090601FF2040404080404040C1
:101CB000200109090602FF8080808080808080806A
:101CC0000309090601FF8040404020404040800554
:101CD000030306000248A890FF01FFFFFFFFFFFF7C
:101CE000FFFFFFFFFFFFFF0FFFFFFFFFFFFFFFFFF4
:101CF000FFFFFFFFFF1E00000000000000000000CB
:101D000007FFFF380000000000000000000003FF94
:101D1000FF700000000000000000000001FFFF60F5
:101D20000000000000000000000000FFFF60000055
:101D30000000000000000000007FFFC00000000065
:101D4000000000007800003FFFC00FC0FC00000052
:101D500000007818001FFFC03FE1FF0000000000F6
:101D6000783C000FFFC07FF3FF8000000000783C4C
:101D70000007FFC0FFFFFFC000000000783C000329
:101D8000FFC1F87F87E00000000078000001FFC17C
:101D9000F03F03E00000000078000000FFC1E01EFB
:101DA00001E01F0003E0783C03F07FC1E01E01E08A
:101DB0007FC00FF8783C07FC3FC1E01E01E1FFE067
:101DC0001FFC783C0FFE1FC1E01E01E3FFF03FFE49
:101DD000783C1FFE0FC1E01E01E3F3F83F3E783C64
:101DE0003F3F07C1E01E01E7E0FC7C1F783C3E1F3F
:101DF00007C1E01E01E7C07C7C0F783C3C0F03C1AB
:101E0000E01E01E7807C780F783C3C0F03C1E01EA8
:101E100001E7803C7800783C3C0F03C1E01E01E7FD
:101E2000803C7800783C3C0F03C1E01E01E7803C19
:101E30007800783C3C0F03C1E01E01E7C03C78000D
:101E4000783C3C0F03C1E01E01E3E03C78007C3CA1
:101E50003C0F03C1E01E01E3FF3FF8007FBC3C0FD5
:101E600003C1E01E01E1FF3FF8003FBFFC0F03C1CB
:101E7000E01E01E0FF3FF8001FBFFC0F03C1E01EA2
:101E800001E07F3FF8000FBFFC0F0360000000007F
:101E900000000000000000000760000000000000DB
:101EA00000000000000006700000000000000000BC
:101EB000000000000E3800000000000000000000DC
:101EC00000001C1E000000000000000000000000D8
:101ED000780FFFFFFFFFFFFFFFFFFFFFFFFFF00196
:101EE000FFFFFFFFFFFFFFFFFFFFFFFF800000007E
:101EF00000000000000000000000000000000000E2
:101F000000000000000000000000000000000000D1
:101F10000C000000000000000C00000000000000A9
:101F2000120000000000000023000000000000007C
:101F300021000000000000004C80000000000000B4
:101F40005E800000000000009240000000000000E1
:101F5000A14000000000000121200000000000025C
:101F60007F90000000000002001000000000000749
:101F7000FFF8000000000004000800000000000856
:101F8000000400000000000800060000000000102F
:101F900000020000000000301E01000000000020D0
:101FA0007F81000000000041FFE08000000000434E
:101FB000FCF08000000000873B7840000000018EAC
:101FC000DBFC60000000010FEBCC20000000021FD2
:101FD000EDB610000000021FDEB61000000004394C
:101FE000CD7F080000000436E0FF08000000087EF6
:101FF000C0BB84000000187F005D86000000107FD9
:10200000C0ED82000000203CC07301000000203BB6
:10201000337F01000000701BE77E03800000C81DB5
:10202000EEDE04C00000880FDEDC04400001240F57
:10203000DF3C092000012607DBF8192000027203AB
:10204000E7F0139000025101FFE0229000048900A4
:102050007F802448000904801E004824000BFE40B5
:102060000000DFF40010004000008002001FFFFFAE
:10207000FFFFFFFE00000000000000000000000065
:10208000000000000000000000000000001022100E
:102090003C3C0E1F001022100422110400102210DC
:1020A0000822110400102210083C11040010221014
:1020B000102211040010221020221104001E1C1EE8
:1020C0003C3C0E0400000000000000000000000086
:1020D0000000000000000000000000000000000000
:1020E00000000000000000000000000000000000F0
:1020F00000000000000000000000000000000000E0
:1021000000000000000000000000000000000000CF
:1021100000000000000000000000000000000000BF
:10212000000000000000000000000000060900FEA2
:1021300006018902FE20FFFE07FE06FE00000006E3
:1021400000070106060602008080808000800303ED
:1021500003060103A0A0A00507070600FF5050F8E2
:1021600050F850500509090600FE2070A8A07028FC
:10217000A870200608080600FF40A8481020485410
:10218000080507070600FF609090609890680103BB
:10219000030602038080800207070602FF4080805A
:1021A000808080400207070602FF80404040404098
:1021B000800505050600008850F8508805050506CD
:1021C00000002020F820200204040602FEC0404047
:1021D00080050101060002F8020202060200C0C0EA
:1021E0000406060601001010204080800406060642
:1021F000010060909090906003060606010040C0C8
:10220000404040E00406060601006090102040F0C7
:10221000040606060100F020601010E00506060620
:10222000000010305090F810040606060100F080FF
:10223000E01010E00406060601006080E090906067
:10224000040606060100F0101020404004060606B1
:1022500001006090609090600406060601006090A6
:1022600090701060020505060200C0C000C0C002E8
:1022700007070602FEC0C000C040408005050506F5
:1022800000001860806018050303060001F800F8DC
:10229000050505060000C0300830C0040707060128
:1022A0000060901060400040050606060000709037
:1022B000A8B08070050606060000205088F88888BF
:1022C000050606060000F088F08888F00406060679
:1022D0000100609080809060040606060100E09096
:1022E000909090E0040606060100F080E08080F007
:1022F000040606060100F080E080808004060606E1
:102300000100609080B09060040606060100909085
:10231000F0909090030606060100E040404040E047
:102320000506060600003810101090600406060628
:10233000010090A0C0A090900406060601008080D5
:10234000808080F005060606000088D8A8A8888846
:1023500004060606010090D0B0909090050606068F
:102360000000708888888870040606060100E090E6
:1023700090E080800407070601FF609090D0B06075
:1023800010040606060100E09090E0909004060616
:10239000060100609040209060050606060000F8E7
:1023A00020202020200406060601009090909090A6
:1023B00060040606060100909090F0606005060635
:1023C0000600008888A8A8D88805060606000088A8
:1023D00050202050880506060600008888502020DE
:1023E00020040606060100F010204080F0030606D7
:1023F000060100E080808080E0040606060100807F
:102400008040201010030606060100E02020202056
:10241000E00503030600032050880501010600FEC5
:10242000F80202020602048040040404060100705F
:102430009090700406060601008080E09090E00411
:102440000404060100708080700406060601001076
:10245000107090907004040406010060B0C0700415
:102460000606060100205040E04040040606060132
:10247000FE6090907010600406060601008080E007
:102480009090900306060601004000C04040E00323
:1024900008080601FE200060202020A04004060657
:1024A0000601008080A0C0A090030606060100C0BF
:1024B00040404040E0050404060000D0A8A888047D
:1024C0000404060100E090909004040406010060FA
:1024D0009090600406060601FEE09090E080800483
:1024E00006060601FE7090907010100404040601A8
:1024F00000A0D0808004040406010070C030E00415
:1025000006060601004040E0405020040404060195
:1025100000909090700404040601009090606005A3
:10252000040406000088A8A85004040406010090D2
:102530006060900406060601FE9090907090600422
:102540000404060100F02040F00307070601002004
:102550004040804040200107070602FF80808080C5
:1025600080808003070706010080404020404080B3
:1025700004020206010350A0FFFFFFFFFFFFFFFF61
:10258000FFFFFFFFFFFFFFFFFFFFFFFFFFFFFFFF5B
:10259000FFFFFFFFFFFFFFFFFF0000000600070136
:1025A0000606060200800080808080040606060180
:1025B000FF2070A0A070200507070600FF304840EC
:1025C000F04040F8050505060000A8508850A80511
:1025D00006060600008850F820F8200107070602CA
:1025E000FF808080008080800407070601FF7080E4
:1025F00060906010E0030101060105A006070706D0
:102600000000788494A49484780305050601016091
:10261000A06000E00505050600002850A050280431
:102620000303060100F01010040101060102F00688
:1026300007070600007884B4A4A484780401010686
:102640000105F00403030601026090600507070618
:1026500000FF2020F8202000F803050506010140B6
:10266000A02040E0030505060101C0204020C00273
:10267000020206020440800405050601FF9090B0A6
:10268000D08005060606000078E8E86828280101E1
:1026900001060202800202020602FE4080030505D6
:1026A00006010140C04040E003050506010140A0CD
:1026B0004000E0050505060000A0502850A00508D0
:1026C000080600FF40C0405070307810050808062A
:1026D00000FF40C04050680810380508080600FF99
:1026E000C0204030F03078100407070601002000B9
:1026F0002060809060050707060000402020507091
:10270000888805070706000010202050708888057B
:10271000070706000020502050708888050707062C
:1027200000002850205070888805070706000050D8
:1027300000205070888805070706000020502050B0
:1027400070888805060606000078A0F0A0A0B804EE
:1027500008080601FE609080809060204004070712
:102760000601004020F080E080F004070706010029
:102770002040F080E080F00407070601002050F0C0
:1027800080E080F00407070601005000F080E08040
:10279000F00307070601008040E0404040E00307E7
:1027A000070601002040E0404040E0030707060123
:1027B0000040A0E0404040E0030707060100A00001
:1027C000E0404040E00506060600007048E8484842
:1027D0007004070706010050A090D0B09090040745
:1027E00007060100402060909090600407070601F2
:1027F0000020406090909060040707060100205080
:10280000609090906004070706010050A0609090CF
:1028100090600407070601005000609090906005EA
:10282000050506000088502050880408080601FFAE
:102830001070B0B0D0D0E08004070706010040203F
:1028400090909090600407070601002040909090BF
:10285000906004070706010020509090909060045B
:10286000070706010050009090909060050707064A
:102870000000102088502020200406060601008059
:10288000E09090E0800406060601006090A0A09011
:10289000A004070706010040200070909070040714
:1028A00007060100204000709090700407070601A1
:1028B000002050007090907004070706010050A09F
:1028C0000070909070040606060100500070909011
:1028D00070040707060100205020709090700504D6
:1028E0000406000070A8B0780406060601FE708099
:1028F0008070204004070706010040200060B0C03F
:102900007004070706010020400060B0C070040793
:102910000706010020500060B0C0700406060601E2
:1029200000500060B0C0700307070601008040003F
:10293000C04040E0030707060100204000C04040BF
:10294000E003070706010040A000C04040E0030686
:1029500006060100A000C04040E004070706010091
:102960003060107090906004070706010050A000CE
:10297000E0909090040707060100402000609090CE
:102980006004070706010020400060909060040783
:1029900007060100205000609090600407070601C0
:1029A0000050A000609090600406060601005000F0
:1029B000609090600505050600002000F8002004E6
:1029C000040406010070B0D0E004070706010040CF
:1029D00020009090907004070706010020400090AE
:1029E00090907004070706010020500090909070AE
:1029F0000406060601005000909090700409090634
:102A000001FE20400090909070906004080806013C
:102A1000FE8080E09090E080800408080601FE506F
:102A2000009090907090605072696E742066726F22
:102A30006D205344005072696E742066726F6D2071
:102A4000534400022E2E004D61696E005072696E73
:102A5000740043616E63656C00537461727420701E
:102A600072696E7420003F00536D6F6F7468696EF9
:102A70006700536D6F6F7468696E67005A005A0083
:102A80005900590058005800436F727265637469A9
:102A90006F6E00436F7272656374696F6E004D6193
:102AA000696E0046696C616D656E7400447269768A
:102AB0006520537472656E677468004261636B6C65
:102AC0006173680053746570732F6D6D004A657291
:102AD0006B00416363656C65726174696F6E00566B
:102AE000656C6F6369747900436F6E6669677572B0
:102AF0006174696F6E004573746570732F6D6D003E
:102B00004573746570732F6D6D005A7374657073BF
:102B10002F6D6D005A73746570732F6D6D0059734E
:102B2000746570732F6D6D005973746570732F6DBC
:102B30006D005873746570732F6D6D0058737465F4
:102B400070732F6D6D00416476616E636564205310
:102B5000657474696E67730056652D6A65726B00E3
:102B600056652D6A65726B00567A2D6A65726B0028
:102B7000567A2D6A65726B0056792D6A65726B0004
:102B800056792D6A65726B0056782D6A65726B00F6
:102B900056782D6A65726B00416476616E63656478
:102BA0002053657474696E677300416D61782045C8
:102BB00000416D6178204500416D6178205A0041E7
:102BC0006D6178205A00416D6178205900416D6136
:102BD00078205900416D6178205800416D6178205E
:102BE0005800412D74726176656C00412D747261DC
:102BF00076656C00412D7265747261637400412DBD
:102C00007265747261637400416363656C00416353
:102C100063656C00416476616E636564205365741E
:102C200074696E6773005654726176206D696E0028
:102C30005654726176206D696E00566D696E00564D
:102C40006D696E00566D6178204500566D61782083
:102C50004500566D6178205A00566D6178205A0003
:102C6000566D6178205900566D6178205900566D77
:102C70006178205800566D61782058004164766173
:102C80006E6365642053657474696E6773004C6F7E
:102C90006164206D6D004C6F6164206D6D00556E38
:102CA0006C6F6164206D6D00556E6C6F6164206D9A
:102CB0006D00416476616E6365204B00416476610E
:102CC0006E6365204B00416476616E6365642053DA
:102CD000657474696E677300450045005A005A00B8
:102CE000585900585900436F6E74726F6C004469F4
:102CF0007361626C65207374657070657273004DEA
:102D00003834004175746F2D63616C69627261744F
:102D100065004C6576656C20582041786973000029
:102D20004175746F20686F6D6500473238004D6FD4
:102D300076652061786973004D61696E004578742D
:102D4000727564657220004D6F7665205A004D6F74
:102D500076652059004D6F76652058004D6F766579
:102D60006D656E7400457874727564657220004DEF
:102D70006F766520302E316D6D004D6F7665203198
:102D80006D6D004D6F76652031306D6D004D6F7645
:102D900065206178697300486F74656E6420746F94
:102DA0006F20636F6C64004578747275646572207F
:102DB000004D6F7665205A004D6F76652059004DA5
:102DC0006F76652058004D6F7665205A004D6F76FE
:102DD000652059004D6F7665205800576169742051
:102DE000666F720066696C616D656E7420707572D5
:102DF00067650000506C6561736520776169742EAA
:102E000000507265737320627574746F6E00746F16
:102E100020726573756D65207072696E74005761FC
:102E2000697420666F720066696C616D656E7420EE
:102E30006C6F616400496E736572742066696C61C1
:102E40006D656E7400616E642070726573732062CC
:102E50007574746F6E00746F20636F6E74696E7535
:102E60006500507265737320627574746F6E0074C0
:102E70006F2068656174206E6F7A7A6C65004E6FA2
:102E80007A7A6C652068656174696E6700506C655C
:102E900061736520776169742E2E2E005761697405
:102EA00020666F720066696C616D656E7420756E68
:102EB0006C6F6164005761697420666F72006669A7
:102EC0006C616D656E74206368616E676500746F18
:102ED000207374617274005061726B696E672E2E7C
:102EE0002E004368616E67696E672046696C616D8C
:102EF000656E7400554E4C4F41442046494C414D3F
:102F0000454E54004C4F41442046494C414D454E9E
:102F1000540020204E6F7A7A6C653A2000200045DC
:102F20006E642066696C616D656E74206368616EA5
:102F30006765005075726765206D6F7265000043AC
:102F400068616E67652066696C616D656E740055B9
:102F50006E6C6F61642066696C616D656E74004CA7
:102F60006F61642066696C616D656E74004D36300A
:102F70003020423020542564004D373032203B252C
:102F800064004D37303220542564004D37303120F5
:102F900054256400507265686561742043757374CC
:102FA0006F6D005072656865617420437573746F4E
:102FB0006D00507265686561742041425300507223
:102FC000656865617420504C41004261636B004E3E
:102FD0006F2053442063617264005072696E7420E4
:102FE00066726F6D2053440041626F757420507299
:102FF000696E746572004368616E67652066696C0E
:10300000616D656E74004368616E67652066696C0A
:10301000616D656E74004D36303020423000436F74
:103020006E66696775726174696F6E0054656D7064
:1030300065726174757265004D6F76656D656E744D
:1030400000526573756D65207072696E74005475F9
:103050006E650053746F70207072696E74005061F9
:10306000757365207072696E7400496E666F2073A7
:10307000637265656E0053746F70207072696E7450
:10308000004D61696E005072696E742061626F72EA
:10309000746564004D3234004D323520500A4D3293
:1030A000340050726F6265205A204F6666736574F3
:1030B00000426162797374657020590042616279DF
:1030C00073746570205800466C6F7700466C6F779C
:1030D0000046616E2073706565640046616E207302
:1030E000706565640042656400426564004E6F7AF5
:1030F0007A6C65004E6F7A7A6C6500537065656412
:10310000005370656564004D61696E0042616279CB
:103110007374657020590042616279737465702020
:103120005800436F6F6C646F776E0046616E20735A
:10313000706565640046616E207370656564004269
:10314000656400426564004E6F7A7A6C65004E6F6C
:103150007A7A6C65004D61696E00526573746F72A6
:1031600065206661696C73616665004C6F616420FF
:1031700073657474696E67730053746F726520733E
:10318000657474696E67730050726F6265205A20AF
:103190004F666673657400416476616E6365642092
:1031A00053657474696E6773004D61696E00507287
:1031B0006F6265205A204F6666736574004C756CAB
:1031C0007A426F74204D696E692072656164792E50
:1031D000005072696E74696E672E2E2E00507269EF
:1031E0006E7420706175736564004361726420724F
:1031F000656D6F766564004361726420696E736506
:1032000072746564004D33310043616E6E6F7420DB
:10321000656E746572207375626469723A20002E5F
:103220000A006F70656E206661696C65642C2046CB
:10323000696C653A20006175746F25632E670065BF
:1032400072726F722077726974696E6720746F2072
:1032500066696C650A004E6F742053442070726971
:103260006E74696E670A005344207072696E7469E7
:103270006E67206279746520002E0A0044656C65D3
:1032800074696F6E206661696C65642C2046696C98
:10329000653A200046696C652064656C65746564F8
:1032A0003A0057726974696E6720746F2066696CA2
:1032B000653A20002E0A006F70656E206661696CA9
:1032C00065642C2046696C653A20002E0A006F70F8
:1032D000656E206661696C65642C2046696C653A90
:1032E000200046696C652073656C65637465640ACB
:1032F000002053697A653A200046696C65206F703A
:10330000656E65643A20002066696C653A20006647
:103310007265736800646F696E67004E6F77200096
:10332000454E4420535542524F5554494E450A008C
:103330002220706F73002220706172656E743A22D1
:1033400000535542524F5554494E452043414C4C31
:10335000207461726765743A2200747279696E67CD
:1033600020746F2063616C6C207375622D67636FCE
:1033700064652066696C6573207769746820746F72
:103380006F206D616E79206C6576656C732E204DB3
:103390004158206C6576656C2069733A310A004D9E
:1033A0003234004D32332025730053442063617260
:1033B00064206F6B0A006F70656E526F6F742066C9
:1033C00061696C65640A00766F6C756D652E696E57
:1033D0006974206661696C65640A00534420696EF3
:1033E0006974206661696C0A00286E6F2066696CDA
:1033F00065290043616E6E6F74206F70656E207377
:10340000756264697220007C3C3E5E2B3D3F2F5B01
:103410005D3B2C2A225C004F4646004F4E00656300
:10342000686F3A004572726F723A004572726F723D
:103430002077726974696E6720746F204545505219
:103440004F4D210A00507265737320627574746F5A
:103450006E20286F72204D3130382920746F20681B
:10346000656174206E6F7A7A6C650A0050726573BC
:103470007320627574746F6E20286F72204D313026
:10348000382920746F20726573756D650A00496E66
:10349000736572742066696C616D656E7420616E0F
:1034A0006420707265737320627574746F6E202867
:1034B0006F72204D313038290A004D3630303A20B5
:1034C000546F6F20636F6C6400486F74656E642086
:1034D000746F6F20636F6C640A00486F74656E646C
:1034E00020746F6F20636F6C640A00496E7365729D
:1034F000742066696C616D656E7420616E64207005
:103500007265737320627574746F6E20286F7220F9
:103510004D313038290A0063616E63656C00726555
:1035200073756D656400726573756D6500706175A6
:1035300073656400706F7765726F6666002F2F6128
:103540006374696F6E3A0020573A0020573A00457D
:103550007874727564657220436F6F6C696E672E44
:103560002E2E00457874727564657220486561740A
:10357000696E672E2E2E00202F002042403A002038
:10358000403A004D383420582059205A20450054E4
:103590006865726D616C2052756E61776179004566
:1035A0003120544845524D414C2052554E415741CF
:1035B000590042656400202D20496E76616C696473
:1035C000206578747275646572206E756D626572BF
:1035D00020210A0048656174696E67206661696C24
:1035E0006564004265640048656174696E672066C1
:1035F00061696C65640045312048656174696E6776
:10360000206661696C6564004D494E54454D5020FB
:10361000747269676765726564004531204572722E
:103620003A204D494E54454D5000426564004D418D
:103630005854454D5020747269676765726564001F
:103640004531204572723A204D415854454D500045
:1036500042656400626564002C2073797374656D43
:103660002073746F707065642120486561746572A1
:103670005F49443A200023646566696E65204445CD
:103680004641554C545F004B6420004B6920004B71
:103690007020000062656400504944204175746FD9
:1036A00074756E652066696E697368656421205063
:1036B000757420746865206C617374204B702C20C5
:1036C0004B6920616E64204B6420636F6E7374617C
:1036D0006E74732066726F6D2062656C6F772069FF
:1036E0006E746F20436F6E66696775726174696F7F
:1036F0006E2E680A00504944204175746F74756ECF
:1037000065206661696C6564212074696D656F75FB
:10371000740A00546865726D616C2052756E617731
:10372000617900453120544845524D414C20525555
:103730004E41574159004265640048656174696EA5
:1037400067206661696C6564004531204865617475
:10375000696E67206661696C65640042656400504B
:103760004944204175746F74756E65206661696C9B
:103770006564212054656D70657261747572652091
:10378000746F6F20686967680A00204B643A2000F4
:10379000204B693A2000204B703A20000A20436CED
:1037A000617373696320504944200A002054753ABC
:1037B0002000204B753A2000206D61783A200020CF
:1037C0006D696E3A200020643A20002062696173BE
:1037D0003A2000504944204175746F74756E65201D
:1037E00073746172740A00504944204175746F7497
:1037F000756E65206661696C6564212054656D7025
:103800006572617475726520746F6F20686967688E
:103810000A001000AD0330016A0150022B01700351
:103820000A019004F500B005E500D006D800F007C5
:10383000CE001009C500300ABE00500BB700700C56
:10384000B100900DAB00B00EA600D00FA200F0109A
:103850009D001012990030139500501492007015BD
:103860008E0090168B00B0178700D0188400F019D6
:103870008100101B7E00301C7B00501D7900701EE3
:103880007600901F7300B0207000D0216E00F022EF
:103890006B001024690030256600502663007027F5
:1038A000610090285E00B0295C00D02A5900F02BFE
:1038B0005600102D5400302E5100502F4E00703005
:1038C0004B0090314800B0324500D0334200F03414
:1038D0003E0010363B003037370050383300703927
:1038E0002E00903A2900B03B2300D03C1B00F03D55
:1038F0001100103F0100F03F00001000C90210014C
:103900002C014001220170011801B0010E01F001EB
:1039100004015002FA00B002F0003003E600D003C8
:10392000DC009004D2007005C800A006BE000008AC
:10393000B400B009AA00D00BA000600E9600601180
:103940008C000015820020197800C01D6E00A02296
:103950006400B0275A00902C500000314600E0343B
:103960003C0010383200903A2800603C1E00A03D18
:103970001400803E0A00203F00006F70656E005406
:103980005249474745524544003A20007A5F6D61ED
:1039900078007A5F6D696E00795F6D617800795F9C
:1039A0006D696E00785F6D617800785F6D696E009B
:1039B0005265706F7274696E6720656E6473746FA0
:1039C00070207374617475730A00456E6473746F4C
:1039D0007073202563202563202563202563002044
:1039E0005A3A0020593A0020583A00656E647374C0
:1039F0006F7073206869743A2000486F6D696E6754
:103A0000206661696C656400496E76616C6964204A
:103A100065787472756465720A0045303A20005A00
:103A20003A2000593A20004D53312C4D53322C4D41
:103A300053332050696E730A583A20004D696372FF
:103A40006F737465707320756E617661696C616205
:103A50006C650A00205A3A0020593A0020436F75DD
:103A60006E7420583A00C23100001C260000F41980
:103A70000000D80F0000EB080000C0040000750231
:103A800000004001000024F4D43050C38E20C2A2B4
:103A90004017828B7011127A910D816CD90AA8613E
:103AA000E108C7586607615143061E4B5D05C145D5
:103AB000A7041A411104093D9803713931034036B6
:103AC000DB0265339102D4305402802E1D02632C38
:103AD000EE01752AC501B028A001102781018F25AC
:103AE00064012B244B01E0223401AC211F018D2005
:103AF0000D01801FFC00841EED00971DDF00B81C27
:103B0000D200E61BC600201BBC00641AB200B2192A
:103B1000A8000A19A0006A189900D117910040174F
:103B20008B00B516840031167E00B31579003A1566
:103B30007300C7146F0058146A00EE1366008813F0
:103B4000630025135E00C7125B006C12570015124C
:103B50005400C111510070114F0021114B00D610BB
:103B600049008D1047004610440002104200C00F6B
:103B70004000800F3E00420F3C00060F3B00CB0E82
:103B80003800930E37005C0E3500270E3400F30D1D
:103B90003200C10D3100900D3000600D2E00320D4D
:103BA0002D00050D2C00D90C2B00AE0C2900850C26
:103BB00029005C0C2700350C27000E0C2600E80BB2
:103BC0002400C40B2400A00B23007D0B23005A0B00
:103BD0002100390B2100180B2000F80A1F00D90A18
:103BE0001E00BB0A1E009D0A1D00800A1D00630AFC
:103BF0001C00470A1B002C0A1B00110A1A00F709B7
:103C00001A00DD091900C4091900AB09190092094D
:103C100017007B091800630917004C0916003609C4
:103C20001600200916000A091500F5081500E0081D
:103C30001400CC081400B8081400A408140090085C
:103C400013007D0812006B08130058081200460884
:103C50001200340811002308110012081100010895
:103C60001100F0071000E0071000D0071000C00797
:103C70001000B0070F00A107100091070E00830786
:103C80000F0074070F0065070E0057070E00490765
:103C90000E003B070D002E070E0020070D00130736
:103CA0000D0006070D00F9060C00ED060D00E006FC
:103CB0000C00D4060C00C8060C00BC060C00B006B4
:103CC0000C00A4060B0099060C008D060B00820662
:103CD0000B0077060B006C060B0061060A00570606
:103CE0000B004C060A0042060A0038060A002E069F
:103CF0000A0024060A001A060A0010060900070630
:103D00000A00FD050900F4050900EB050900E205BC
:103D10000900D9050900D0050900C7050900BE053D
:103D20000900B5050800AD050800A50509009C05BA
:103D30000800940508008C050800840508007C052F
:103D40000800740508006C050700650508005D059E
:103D50000700560508004E05070047050700400507
:103D6000080038050700310507002A05070023056C
:103D700007001C050600160507000F0507000805CB
:103D8000060002050700FB040600F5040700EE0428
:103D90000600E8040600E2040700DB040600D50480
:103DA0000600CF040600C9040600C3040600BD04D3
:103DB0000600B7040600B1040500AC040600A60422
:103DC0000600A00405009B0406009504050090046D
:103DD00006008A04050085040500800406007A04B4
:103DE000050075040500700405006B0405006604F9
:103DF0000500610405005C04050057040500520439
:103E000005004D04050048040500430405003E0478
:103E100004003A04050035040500300404002C04B5
:103E2000050027040400230405001E0404001A04EE
:103E3000040016040500110404000D040400090424
:103E400005000404040000040400FC030400F8035B
:103E50000400F4030400F0030400EC030400E8038E
:103E60000400E4030400E0030400DC030400D803BE
:103E70000400D4030400D0030400CC030400C803EE
:103E80000300C503030024F404D9201BC40C5C0EFA
:103E90009804C4095F0265077101F405F900FB0489
:103EA000B30048048700C1036900580355000303A9
:103EB0004500BE023A008402310053022A00290262
:103EC000250004022000E4011C00C8011900AF0114
:103ED00017009801140084011300710110006101A2
:103EE000100051010E0043010D0036010B002B01A3
:103EF0000B0020010B00150109000C010900030152
:103F00000800FB000800F3000800EB000700E400D5
:103F10000600DE000600D8000600D2000600CC0035
:103F20000500C7000500C2000500BD000400B9007F
:103F30000400B5000400B1000400AD000400A900B5
:103F40000400A5000300A20003009F0004009B00E2
:103F50000300980003009500020093000300900006
:103F600003008D0002008B00030088000200860021
:103F7000020084000300810002007F0002007D0037
:103F800002007B0002007900020077000100760049
:103F900002007400020072000100710002006F0054
:103FA00002006D0001006C0002006A00010069005F
:103FB0000200670001006600010065000100640066
:103FC00002006200010061000100600001005F006A
:103FD00002005D0001005C0001005B0001005A006E
:103FE000010059000100580001005700010056006F
:103FF000010055000100540001005300000053006F
:1040000001005200010051000100500001004F006A
:1040100001004E0000004E0001004D0001004C0068
:1040200001004B0000004B0001004A000100490064
:104030000100480000004800010047000100460060
:10404000000046000100450000004500010044005A
:104050000100430000004300010042000000420054
:1040600001004100000041000100400001003F004C
:1040700000003F0001003E0000003E0001003D0046
:1040800000003D0001003C0000003C0000003C003E
:1040900001003B0000003B0001003A0000003A0034
:1040A000010039000000390001003800000038002C
:1040B0000000380001003700000037000100360022
:1040C0000000360000003600010035000000350019
:1040D000000035000100340000003400000034000E
:1040E0000100330000003300000033000100320003
:1040F00000003200000032000100310000003100F9
:1041000000003100010030000000300000003000ED
:1041100001002F0000002F0000002F0000002F00E2
:1041200001002E0000002E0000002E0001002D00D6
:1041300000002D0000002D0000002D0001002C00CB
:1041400000002C0000002C0000002C0001002B00BF
:1041500000002B0000002B0000002B0001002A00B3
:1041600000002A0000002A0000002A0001002900A7
:10417000000029000000290000002900000029009B
:10418000010028000000280000002800000028008E
:104190000000280001002700000027000000270081
:1041A0000000270000002700010026000000260074
:1041B0000000260000002600000026000100250067
:1041C000000025000000250000002500000025005B
:1041D000000025000100240000002400000024004D
:1041E0000000240000002400010023000000230040
:1041F0000000230000002300000023000000230033
:104200000000230001002200000022000000220024
:104210000000220000002200000022000100210016
:10422000000021000000210000002100000021000A
:1042300000002100000021000100200000002000FB
:1042400000002000000020000000200000002000EE
:10425000000020000000200001001F0000001F00DF
:1042600000001F0000001F0000001F0000001F00D2
:1042700000001F0001001E0000001E0000001E00C4
:1042800000001E00000020204D36303320003A0A86
:104290000020286D6D29002055004C0046696C6196
:1042A0006D656E74206C6F61642F756E6C6F6164E8
:1042B000206C656E677468733A0A00204500205AC6
:1042C0000020204D393037205800537465707065D8
:1042D00072206D6F746F722063757272656E747385
:1042E0003A0A0020204D393030204B004C696E6571
:1042F000617220416476616E63653A0A0020204D48
:10430000383531205A005A2D50726F6265204F6641
:10431000667365740020440020490020204D33302E
:104320003420500020440020490020204D333031FB
:104330002050005049442073657474696E67733A65
:104340000A0020460020420020480020204D313441
:10435000352053004D6174657269616C2068656138
:1043600074757020706172616D65746572733A0A5C
:104370000020204D3432302053004175746F2042AC
:104380006564204C6576656C696E673A0A00204565
:1043900000205A00205900205800205400205300CB
:1043A00020204D32303520420020453C6D61785F41
:1043B000655F6A65726B3E0020583C6D61785F787E
:1043C0005F6A65726B3E20593C6D61785F795F6A08
:1043D00065726B3E205A3C6D61785F7A5F6A6572E8
:1043E0006B3E00416476616E6365643A20423C6DC9
:1043F000696E5F7365676D656E745F74696D655F27
:1044000075733E20533C6D696E5F666565647261CD
:1044100074653E20543C6D696E5F74726176656CA4
:104420005F66656564726174653E002054002052C9
:104430000020204D323034205000416363656C65AC
:10444000726174696F6E2028756E6974732F733290
:10445000293A20503C7072696E745F616363656CC9
:104460003E20523C726574726163745F6163636580
:104470006C3E20543C74726176656C5F6163636569
:104480006C3E0A00204500205A0020590020204D93
:104490003230312058004D6178696D756D2041636F
:1044A00063656C65726174696F6E2028756E6974DE
:1044B000732F7332293A0A00204500205A002059F0
:1044C0000020204D3230332058004D6178696D75E1
:1044D0006D206665656472617465732028756E6908
:1044E00074732F73293A0A005374657073207065D2
:1044F0007220756E69743A0A0020204D31343920DB
:1045000043203B20556E69747320696E2043656CAF
:10451000736975730A002020473231202020203B28
:1045200020556E69747320696E206D6D004861724C
:1045300064636F6465642044656661756C742053C0
:10454000657474696E6773204C6F616465640A00FA
:10455000282300002823000064000000E803000076
:1045600000009643000096430000004100002042F6
:104570000000C9420000C9420000C8440000D24304
:10458000290A002062797465733B206372632000FE
:104590002073746F7265642073657474696E6773D9
:1045A000207265747269657665642028002028632E
:1045B000616C63756C6174656429210A0020213D7A
:1045C0002000454550524F4D20435243206D6973A2
:1045D0006D61746368202D202873746F726564297F
:1045E00020002053697A653A2000496E6465783A64
:1045F0002000204D61726C696E3D563634290A00E8
:10460000454550524F4D2076657273696F6E206D2F
:1046100069736D617463682028454550524F4D3D64
:1046200000290A002062797465733B20637263205D
:104630000053657474696E67732053746F72656498
:104640002028000A003B20454550524F4D20496E1E
:104650006465783A20005570646174696E67207AE9
:104660006F666673657420696E20454550524F4DE4
:104670003A2000454550524F4D2064617461736982
:104680007A65206572726F722E0A0050726F6269CD
:104690006E67206661696C65640A0050726F6269BA
:1046A0006E67206661696C6564005761726E696E41
:1046B000673A20486F6D696E672042756D702044BF
:1046C000697669736F72203C20310A000202044847
:1046D0006F6D652025732573257320666972737469
:1046E000002066697273740A00486F6D65200020AF
:1046F000746F6F206C6F6E67206578747275736964
:104700006F6E2070726576656E7465640A00206352
:104710006F6C6420657874727573696F6E20707247
:104720006576656E7465640A0020453A00205A3A41
:104730000020593A00583A000000F0410000F041D2
:1047400000000041FF01010000A0400000A0400067
:1047500000004000002543000045430000214300C5
:104760000040C000003E4300001F43000022430001
:10477000003E4300001F43000040C00000E0C000B6
:104780000000C020746F6F206C6F6E6720657874B6
:10479000727573696F6E2070726576656E7465648C
:1047A0000A0020636F6C6420657874727573696F9A
:1047B0006E2070726576656E7465640A006275734A
:1047C000793A2070617573656420666F7220696E36
:1047D0007075740A00627573793A2070617573653B
:1047E0006420666F7220757365720A006275737952
:1047F0003A2070726F63657373696E670A004D319A
:1048000031372050726F626520737563636573730F
:1048100066756C0A0020496E76616C696420657863
:104820007472756465722000205A3A200020593A4B
:10483000200042656420583A200050726F62652063
:104840005A204F66667365743A20003F5A206F7590
:1048500074206F662072616E676520282D32207487
:104860006F2035290A004D31343520533C696E6480
:1048700065783E206F7574206F662072616E676583
:104880002028302D31290A00436C69636B20746F36
:1048900020726573756D652E2E2E00220A00556EEE
:1048A0006B6E6F776E20636F6D6D616E643A202260
:1048B00000454550524F4D204F4B0A004E6F206D22
:1048C0006F76652E004543484F00494E464F0045E0
:1048D00052524F52530044525952554E00434F4D7D
:1048E0004D554E49434154494F4E006F666600C5D1
:1048F00048CA48CF48D648DD4844454255473A0063
:104900004C756C7A426F74204D696E69204C43443B
:10491000204F46462E00205A0020590058002020E3
:104920004D61783A2000205A00205900580020207C
:104930004D696E3A2000536F667420656E6473741F
:104940006F70733A20002569730025696D20256911
:1049500073002569682025696D2025697300256924
:1049600064202569682025696D2025697300256903
:104970007920256964202569682025696D202569CD
:1049800073005072696E742074696D653A20004D31
:104990003131332053002F2F20004361703A004300
:1049A00048414D4245525F54454D50455241545542
:1049B0005245004D4F54494F4E5F4D4F44455300B3
:1049C000544845524D414C5F50524F544543544911
:1049D0004F4E004155544F5245504F52545F53442F
:1049E0005F5354415455530050524F4D50545F53F0
:1049F0005550504F525400454D455247454E43592E
:104A00005F50415253455200434153455F4C494723
:104A100048545F4252494748544E45535300544FFF
:104A200047474C455F4C494748545300534F465401
:104A3000574152455F504F574552004255494C44EB
:104A40005F50455243454E54004C4556454C494EE7
:104A5000475F44415441005A5F50524F4245004124
:104A600055544F4C4556454C005052494E545F4AA0
:104A70004F420050524F4752455353004155544FF7
:104A80005245504F52545F54454D5000564F4C556F
:104A90004D455452494300454550524F4D004249FF
:104AA0004E4152595F46494C455F5452414E534620
:104AB00045520053455249414C5F584F4E5F584F45
:104AC0004646004649524D574152455F4E414D457D
:104AD0003A4D61726C696E20204649524D574152E1
:104AE000455F56455253494F4E3A322E302E302EA6
:104AF0003131352045585452554445525F54595030
:104B0000453A4165726F7374727564657220534FD4
:104B1000555243455F434F44455F55524C3A687484
:104B20007470733A2F2F636F64652E616C657068C3
:104B30006F626A656374732E636F6D2F6469666656
:104B40007573696F6E2F4D41524C494E2050524F34
:104B5000544F434F4C5F56455253494F4E3A312EB6
:104B600030204D414348494E455F545950453A4CD9
:104B7000756C7A426F74204D696E69204C434420F5
:104B800045585452554445525F434F554E543A315F
:104B900020555549443A30383366363866312D3021
:104BA0003238652D343934632D393865312D66320C
:104BB000653064666165653961350A0020284E6F8D
:104BC0007420796574206D65617375726564290060
:104BD000202041766572616765206D65617375722D
:104BE0006564206261636B6C61736820286D6D2958
:104BF0003A002020536D6F6F7468696E6720286DCE
:104C00006D293A2020202020202020202020202034
:104C100020202020530020204261636B6C61736868
:104C20002044697374616E636520286D6D293A2094
:104C30002020202020202000202020202028463155
:104C40002E30203D2066756C6C2C2046302E302096
:104C50003D206E6F6E65290A002020436F727265D9
:104C60006374696F6E20416D6F756E742F46616459
:104C7000652D6F75743A20202020204600616374F2
:104C80006976653A0A00696E004261636B6C617314
:104C90006820636F7272656374696F6E2069732038
:104CA00000205A0020506F736974696F6E616C2028
:104CB0004572726F723A0A004E6F7A7A6C652054B0
:104CC0006970204F757465722044696D656E7369F3
:104CD0006F6E733A0A002020546F703A2000202033
:104CE00046726F6E743A200020204C6566743A203C
:104CF000004261636B6C6173683A0A00205A00439A
:104D0000656E7465723A0A00202046726F6E743ABE
:104D1000200020204C6566743A20002020546F70DB
:104D20003A200053696465733A0A00426564204C76
:104D30006576656C696E6720004661696C65642004
:104D4000746F20656E61626C6520426564204C65FD
:104D500076656C696E670A00426564204C6576650D
:104D60006C20436F7272656374696F6E204D61745D
:104D70007269783A000A0A426564204C6576656C6F
:104D800020436F7272656374696F6E204D61747237
:104D900069783A00202B000A436F7272656374656C
:104DA0006420426564204865696768742076732EC4
:104DB0002042656420546F706F6C6F67793A0A0007
:104DC000202B000A42656420486569676874205496
:104DD0006F706F6772617068793A0A2020202B2DFE
:104DE0002D2D204241434B202D2D2B0A2020207CAD
:104DF00020202020202020202020207C0A204C2041
:104E00007C20202020282B29202020207C20520AB2
:104E10002045207C20202020202020202020207CB5
:104E200020490A2046207C20282D29204E20282B8E
:104E300029207C20470A2054207C2020202020206C
:104E400020202020207C20480A2020207C20202098
:104E500020282D29202020207C20540A2020207C5E
:104E600020202020202020202020207C0A202020FC
:104E70004F2D2D2046524F4E54202D2D2B0A2028E9
:104E8000302C30290A003474682070726F626520FB
:104E9000706F696E742C2064697374616E63652031
:104EA00066726F6D20706C616E653A200020284438
:104EB000525952554E2900473239204175746F209E
:104EC000426564204C6576656C696E67003F2028FA
:104ED0004C2C522C462C4229206F7574206F662072
:104EE000626F756E64732E0A003F50726F626520A8
:104EF000706F696E74732028592920697320696D59
:104F0000706C61757369626C652028322D32292EB0
:104F10000A003F50726F626520706F696E74732073
:104F200028582920697320696D706C6175736962F6
:104F30006C652028322D32292E0A003F285629651B
:104F400072626F7365206C6576656C206973206989
:104F50006D706C61757369626C652028302D342921
:104F60002E0A0043757272656E742066696C653A2C
:104F70002000456E642066696C65206C6973740A54
:104F800000426567696E2066696C65206C697374A0
:104F90000A00416476616E6365204B3D003F4B2003
:104FA00076616C7565206F7574206F662072616E16
:104FB00067652028302D3130292E0A004D313137D8
:104FC00020486F7420456E642048656174696E677F
:104FD0002E2E2E0A4D3130342053313730205430AC
:104FE0000A473238204F310A473120593235205A8A
:104FF00031302046353030300A4D31303920523191
:1050000037302054300A4D3131372052657769707E
:10501000696E67206E6F7A7A6C650A54300A473180
:105020002058343520593137322046353030300A57
:105030004731205A310A4D31303920523137300A48
:1050400047312058343520593137322046343030FA
:10505000300A473120583435205931373220463410
:105060003030300A4731205834352059313732201A
:1050700046343030300A47312058343520593137E2
:10508000322046343030300A4731205834352059E8
:105090003137322046343030300A473120583435E9
:1050A00020593137322046343030300A47312058C9
:1050B000343520593137322046343030300A4731C8
:1050C0002058343520593137322046343030300AB8
:1050D000473120583435205931373220463430306A
:1050E000300A473120583435205931373220463480
:1050F0003030300A4731205834352059313732208A
:1051000046343030300A4731205834352059313751
:10511000322046343030300A4731205A31350A4D7A
:105120003130362053323535200A47302058302070
:1051300059300A4D31303920523136302054300A3E
:105140004D3130370A0020466C6F773A20002064DA
:105150003A0020693A0020703A00204500205A00A9
:10516000205900204D393220580043290A0061623D
:105170006C656420286D696E2074656D7020006414
:10518000697300656E00436F6C6420657874727596
:105190006465732061726520002054002052004134
:1051A0006363656C65726174696F6E3A2050004983
:1051B0006E76616C69642065787472756465720AD4
:1051C0000020643A0020693A0020703A00536C6570
:1051D00065702E2E2E0047322F47332062616420E7
:1051E000706172616D65746572730A0050726F62EE
:1051F00065205A204F66667365743A2000446F6ECE
:105200006520736176696E672066696C652E0A0099
:1052100053442072656164206572726F720A0044A3
:105220006F6E65207072696E74696E672066696C56
:10523000650A0053544F505045442E200050726967
:105240006E7465722073746F707065642064756528
:1052500020746F206572726F72732E2046697820F9
:10526000746865206572726F7220616E6420757358
:1052700065204D39393920746F20726573746172FD
:10528000742E202854656D70657261747572652086
:1052900069732072657365742E2053657420697478
:1052A0002061667465722072657374617274696ED0
:1052B00067290A004E6F20436865636B73756D2024
:1052C00077697468206C696E65206E756D626572B1
:1052D0002C204C617374204C696E653A20004E6F2F
:1052E00020436865636B73756D2077697468206C03
:1052F000696E65206E756D6265722C204C617374E9
:10530000204C696E653A2000636865636B73756D48
:10531000206D69736D617463682C204C6173742017
:105320004C696E653A20004C696E65204E756D6261
:105330006572206973206E6F74204C617374204C09
:10534000696E65204E756D6265722B312C204C6143
:105350007374204C696E653A20004D313130005233
:105360006573656E643A20002042002050006F6B28
:1053700000220A00656E7175657565696E67202289
:1053800000504944204175746F74756E65206661E4
:10539000696C65642120426164206578747275646B
:1053A0006572206E756D6265720A004265642063E5
:1053B0006F6F6C696E672E2E2E00426564206865E3
:1053C0006174696E672E2E2E006F6B004732382095
:1053D0005A0A473020583830205931393020463366
:1053E0003030300A4D313137205072696E7420618F
:1053F000626F727465642E002020506C616E6E6561
:105400007242756666657242797465733A2000204F
:1054100046726565204D656D6F72793A2000436F65
:105420006D70696C65643A204D61792020362032B8
:105430003031390A00207C20417574686F723A203F
:1054400028416C657068204F626A656374732049F7
:105450006E632E2C204C756C7A426F7420476974F1
:10546000205265706F7369746F7279290A00002089
:105470004C61737420557064617465643A20003225
:105480002E302E302E3131350A004D61726C696E2E
:105490000020536F6674776172652052657365747E
:1054A0000A00205761746368646F672052657365F2
:1054B000740A002042726F776E206F7574205265F7
:1054C0007365740A002045787465726E616C2052B1
:1054D000657365740A00506F77657255700A0073C2
:1054E000746172740A004B494C4C45442E200050A4
:1054F00072696E7465722068616C7465642E206BCD
:10550000696C6C28292063616C6C6564210A004B0E
:10551000494C4C20636175736564206279204B4966
:105520004C4C20627574746F6E2F70696E0A004B5C
:10553000494C4C2063617573656420627920746FF7
:105540006F206D75636820696E616374697665208C
:1055500074696D65202D2063757272656E742063A9
:105560006F6D6D616E643A20004D3132310A473003
:10557000205A31300A4732382058302059300A47F3
:1055800031320A4D31303920523136300A4D313105
:10559000372050726F62696E6720626564007072B6
:1055A0006F62655F7265776970650050726F6269DE
:1055B0006E67206661696C6564004D313137204249
:1055C0006564206C6576656C696E67206661696CE0
:1055D00065642E0A4730205A31300A473020453062
:1055E0000A4D3330302050323520533838300A4D90
:1055F000333030205035302053300A4D3330302096
:1056000050323520533838300A4D33303020503541
:10561000302053300A4D333030205032352053384B
:1056200038300A47342053310070726F62655F660C
:1056300061696C65640050726F74656374656420A1
:1056400050696E0A0025301D0C1E282924311C0BC0
:10565000184527232F1B0A174443222B1A414204C3
:105660003803FF360408060600014942376FF27816
:10567000DA949DAC2EEAE200E400E00012791124F5
:105680001FBECFEFD1E2DEBFCDBF00E00CBF14E004
:10569000A0E0B2E0EEEEFCE702E00BBF02C0079034
:1056A0000D92A839B107D9F726E1A8E9B4E001C005
:1056B0001D92A839B207E1F71BE2CEE3DBE200E07E
:1056C00006C021970109802FFE010F948136C53352
:1056D000D10780E00807A9F70E946D360D94663E59
:1056E0000C9400001F920F920FB60F9211242F936B
:1056F0003F938F939F93AF93BF9380919904909121
:105700009A04A0919B04B0919C043091980423E0EA
:10571000230F2D3720F40196A11DB11D05C026E8E9
:10572000230F0296A11DB11D209398048093990424
:1057300090939A04A0939B04B0939C0480919D0441
:1057400090919E04A0919F04B091A0040196A11D88
:10575000B11D80939D0490939E04A0939F04B093E9
:10576000A004BF91AF919F918F913F912F910F9086
:105770000FBE0F901F9018952FB7F8946091990461
:1057800070919A0480919B0490919C042FBF08957E
:105790003FB7F89480919D0490919E04A0919F043E
:1057A000B091A00426B5A89B05C02F3F19F0019623
:1057B000A11DB11D3FBFBA2FA92F982F8827820F97
:1057C000911DA11DB11DBC01CD0142E0660F771FE7
:1057D000881F991F4A95D1F708958F929F92AF9293
:1057E000BF92CF92DF92EF92FF926B017C01D0DFEC
:1057F0004B015C01C114D104E104F104F1F091D337
:10580000C7DFDC01CB0188199909AA09BB09883EC9
:105810009340A105B10570F321E0C21AD108E10857
:10582000F10888EE880E83E0981EA11CB11CC114FB
:10583000D104E104F10421F7DDCFFF90EF90DF9078
:10584000CF90BF90AF909F908F900895789484B53B
:10585000826084BD84B5816084BD85B5826085BD6C
:1058600085B5816085BDEEE6F0E080818160808352
:10587000E1E8F0E010828081826080838081816035
:105880008083E0E8F0E0808181608083E1EBF0E0FC
:10589000808184608083E0EBF0E0808181608083A0
:1058A000E1E9F0E080818260808380818160808393
:1058B000E0E9F0E0808181608083E1EAF0E08081CE
:1058C00082608083808181608083E0EAF0E0808173
:1058D00081608083E1E2F1E0808182608083808169
:1058E00081608083E0E2F1E0808181608083EAE78B
:1058F000F0E0808184608083808182608083808109
:10590000816080838081806880831092C1000895C7
:105910001F93CF93DF93182FEB0161E016D12097EF
:1059200011F460E004C0CF3FD10531F461E0812F74
:10593000DF91CF911F9145C1E12FF0E0E95FFD4F6D
:10594000E4914E2F50E0FA013197E231F10508F071
:105950009DC08827EE58FF4F8F4F0D94813684B538
:10596000806884BDC7BD97C084B5806284BDC8BD52
:1059700092C080918000806880938000D0938900DD
:10598000C093880088C080918000806280938000EE
:10599000D0938B00C0938A007EC080918000886085
:1059A00080938000D0938D00C0938C0074C0809150
:1059B000B00080688093B000C093B3006CC0809149
:1059C000B00080628093B000C093B40064C0809146
:1059D0009000806880939000D0939900C0939800C5
:1059E0005AC080919000806280939000D0939B0079
:1059F000C0939A0050C0809190008860809390007E
:105A0000D0939D00C0939C0046C08091A000806808
:105A10008093A0008091A0008F7B8093A000D09302
:105A2000A900C093A80037C08091A0008062809335
:105A3000A000D093AB00C093AA002DC08091A0001D
:105A400088608093A000D093AD00C093AC0023C0C9
:105A500080912001806880932001D0932901C09318
:105A6000280119C080912001806280932001D09389
:105A70002B01C0932A010FC0809120018860809380
:105A80002001D0932D01C0932C0105C0C038D10551
:105A90000CF04CCF46CFDF91CF911F91089590E04D
:105AA000FC013197E231F10508F04EC08827EC5730
:105AB000FF4F8F4F0D948136809180008F7703C008
:105AC000809180008F7D8093800008958091800078
:105AD000877FF9CF84B58F7702C084B58F7D84BD71
:105AE00008958091B0008F7703C08091B0008F7DC2
:105AF0008093B0000895809190008F7707C08091C7
:105B000090008F7D03C080919000877F80939000EC
:105B100008958091A0008F7707C08091A0008F7DAD
:105B200003C08091A000877F8093A000089580919A
:105B300020018F7707C0809120018F7D03C0809165
:105B40002001877F809320010895CF93DF9390E019
:105B5000FC01E35BFD4F2491FC01ED56FD4F849168
:105B6000882361F190E0880F991FFC01E35FFC4FEF
:105B7000C591D491FC01ED50FD4FA591B4916111F7
:105B800009C09FB7F8948881209582238883EC917F
:105B90002E230BC0623061F49FB7F8943881822FB6
:105BA000809583238883EC912E2B2C939FBF06C076
:105BB0008FB7F894E8812E2B28838FBFDF91CF9188
:105BC00008951F93CF93DF93282F30E0F901E95F09
:105BD000FD4F8491F901E35BFD4FD491F901ED563E
:105BE000FD4FC491CC23C1F0162F811158DFEC2F4B
:105BF000F0E0EE0FFF1FED50FD4FA591B4918FB770
:105C0000F894111105C09C91ED2FE095E92302C095
:105C1000EC91ED2BEC938FBFDF91CF911F91089505
:105C2000CF93DF93282F30E0F901E95FFD4F849196
:105C3000F901E35BFD4FD491F901ED56FD4FC4919D
:105C4000CC2389F081112BDFEC2FF0E0EE0FFF1F4A
:105C5000E752FD4FA591B491EC91ED2381E090E0E6
:105C600021F480E002C080E090E0DF91CF910895C0
:105C700008951F920F920FB60F9211240BB60F9238
:105C80002F933F934F935F936F937F938F939F9344
:105C9000AF93BF93EF93FF93E0910402F09105025D
:105CA0001995FF91EF91BF91AF919F918F917F9146
:105CB0006F915F914F913F912F910F900BBE0F907D
:105CC0000FBE0F901F9018951F920F920FB60F9254
:105CD00011240BB60F922F933F934F935F936F93C3
:105CE0007F938F939F93AF93BF93EF93FF93E09135
:105CF0000602F09107021995FF91EF91BF91AF91C4
:105D00009F918F917F916F915F914F913F912F91D3
:105D10000F900BBE0F900FBE0F901F9018951F9203
:105D20000F920FB60F9211240BB60F922F933F9341
:105D30004F935F936F937F938F939F93AF93BF9393
:105D4000EF93FF93E0910802F09109021995FF91FA
:105D5000EF91BF91AF919F918F917F916F915F91E3
:105D60004F913F912F910F900BBE0F900FBE0F9050
:105D70001F9018951F920F920FB60F9211240BB619
:105D80000F922F933F934F935F936F937F938F93D4
:105D90009F93AF93BF93EF93FF93E0910A02F0912B
:105DA0000B021995FF91EF91BF91AF919F918F9148
:105DB0007F916F915F914F913F912F910F900BBE0B
:105DC0000F900FBE0F901F9018951F920F920FB655
:105DD0000F9211240BB60F922F933F934F935F9323
:105DE0006F937F938F939F93AF93BF93EF93FF93A3
:105DF000E0910002F09101021995FF91EF91BF919E
:105E0000AF919F918F917F916F915F914F913F9152
:105E10002F910F900BBE0F900FBE0F901F901895F3
:105E20001F920F920FB60F9211240BB60F922F9361
:105E30003F934F935F936F937F938F939F93AF9312
:105E4000BF93EF93FF93E0910202F0910302199543
:105E5000FF91EF91BF91AF919F918F917F916F9142
:105E60005F914F913F912F910F900BBE0F900FBEFE
:105E70000F901F9018951F920F920FB60F9211243A
:105E80000BB60F922F933F934F935F936F937F9334
:105E90008F939F93AF93BF93EF93FF93E0910C0287
:105EA000F0910D021995FF91EF91BF91AF919F91E4
:105EB0008F917F916F915F914F913F912F910F90B3
:105EC0000BBE0F900FBE0F901F9018951F920F9250
:105ED0000FB60F9211240BB60F922F933F934F934F
:105EE0005F936F937F938F939F93AF93BF93EF9342
:105EF000FF93E0910E02F0910F021995FF91EF913F
:105F0000BF91AF919F918F917F916F915F914F91D1
:105F10003F912F910F900BBE0F900FBE0F901F90CF
:105F2000189508951F93CF93DF93EC011D821C8277
:105F30001F821E82198681E0888782E28A871F86F7
:105F40001E86FE01B396CE01C1962FEF2193E8176E
:105F5000F907E1F711E018A3CE01E1D51F8B188EE8
:105F6000198E80E48A8F1B8E80E693E39AAB89AB0F
:105F7000DF91CF911F910895DB01ED91FC91199470
:105F8000EF92FF921F93CF93DF931F921F92CDB793
:105F9000DEB77C01DC01D196ED91FC91D29782E0D5
:105FA00069837A83199520E030E04AE069817A813B
:105FB000C701E2DF182FD701D196ED91FC91D2975E
:105FC00083E01995D701D196ED91FC91D29780E0AD
:105FD0001995812F0F900F90DF91CF911F91FF9016
:105FE000EF9008950F931F93CF93DF93EC018B01F4
:105FF000E9A9FAA982E01995E9A9FAA981E0199518
:1060000020E030E044E1B801CE01B6DF9E012D5C16
:106010003F4F47E1B801CE01AFDFE9A9FAA980E01F
:10602000DF91CF911F910F911994EF92FF921F93DF
:10603000CF93DF93EC017B01E9A9FAA982E01995DE
:10604000E9A9FAA981E0199520E030E045E1B7011E
:10605000CE0192DF182F882339F09E012D5C3F4F2F
:1060600047E1B701CE0188DFE9A9FAA980E01995D7
:10607000812FDF91CF911F91FF90EF900895FC0148
:10608000448F258F9C01245E3F4F42E375CFCF9311
:10609000DF931F92CDB7DEB79E012F5F3F4F46E4DF
:1060A0006BDF89810F90DF91CF910895CF93DF93BC
:1060B0001F92CDB7DEB79E012F5F3F4F47E45CDFF5
:1060C00089810F90DF91CF91089520E030E048E47E
:1060D00053CFCF93DF93EC016A817B81D8DF888334
:1060E0006A817B81CE01E2DF89836A817B81CE0177
:1060F000ECDF8B879E012D5C3F4F6A817B8147E1FE
:10610000CE01DF91CF9138CFCF93DF93EC016A813D
:106110007B8136DF882319F0CE01DBDF81E0DF9160
:10612000CF9108958F929F92AF92BF92CF92EF92AC
:106130000F93CF93DF931F921F92CDB7DEB74C0121
:106140005B012A834983EEDEF401B382A282498196
:1061500047A32A8120A705A3E4A2C3A2C4010F90EC
:106160000F90DF91CF910F91EF90CF90BF90AF90B4
:106170009F908F90C9CFFC016281738133CFCF9301
:10618000DF93EC01EE85FF85309709F019956A8160
:106190007B81CE01DF91CF9148CF362F242FFC0198
:1061A00062817381432F6BCF0F93FC0182819381B6
:1061B000648F458F278F068F9F01245E3F4F4BE3EF
:1061C000BC01CF010F91D8CEFC0160A30895BF920E
:1061D000CF92DF92EF92FF920F931F93CF93DF93B3
:1061E0006C01D62FB42EC22F7801CC2369F0F701B1
:1061F000049120E04B2D6D2FC601D6DFFFEFEF1A83
:10620000FF0AC150D85FF1CFDF91CF911F910F915D
:10621000FF90EF90DF90CF90BF9008958F929F9264
:10622000AF92BF92CF92DF92EF92FF920F931F93A4
:10623000CF93DF935C01C62EC42FD22ED02F220F16
:10624000220F220F1ED0882379F0DC0F8D2C912C89
:10625000CD1751F087012D2D4C2F6C2DC501B7DFC7
:10626000E80CF91CCF5FF4CFDF91CF911F910F9114
:10627000FF90EF90DF90CF90BF90AF909F908F9066
:1062800008950F93FC010150040F84A996A9941757
:1062900018F0081728F402C0081750F0041740F44B
:1062A0002150260F83A995A9961720F4281720F4CA
:1062B00080E007C0281720F481E0261710F0F8CFFF
:1062C00081E00F91089581E008952EE93FE0009765
:1062D00029F0F9013197F1F70197F9CF0895FC0101
:1062E000128280818150838314820895FC01808111
:1062F0009281980F92832181921760F494819F5F1D
:1063000094839381890F821710F08FEF820F83831C
:1063100081E0089580E00895FC0191E08381861773
:1063200008F490E031E0461708F030E0832F892B25
:1063300021E05281451708F420E02823832F892388
:10634000822B0895DC01FB01108212968C9112972A
:10635000818315968C9115978150828313968C9129
:1063600083830895FB0141812381213029F023306B
:1063700031F468EF640F04C0642F485F01C0642FDC
:10638000CBCFDC0115962C9115971696ED91FC91CB
:106390001797CF01820F911D820F911D1192E8175F
:1063A000F907E1F70895FC01A681B7818281481BB6
:1063B0008581483018F0A80FB11D4770382F3695E9
:1063C00036953695562F577080E890E002C0959527
:1063D00087955A95E2F7439F402D1124669566955F
:1063E0006695E62FF0E0E40FF11DEA0FFB1F308108
:1063F000222311F0832B02C080958323808308958C
:10640000FB014181DC0112962C911297421760F03A
:1064100013962C911397241738F0608115962C91C0
:10642000621710F42481BFCF0895CF92DF92FF92BC
:106430000F931F93CF93DF936C01EB01FA809B8145
:10644000913051F030F0923049F0933051F41FEF19
:1064500009C010E001E007C011E004C010E00FEF38
:1064600002C010E000E0F7FE03C0BE01C601C8DFB5
:106470009881900F98839981910F9983FF0C99F7D8
:10648000DF91CF911F910F91FF90DF90CF900895F2
:106490000F931F93CF93DF938901FB01C281D381B7
:1064A0004233D9F058F44531E1F0473109F1443134
:1064B00041F5CE0166DFCE0112DF23C04634E1F0A4
:1064C0004734E1F04B33E9F4B901CE014BDF8823C7
:1064D000C1F0B801CE01A9DF14C0B901CE0190DF2F
:1064E00010C0CE0103DF882369F0CE014ADF09C066
:1064F000B901CE0127DF05C08D8101C08981F80176
:10650000808381E0DF91CF911F910F910895CF9209
:10651000DF92EF92FF920F931F93CF93DF937C0153
:10652000D62FD42EC22F122FC62EC20E6C2D611B59
:10653000183038F00FEF20E04D2DC70135DE185030
:10654000F5CF6C2F687F6D0F2C2F277071F097E0BF
:1065500029272F5F27700FEF10E001C0000F2A9549
:10656000EAF720E04D2DC7011FDEDF91CF911F918B
:106570000F91FF90EF90DF90CF900895CF92DF9230
:10658000EF92FF920F931F93CF93DF937C01D62E50
:10659000D42FC22F122FC42EC20E4C2D411B1830E7
:1065A00038F00FEF21E06D2DC701FEDD1850F5CF5B
:1065B0004C2F487F4D0F2C2F277071F097E0292723
:1065C0002F5F27700FEF10E001C0000F2A95EAF748
:1065D00021E06D2DC701E8DDDF91CF911F910F9173
:1065E000FF90EF90DF90CF900895DF92EF92FF92AF
:1065F0000F931F93CF93DF937C01162FC42FD22EBE
:10660000D02F3FDE8823F9F02D2D4C2F612FC701AD
:106610007EDF2D2F4C2F612FC701B0DF6FEF6D0D87
:10662000610F2D2F4C2FC701A9DF4FEF4D0F4C0FDE
:106630002D2D612FC701DF91CF911F910F91FF90F9
:10664000EF90DF9064CFDF91CF911F910F91FF907A
:10665000EF90DF900895EF92FF920F931F93CF93E7
:10666000DF937C01D62F122FC42F040F212F4C2F24
:106670006D2FC7014CDFCF5F0C13F8CFDF91CF91A7
:106680001F910F91FF90EF900895DF92EF92FF928C
:106690000F931F93CF93DF93EC01162FF42EE22E6E
:1066A000F0DD882329F02E2D4F2D612FCE01D3DF71
:1066B000DF91CF911F910F91FF90EF90DF900895A0
:1066C0000895FC01E60FF11D849190E0982F882732
:1066D0003196E4918E0F911D0895FC0184910895E7
:1066E000FCDF882321F0823011F083E0089586E0FA
:1066F000089580E00895FC018081089566E0E1CF6F
:1067000068E0DFCF0A96FC01849108950B96FC01A6
:1067100084910895DC011496ED91FC9115973196C2
:1067200084910895BF92CF92DF92EF92FF920F93E0
:106730001F93CF93DF938C01E62EDC011496CD914D
:10674000DC911597CE01C9DFF82EF801848195817F
:10675000C7DFC82EF1E0FF1203C02FE0B22E02C047
:10676000BB24BA94D80114968D919C911597CADFD9
:10677000F82EF80184819581C9DFD82ED8011496AE
:106780008D919C911597BCDFB0E6BE1538F400974B
:1067900029F0C80FD91F91E6F92E0FC0F8018481A6
:1067A0009581ACDFF0E4FE1538F4009729F0C80FAE
:1067B000D91F81E4F82E01C06196DE1490F4D8014F
:1067C00050961C92509753961C92539754961C9235
:1067D000549751961C92519752961C9280E090E0EB
:1067E00066C0DF1460F38C2D90E0FE0124912F3FF2
:1067F00011F4219657C0FE104CC0D80114968D910B
:106800009C9115976ADF9E012F5F3F4FFE01882301
:1068100011F08230E1F48491D80153968C93539710
:10682000F901249154962C935497FE013396E491E8
:106830005096EC935097FE013496E4915196EC9368
:106840005197FE013596E4915296EC9320C08491C5
:10685000982F9F709250D80152969C935297829590
:106860008F7051968C935197F9012491822F8F70DC
:1068700054968C93549722952F7053962C9353973C
:10688000FE013296E491E295EF705096EC93CE01C2
:106890000EC0FE013296E491EB219C012E0F311DBA
:1068A000C20FD31FFD1409F48ACFF3949ECFDF915A
:1068B000CF911F910F91FF90EF90DF90CF90BF90FD
:1068C00008954F925F926F927F929F92AF92BF9284
:1068D000CF92DF92EF92FF920F931F93CF93DF93AC
:1068E0001F92CDB7DEB72C01C62E942E622F1ADF71
:1068F0007C01892B09F43AC0F20184819581F0DE94
:10690000B82EF201138904898189C80E8289981AE8
:10691000D92CD01A212F4D2D6C2DC201B2DC882329
:1069200011F1EB0CF11C195F169516951695612E59
:10693000712CD914C1F03C2D57018A2D8E19811765
:1069400070F4F501049120E04D2D632FC2013983CD
:106950002BDCFFEFAF1ABF0A3981385FEECFE60CB0
:10696000F71CD394E6CFF201808901C080E00F903C
:10697000DF91CF911F910F91FF90EF90DF90CF901B
:10698000BF90AF909F907F906F905F904F900895D1
:106990000F931F93CF93DF9300D0CDB7DEB78C0159
:1069A000DC015596ED91FC9156972B834A836983C0
:1069B00019954A81480F2B816981C8010F900F906A
:1069C0000F90DF91CF911F910F917BCFAF92BF922C
:1069D000DF92EF92FF920F931F93CF93DF931F925B
:1069E0001F92CDB7DEB77C01D62E042FDC01559661
:1069F000ED91FC91569729833A831995080F2981C7
:106A0000A22E3A81B32E10E0F50121915F012223DD
:106A100039F0402F6D2DC70154DFD80E180FF4CF79
:106A2000812F0F900F90DF91CF911F910F91FF90C9
:106A3000EF90DF90BF90AF900895DF92EF92FF92BA
:106A40000F931F93CF93DF937C01D62FD42E890110
:106A5000DC015596ED91FC9156971995D80EC0E042
:106A6000F8012491222349F04D2D6D2FC70129DF14
:106A7000D80FC80F0F5F1F4FF3CF8C2FDF91CF912F
:106A80001F910F91FF90EF90DF900895DC01149615
:106A90002D913C9115972115310509F43FC057966A
:106AA0008C915797F901811108C03596E491589659
:106AB000EC935897F9013C9611C0813041F43F9610
:106AC000E4915896EC935897F901709607C03D965B
:106AD000E4915896EC935897F9013E96E4915996B3
:106AE000EC93599758968C915897082E000C990B57
:106AF00059962C915997821B910927FD93955A9687
:106B00002C915A97203441F0829FC001112426E035
:106B1000969587952A95E1F75B968C93089529E7DA
:106B200033E3FC01368B258B0895CF92DF92EF92F1
:106B3000FF920F931F93CF93DF938C017B016A0128
:106B4000CB01FA011995D82F882311F1682FC801BC
:106B5000E9DDF801C189C195FFEFEF1AFF0AC7010E
:106B6000F6011995F801882351F08089C80FC701F3
:106B7000F6011995D82F682FC801D4DDEDCFD0329A
:106B800021F091898389890F01C080898C0F01C010
:106B900080E0DF91CF911F910F91FF90EF90DF90F8
:106BA000CF9008954BE753E3C0CFCF93DF93FC0121
:106BB000248135812617370741F0EC017583648302
:106BC00065DF89E793E39E8B8D8BDF91CF910895ED
:106BD0004F925F926F927F92AF92BF92CF92DF926D
:106BE000EF92FF920F931F93CF93DF93CDB7DEB752
:106BF00029013A019B01AC012419350946095709BD
:106C00008A899B89AC89BD89BC01CD016A197B0940
:106C10008C099D090F940136A801970124193509A3
:106C2000460957090F946536CA01B9016A0D7B1DE3
:106C30008C1D9D1DDF91CF911F910F91FF90EF90C3
:106C4000DF90CF90BF90AF907F906F905F904F900C
:106C5000089580E090E008950895CF92DF92EF923A
:106C6000FF920F931F93CF93DF936C017A018B01F7
:106C7000C0E0D0E0CE15DF0589F0D8016D918D011F
:106C8000D601ED91FC910190F081E02DC60119959E
:106C9000892B11F47E0102C02196ECCFC701DF9150
:106CA000CF911F910F91FF90EF90DF90CF900895BB
:106CB000DC01ED91FC910190F081E02D1994CF92CF
:106CC000EF920F93FC0113AE14AE15AE04962ADAC0
:106CD0000F91EF90CF90089508950E94262CFCDF2D
:106CE0000F946F31C0E0D0E00F94F5312097E1F3BD
:106CF0000E940000F9CFE1ECF4E083AF64AF0895A7
:106D0000EF92FF920F931F93CF93DF937A016F3F20
:106D100071058105910509F048F481EC94E0C8DF24
:106D200085EC94E0F7DC282F30E014C0C091FC041F
:106D3000D091FD044D2F50E0EC2FF0E08B019C0131
:106D4000BF0185EC94E000D6C80FC093FC04D0933B
:106D5000FD049C01C901DF91CF911F910F91FF901C
:106D6000EF900895EF92FF920F931F93CF93DF93CD
:106D70008B01C1ECD4E0FBACECAC4E2D50E06F2DA0
:106D800070E09C0185EC94E035D6F80EFBAEECAEDD
:106D9000DF91CF911F910F91FF90EF900895EF92A7
:106DA000FF920F931F93CF93DF938B01C1ECD4E03D
:106DB000FBACECAC4E2D50E06F2D70E09C0185ECEF
:106DC00094E062D6F80EFBAEECAEDF91CF911F914E
:106DD0000F91FF90EF9008956FEF7FEFC3CF4FEFCC
:106DE0005FEF8ECFCF9385E896E00E942D69C82F84
:106DF00060E870E085E896E0B5DFC53138F460E220
:106E000070E080E090E0EBDFCF5FF7CFCF910895A7
:106E10004F925F926F927F928F929F92AF92BF92AA
:106E2000CF92DF92EF92FF920F931F93CF93DF9356
:106E3000CDB7DEB72D970FB6F894DEBF0FBECDBF2E
:106E400080917B06882309F48AC06091590C709167
:106E50005A0C072E000C880B990B0F949B3311E0F2
:106E60002091550C3091560C4091570C5091580C74
:106E70000F94FC3418160CF010E06091350C7091F2
:106E8000360C072E000C880B990B0F949B33209126
:106E9000310C3091320C4091330C5091340C0F94E2
:106EA000FC3418160CF410681093B304C0906202FE
:106EB000D0906302E0906402F090650220E030E040
:106EC000A901C701B6010F94F93287FD05C020E082
:106ED00030E040E05FE304C020E030E040E05FEB02
:106EE000C701B6010F9420320F946833CB010E9482
:106EF0008387BC018EEA94E00F941D3BC09066022C
:106F0000D0906702E0906802F090690220E030E0E3
:106F1000A901C701B6010F94F93287FD05C020E031
:106F200030E040E05FE304C020E030E040E05FEBB1
:106F3000C701B6010F9420320F946833CB010E9431
:106F40008387BC0189EA94E00F941D3B8AE692E0B6
:106F50000E94658CBC0181EA94E00F941D3B0E9465
:106F60005A6A182F81E050D62091B30427FF03C03E
:106F700048E00CE002C042E102E08091F90490E0B8
:106F8000449774F48091FB04841750F027FD34C1BA
:106F90008BE496E17C0123E060E585EC94E03ED94A
:106FA0008091F9048431B0F48091FB04823090F038
:106FB000112309F424C18091500C882309F41FC1C6
:106FC0008BEB95E17C0102E123E042E068E685EC91
:106FD00094E024D98091F9048C31D0F59091B304D8
:106FE0008090550C9090560CA090570CB090580C77
:106FF000C090590CD0905A0C843128F48091FB0435
:10700000883008F033C28091F904883008F40EC249
:107010008091F9048C3108F410C28090310C90906A
:10702000320CA090330CB090340C8091350C9091C0
:10703000360C2091F904283008F405C28091F90437
:107040008C3108F407C28091F9048C3108F408C22D
:107050008091EA0883FF26C080911A07882311F1E6
:107060008091F9048433F0F48091FB048A32D0F0EB
:1070700007E028E04AE26AE285EC94E006DB05E0FE
:1070800022E04CE262E385EC94E0FFDA04E02AE0DF
:1070900041E36AE285EC94E0A8DA4BE262E385EC36
:1070A00094E07BD88091F904853328F48091FB0427
:1070B000813308F0A7C00E94046F823048F090919D
:1070C000F904943328F49091FB04923308F0A2C0A1
:1070D0008091F9048F3208F05EC08091FB04883201
:1070E00008F459C00F94902D2B013C018CE3C82E5D
:1070F000D12CE12CF12CC301B201A70196010F9410
:107100004336CA01B901A70196010F944336CA015B
:10711000062FD72E5901AE014F5F5F4F7A0150E81D
:10712000451651E5550651E06506710408F48CC01A
:10713000B90128E130E040E050E00F9443362901E6
:107140003A01DF920F93C50168E170E00F941C369D
:107150009F938F935F924F928DEA95E19F938F93C8
:10716000FF92EF920F944C3B0FB6F894DEBF0FBE28
:10717000CDBF5AE0451651046104710408F08EC079
:1071800098E0892F880F980F892F81956FE2855A93
:10719000B2DDC70121DE8091F9048632A0F480912E
:1071A000FB048E3180F008E020E84EE160E085ECE1
:1071B00094E06BDA8091F904863228F48091FB0424
:1071C0008F3108F06DC08091F904823328F48091EA
:1071D000FB048B3208F00EC18091F904813408F071
:1071E0003AC28091FB04873308F435C26EE380E035
:1071F00082DD812FF7DD2FC287E296E1CBCE81EFD2
:1072000095E1E0CE04E02AE441E366E385EC94E016
:10721000ECD951CFF8E48F9FB0011124072E000C58
:10722000880B990B0F949B332AE037ED43E25CE324
:107230000F9437350F946D33262F02E042E367E356
:1072400085EC94E022DA44CF84E6A816B10498F4E1
:10725000DF920F933F932F9383EA95E19F938F9350
:10726000FF92EF920F944C3B0FB6F894DEBF0FBE27
:10727000CDBF95E086CFDF920F933F932F938BE99D
:1072800095E19F938F93FF92EF920F944C3B0FB633
:10729000F894DEBF0FBECDBF96E073CF99E071CFFB
:1072A00060E085EC94E00E94E43065E283E023DD59
:1072B00068E570E080E090E092DD65E28BE01BDD48
:1072C000112321F08EEA94E087DD24C080911B0D0C
:1072D00080FD17C03EEAE32E34E0F32EF701619102
:1072E0007F016623B9F06F3234F4062E000C770B61
:1072F000880B990B04C06FE370E080E090E06FDDD5
:10730000EDCF80911A0D80FDDDCF6FEF7FEF8FE81D
:1073100095E145DD65E288E2EEDC69E570E080E05C
:1073200090E05DDD65E280E3E6DC112321F089EA8F
:1073300094E052DD24C080911B0D81FD17C029EA25
:10734000E22E24E0F22EF70161917F016623B9F06D
:107350006F3234F4062E000C770B880B990B04C0A7
:107360006FE370E080E090E03ADDEDCF80911A0DA0
:1073700081FDDDCF6FEF7FEF8FE895E110DD65E2F6
:107380008DE4B9DC6AE570E080E090E028DD65E23C
:1073900085E5B1DC112321F081EA94E01DDD24C0F4
:1073A00080911B0D82FD17C091EAE92E94E0F92E21
:1073B000F70161917F016623B9F06F3234F4062E34
:1073C000000C770B880B990B04C06FE370E080E032
:1073D00090E005DDEDCF80911A0D82FDDDCF6FEFDE
:1073E0007FEF84E995E1DBDC61E085EC94E00E94CD
:1073F000E430E9CE83E008D462E383E07CDC66E03D
:1074000070E080E090E0EBDC81E0FED362E38CE0B2
:1074100072DC80915C0290915D020E944D87DCDC01
:1074200065E270E080E090E0DADCD6CE8091480C36
:1074300011112DC08111ECCD2AC08091FB04853142
:1074400008F059C0EACD2091240C111184C02111FB
:10745000F5CD81C08091FB04853108F0B0C0F3CD3B
:107460008091FB04853108F0DAC0F2CD90FD03C0B5
:1074700081E596E102C089E696E17C010CE022E01C
:1074800048E068E085EC94E00E940E31BCCDB60186
:10749000DD0C880B990B0F949B3320E030E040E02B
:1074A0005FE30F9420320F946833CB010E944D8725
:1074B0007C01FC0180818032E1F4F701818180321E
:1074C00011F401E001C002E0902F990F900F892F75
:1074D000819567E0815F0FDC83E090E0801B91097C
:1074E0008E0D9F1D79DC69E070E080E090E077DC34
:1074F0008FCD03E0E9CF20E030E040E05FE3C5015D
:10750000B4010F9420320F946833CB010E944D8751
:107510007C01FC0180818032E1F4F70181818032BD
:1075200011F401E001C002E0902F990F900F892F14
:1075300081956CE1815FDFDB83E090E0801B910946
:107540008E0D9F1D49DC69E070E080E090E047DC33
:1075500064CD03E0E9CFBC01990F880B990B0F9420
:107560009B3320E030E040E05FE30F9420320F9443
:107570006833CB010E944D877C01FC018081803201
:10758000E1F4F7018181803211F401E001C002E0F1
:10759000902F990F900F892F819567E0845AABDB6C
:1075A00083E090E0801B91098E0D9F1D15DC69E042
:1075B00070E080E090E013DC41CD03E0E9CF20E013
:1075C00030E040E05FE3C501B4010F9420320F9436
:1075D0006833CB010E944D877C01FC0180818032A1
:1075E000E1F4F7018181803211F401E001C002E091
:1075F000902F990F900F892F81956CE1845A7BDB36
:1076000083E090E0801B91098E0D9F1DE5DB69E012
:1076100070E080E090E0E3DB16CD03E0E9CF00917D
:10762000500C002309F414CD6CE187E664DBF4E62A
:107630000F9FC001112481589F4F6FEF70E00F948E
:107640003036CB010E944D87C7DB65E270E080E0F9
:1076500090E0C5DBFDCC2D960FB6F894DEBF0FBED3
:10766000CDBFDF91CF911F910F91FF90EF90DF90F1
:10767000CF90BF90AF909F908F907F906F905F90D2
:107680004F9008950F931F93CF93DF93CDB7DEB73D
:1076900028970FB6F894DEBF0FBECDBF8A0123E056
:1076A000660F771F2A95E1F7680F791F48E050E0D1
:1076B000CE0101960F94803A29813A81F8018081A8
:1076C00091812817390790F08217930760F09C8109
:1076D0008281981758F081E090E03B812381231745
:1076E00038F080E005C081E090E002C08FEF9FEFAE
:1076F00028960FB6F894DEBF0FBECDBFDF91CF91B5
:107700001F910F910895EF92FF920F931F93CF93C4
:10771000DF93EC018B017A018A859B858617970799
:1077200029F08881998141DA1B870A8788859985A4
:10773000019681F00E811F81B7018881998132DA2B
:10774000080F111D888599858017910718F481E02D
:1077500090E010C06E818A81680F97014C8188810A
:10776000998134D92E813F81280F311D3F832E838B
:1077700080E090E0DF91CF911F910F91FF90EF900B
:1077800008954F925F926F927F928F929F92AF92E5
:10779000BF92CF92DF92EF92FF920F931F93CF93FE
:1077A000DF93CDB7DEB72D970FB6F894DEBF0FBECF
:1077B000CDBF6C012A013B01490158011B861C8683
:1077C000CE0101967C0188E0F70111928A95E9F7D4
:1077D000DB01CA0127E0B695A795979587952A956D
:1077E000D1F79A838983F42FFF77FD878F2F8058F5
:1077F0008B838C831A8619864F3F5105610571056D
:1078000009F018F460E070E026C06091B604709151
:10781000B7048E01075F1F4F970142E45BE380913D
:10782000B4049091B5040E947E6797FDEBCF698503
:107830007A8583E0660F771F8A95E1F78091B4041B
:107840009091B504680F791F48E050E0C7010F948C
:10785000803A6F8178856115710519F44B86B60100
:1078600006C0C616D70619F08D8580688B87AE01D5
:10787000455F5F4FC401F50119952D960FB6F89439
:10788000DEBF0FBECDBFDF91CF911F910F91FF9053
:10789000EF90DF90CF90BF90AF909F908F907F90B0
:1078A0006F905F904F9008956F927F928F929F920A
:1078B000AF92BF92CF92DF92EF92FF920F931F93FE
:1078C000CF93DF9300D01F92CDB7DEB76C017B0161
:1078D0003A015901480119821A821B821C82AE01A9
:1078E0004F5F5F4FB301C7010E94DE677C01498192
:1078F0005A816B817C81411551056105710529F023
:1079000084019501C6013DDFE6CF0F900F900F90E7
:107910000F90DF91CF911F910F91FF90EF90DF902B
:10792000CF90BF90AF909F908F907F906F90089571
:1079300021E02093B804E4EBF4E091838083738327
:10794000628380E090E008957F92AF92BF92CF92E1
:10795000DF92EF92FF920F931F93CF93DF93CDB7F8
:10796000DEB72C970FB6F894DEBF0FBECDBF6C010B
:10797000762EF72F842FE52FB901A801D601149692
:10798000AD90BC9015979091B804911109C021EC6D
:1079900036E1482F672DC60150D880E090E018C02E
:1079A000DA82C9827B82FC838D83EE8318861F82F4
:1079B000FA86E9861C861B8603E81BE39E012F5F7F
:1079C0003F4FC501DEDEB501C601EFD88F81988536
:1079D0002C960FB6F894DEBF0FBECDBFDF91CF91CE
:1079E0001F910F91FF90EF90DF90CF90BF90AF90DD
:1079F0007F900895CF92DF92EF92FF920F931F93A3
:107A0000CF93DF93CDB7DEB72C970FB6F894DEBFD8
:107A10000FBECDBF7C01C901F701C480D580209184
:107A2000B804211107C021EA36E1C70106D880E079
:107A300090E01BC0FA82E9826B837C834D835E8376
:107A400018861F821A8709871C861B8603E81BE39A
:107A50009E012F5F3F4F48E757E6BC01C60124DF78
:107A6000B601C701A2D88F8198852C960FB6F894DD
:107A7000DEBF0FBECDBFDF91CF911F910F91FF9061
:107A8000EF90DF90CF900895CF92DF92EF92FF9228
:107A90000F931F93CF93DF93CDB7DEB72C970FB61D
:107AA000F894DEBF0FBECDBF7C01C901F701C480D1
:107AB000D5802091B804211108C021E836E1C70122
:107AC0000E941D3580E090E01BC0FA82E9826B8342
:107AD0007C834D835E8318861F821A8709871C86E4
:107AE0001B8603E81BE39E012F5F3F4F4BE757E6E2
:107AF000BC01C601D9DEB601C70157D88F81988570
:107B00002C960FB6F894DEBF0FBECDBFDF91CF919C
:107B10001F910F91FF90EF90DF90CF900895CF933A
:107B2000DF93EC01262F4CAD6BAD04960E94C83458
:107B30002BAD082E000C990B820F911D8BAF81E0AD
:107B400090E0DF91CF9108950F939CE0899F802D65
:107B5000112421E0280F2093C004845F8093BF0488
:107B600090E002964091F90450E08417950714F4D0
:107B700080E033C0822F90E02091FB0430E0821738
:107B80009307B4F76623A9F061E085EC94E00E94C6
:107B9000E4304091C0044E5F0BE020E860E085ECEB
:107BA00094E00E94453360E085EC94E00E94E4306C
:107BB00005C061E085EC94E00E94E4306091BF0470
:107BC0008091F9046817A0F29091C0048091FB04A1
:107BD000891770F280E08FD881E00F910895CF93DC
:107BE000DF93FC0185ADEF012496811105C081E092
:107BF00085AFCE010E948430CE01DF91CF910C94ED
:107C0000BB306FEF7FEFCBC8482F50E02091BE0410
:107C1000022E000C330B4217530781F08093BE04F1
:107C2000813031F46BE271E285EC94E00C94D5354F
:107C30006CEA77E185EC94E00C94D5350895EF92E9
:107C4000FF920F9381EC94E0CADF8DEEE82E8EE177
:107C5000F82E00E428E040E060E085EC94E00E942B
:107C60000E3167E273E085EC94E00E94D53523E4A1
:107C700033E041E169E385EC94E00E94E63467E992
:107C80007BE085EC94E00E94D53528E433E04CE1BC
:107C90006AE385EC94E00E94E63462EF7EE085ECD6
:107CA00094E00E94D53524E533E049E26BE385ECAE
:107CB00094E00E94E63462EF7EE085EC94E00E945E
:107CC000D53520E633E04EE36DE385EC94E00E9489
:107CD000E63422E633E04EE362E485EC94E00E9471
:107CE000E63485EC94E00E94BF308111AECF64ECA5
:107CF00079E080E090E00E94B4866CEA77E185EC60
:107D000094E00F91FF90EF900C94D53561E08DEEEB
:107D10009EE195DF64EC79E080E090E00C94B4861D
:107D2000EF92FF920F93F2DF81EC94E058DF89ED40
:107D3000E82E8CE1F82E06E22EE040E068E085ECCB
:107D400094E00E940E3183E05FDF22E633E040E3FF
:107D500065E285EC94E00E94E6342CE633E04CE3E7
:107D600067E085EC94E00E94E63485EC94E00E94A4
:107D7000BF308111DCCF64EC79E080E090E00F91BE
:107D8000FF90EF900C94B48660E070E08BE291E29B
:107D9000CFCD1F93CF93DF93C091C604C695C695F0
:107DA00081EC94E01CDFDC2FDD0F1D2F1C0F83E026
:107DB0002BDF6C2F80E00E947B3685E896E00CD8A4
:107DC0006D2F80E00E947B368EEE96E11ADF612FE8
:107DD00080E00E947B3681EE96E113DF85EC94E033
:107DE0000E94BF308111E3CFDF91CF911F910895A1
:107DF0000895CF93E62F6CE0869F602D112481E0DB
:107E0000860F8093C004645F6093BF04462F50E0E8
:107E10004E5F5F4F2091F90430E0421753070CF496
:107E20004CC090E02091FB0430E0821793070CF0E7
:107E300044C0CE2F8EE30E947B3665E470E080E084
:107E400090E00E94EF3661E36C0F062E000C770B7A
:107E5000880B990B0E94EF3660E270E080E090E0C2
:107E60000E94EF366091550C7091560C8091570C22
:107E70009091580C0F946833CB010E944D870E945B
:107E8000EC366FE270E080E090E00E94EF360E94F6
:107E90005A6A811109C085E0C89FF0011124EC5B8A
:107EA000F34F8481811109C08091590C90915A0C33
:107EB0000E944D87CF910C94EC36CF910895CF92CC
:107EC000DF92EF92FF920F931F93CF93DF931F9256
:107ED0001F92CDB7DEB77B01622F498335DE498122
:107EE000882309F444C0442311F101151105F9F464
:107EF000C7010E944E6925E130E0281B310937FF98
:107F000002C02F5F3F4F3595279530E82158822FCB
:107F1000830F87FD0DC060E270E080E090E02A836F
:107F200039830E94EF36398131502A81F0CF30E811
:107F3000C32ED12CB601C7010E94CF367601E81AB4
:107F4000F90A0115110511F41E2D07C0FF24B70110
:107F5000C8010E94B2361E2D181B173040F060E297
:107F600070E080E090E00E94EF36181BF6CF0F9093
:107F70000F90DF91CF911F910F91FF90EF90DF90C5
:107F8000CF9008950F93CF93DF93982F862FEA0118
:107F9000692FDADD882331F162E770E0CE010E94BB
:107FA000CF36C2E7C81BC73040F060E270E080E027
:107FB00090E00E94EF36C81BF6CF6091BF048AE7BD
:107FC0000E947B36602F000F770B880B990B0E9465
:107FD000EF3660E270E080E090E0DF91CF910F91AA
:107FE0000C94EF36DF91CF910F910895CF92DF92ED
:107FF000EF92FF920F931F93CF93DF93982F862FCB
:108000006A017901692FA0DD882309F447C0C701FF
:10801000002321F00E944E69182F03C00E942D6991
:10802000182FC3E1D0E0C11BD1098C2F880FC80FD6
:10803000CC0FD0E0BE01C6010E94CF36C81B6AE358
:1080400070E080E090E00E94EF36C73040F060E2E0
:1080500070E080E090E00E94EF36C81BF6CF8AEF18
:10806000189F802D11246091BF0480580E947B3698
:10807000C701002349F0DF91CF911F910F91FF902D
:10808000EF90DF90CF90BDCDDF91CF911F910F91F9
:10809000FF90EF90DF90CF900C94EC36DF91CF9172
:1080A0001F910F91FF90EF90DF90CF900895BF92B6
:1080B000CF92DF92EF92FF920F931F93CF93DF93B4
:1080C0006C017B010E944E69C82FC7010E942D6977
:1080D00003E110E0081B11098C2F90E0BB24B3943E
:1080E000081719071CF0B12CC5E201C0CFE12C2FF5
:1080F00030E0A9014E5F5F4F8091F90490E048178E
:10810000590744F0295031098091FB0490E082170F
:108110009307BCF5D0E0E114F104D9F16AE370E013
:1081200080E090E00E94EF36BB2081F0C45F809138
:10813000F904C81770F12C2F30E0295031098091D3
:10814000FB0490E0821793071CF423C0DD2309F1A0
:10815000802F880F800F6C2F880F0E947B3660E283
:1081600070E080E090E00E94EF36C701DF91CF9190
:108170001F910F91FF90EF90DF90CF90BF900C94E4
:10818000EC366C2F80E00E947B36C6013ADDD1E0F0
:10819000C2CFDF91CF911F910F91FF90EF90DF90B1
:1081A000CF90BF900895CF92DF92EF92FF920F93FE
:1081B0001F93CF93DF931F92CDB7DEB7182F7A01AD
:1081C000D22ECA0169830E944E69082F812F880F21
:1081D000810FC82ECC0C1CE06981169F100D112454
:1081E000DD20C1F061E085EC94E00E94E430202FB6
:1081F000220F200F220F2E5F0BE047EF410F6FEF92
:108200006C0D85EC94E00E94453360E085EC94E0D1
:108210000E94E430612F8C2D0E947B36C701F1DC77
:10822000DD2071F061E085EC94E00F90DF91CF915B
:108230001F910F91FF90EF90DF90CF900C94E4305E
:108240000F90DF91CF911F910F91FF90EF90DF90F2
:10825000CF9008958F929F92AF92BF92DF92EF924C
:10826000FF920F931F93CF93DF93EC015B01D42E0A
:1082700049016CE080E00E947B36C401C2DC01153C
:10828000110521F0B80181E00E94146AE114F104A3
:1082900011F0C701B6DC91E02D2D2927A50164E07E
:1082A00081E081DFCE010E944E692D2DAE0164E098
:1082B00094E1981B892FDF91CF911F910F91FF902F
:1082C000EF90DF90BF90AF909F908F906CCFEF9228
:1082D000FF920F93CF93DF93D82FC62F7901682F8A
:1082E0008C2F32DC8823F1F0002331F062E070E063
:1082F00080E090E00E94EF362D2F4C2F64E1C70103
:108300000E94C56968E770E00E94B236C8E7C81BE2
:10831000C73040F060E270E080E090E00E94EF360D
:10832000C81BF6CFDF91CF910F91FF90EF9008958A
:108330008F929F92AF92BF92CF92DF92EF92FF9275
:108340000F936B017C018090BA049090BB04A090C5
:10835000BC04B090BD04A50194010F94F9328823A8
:1083600001F120E030E0A901C701B6010F94F93214
:10837000882351F0A5019401C701B6010F94F93289
:1083800087FD04C081E003C080E001C08FEF8093CF
:10839000B904C092BA04D092BB04E092BC04F0923B
:1083A000BD048091F904813128F48091FB0483306D
:1083B00008F048C08091F904853128F48091FB04CD
:1083C000843108F04FC08091F9048F3308F057C012
:1083D0008091FB048F3208F452C08CE4E82E87E1D0
:1083E000F82E00E123E04FE265E085EC94E00E9486
:1083F0000E319CE7E92E97E1F92E23E04FE26AE582
:1084000085EC94E00E940E318091B90440E3481B52
:1084100022E3E22E27E1F22E0DE022E06EE685EC6B
:1084200094E00E940E318091B90441E3481B38E189
:10843000E32E37E1F32E22E069E185EC94E00E941F
:108440000E311DC08091B90444E0481B5DEFE52E5C
:1084500056E1F52E0CE022E062E485EC94E00E9407
:108460000E31A8CF45E1E42E47E1F42E01E023E0F0
:1084700044E16CE385EC94E00E940E31A4CF0F91AF
:10848000FF90EF90DF90CF90BF90AF909F908F9034
:108490000895CF92EF920F93CF93DF93C1ECD4E086
:1084A0001B821A8284E893E099838883CC24CA943F
:1084B000EE24EA9402E522E143E160E172E0CE01BC
:1084C0000E945F3680E993E099838883DF91CF91A2
:1084D0000F91EF90CF9008955A9887FD52C05B9806
:1084E00000000000000000005A9A5A98282F220F1E
:1084F00086FD53C05B9800000000000000005A9AFF
:108500005A98922F990F26FD46C05B9800000000F4
:10851000000000005A9A5A98892F880F96FD39C09A
:108520005B9800000000000000005A9A5A98982FAB
:10853000990F86FD2CC05B98000000000000000031
:108540005A9A5A98892F880F96FD1FC05B98000091
:108550000000000000005A9A5A98982F990F86FD43
:1085600012C05B9800000000000000005A9A5A9860
:1085700096FD15C05B9800000000000000005A9AAC
:1085800008955B9AADCF5B9AEDCF5B9AE0CF5B9A93
:10859000D3CF5B9AC6CF5B9AB9CF5B9AACCF5B9ACD
:1085A000EACF2F923F925F927F929F92AF92BF92BB
:1085B000CF92DF92EF92FF920F931F93CF93DF93AF
:1085C0007C011B01942E69018AE0481709F47BC0E5
:1085D000A5E14A134EC0DB011296ED91FC91139771
:1085E0001281C681D7815D9A88E28A950000E9F7F9
:1085F00000EE010F80E1582E510E98E2792E88EF9F
:108600006BDF872D8A950000E9F7103208F046C02D
:10861000812F8077806860DF812F8295807F5CDF8B
:10862000872D8A950000E9F780E856DF80E054DF67
:10863000872D8A950000E9F78AEF4EDF872D8A950E
:108640000000E9F75E01B0E1AB0EB11C8881807FCC
:1086500043DF89918295807F3FDFCA15DB05B1F743
:10866000872D8A950000E9F71F5F0F5F1511C7CFAF
:108670005D989601492DB101C701DF91CF911F91FE
:108680000F91FF90EF90DF90CF90BF90AF909F90B1
:108690007F905F903F902F900C944832802F80778E
:1086A00080681ADF802F8295807F16DF872D8A955C
:1086B0000000E9F780E810DF80E80EDF872D8A955B
:1086C0000000E9F7B9CF559A5D98539A5B98529A92
:1086D0005A9A5D9AC8E28C2F8A950000E9F788E7DC
:1086E00090E00E94653188EFF7DE8C2F8A950000BC
:1086F000E9F780E2F1DE80E0EFDE8C2F8A95000062
:10870000E9F780E0E9DE80E8E7DE8C2F8A9500005B
:10871000E9F780E0E1DE80E1DFDE8C2F8A95000062
:10872000E9F78FE090E00E94653180E2D5DE80E4D9
:10873000D3DE8C2F8A950000E9F780E2CDDE80E65B
:10874000CBDECA950000E9F710E0D8E208E2812FFD
:1087500080778068C1DE812F8295807FBDDE8D2F7E
:108760008A950000E9F780E8B7DE80E0B5DE8D2F5E
:108770008A950000E9F78AEFAFDE8D2F8A95000019
:10878000E9F7C0E280E0A8DE80E0A6DE9D2F9A95A2
:108790000000E9F7C150B1F788EF9EDE802F8A957F
:1087A0000000E9F71F5F103209F0D1CF80E094DEBE
:1087B00080EC92DE88E28A950000E9F75D9859CF57
:1087C000CF93DF931F921F92CDB7DEB789839A8331
:1087D0000E942B6520E040E060E070E089819A8192
:1087E0000F900F90DF91CF910C94AE65EF92FF92B6
:1087F0000F931F9380911E028823B9F080919B08EC
:10880000811103C00DED18E002C00BE918E086E607
:10881000E82E8AE2F82E29E53AE24FEF55E062E5CC
:108820007AE28CE49AE20E945A670E940F6A8823D7
:10883000B1F08091FF05882361F08DED98E00E94F2
:1088400061730E94D3651F910F91FF90EF900C947C
:10885000E46E1F910F91FF90EF900C94DA651F91D9
:108860000F91FF90EF9008950E94B17721E030E0E2
:10887000811102C020E030E030937A06209379061F
:108880001092530681E080931F0683E080931E02BE
:108890000895CF92DF92EF92FF920F931F93CF93A1
:1088A000DF930E94AE786C0161E081E00E94576620
:1088B000C0915306D0E081E0C81AD108C11117C099
:1088C00080915206811104C00E940F6A811195C0E7
:1088D00080911E02882359F081E0909152069111F7
:1088E00080E004E024E047E45AE26D2F4BDB6DEDBD
:1088F00078E084E698E00E94977E8091DD088F32D0
:1089000001F18091EA0883FF1CC0C130C1F480915D
:108910005206813021F40E940F6A811176C0809145
:108920001E02882361F081E090915206913009F097
:1089300080E000E22EE343E45AE26D2F23DB92E075
:1089400001C091E080911E02882309F44EC0760197
:1089500011E01C0F8FEFE816F80609F446C0C913A2
:108960003FC060E070E0C7010E94D6749091EA08B1
:108970008091520694FF1CC08C134EC00E940F6A57
:10898000882309F449C08DED98E00E945B7710922E
:10899000530682E090E090937A068093790681E016
:1089A00080931F0610927C0683E080931E0254C0C1
:1089B0008C1304C00E940F6A81113DC080911E0279
:1089C000882361F081E0909152069C1380E000E0E2
:1089D00021E936E147E25AE26D2F79DC912F01C09F
:1089E0009F5F81E0E81AF108B5CFDF5FCF5FD53038
:1089F00009F064CF909351062FC00E94DA658091F0
:108A00001F06882309F464CF27C02EDF80911F063C
:108A1000882309F484CF20C080911E028823F1F2BC
:108A200081E0909152069C1380E001E021E936E15B
:108A300045E35AE2D1CF1092FF050E942B6520E05A
:108A400040E060E070E086EF93E40E94AE658091C4
:108A50001F06882309F4B2CFDF91CF911F910F91A8
:108A6000FF90EF90DF90CF900895FC016083089510
:108A7000CF93DF93EC01072E000C880B990B0F941A
:108A80009B332FE632E143E85AE30F94373568838E
:108A900079838A839B83DF91CF91089565E375E4A1
:108AA0008AE595E40C94EF6568E375E482E795E464
:108AB0000C94EF650C94F886CF93DF9300D01F924F
:108AC000CDB7DEB769837A838B839C8360E2CE0166
:108AD00001960E9402890F900F900F900F90DF91E6
:108AE000CF910895BC01990F880B990B0F949B337C
:108AF0002FE632E143E85AE30F943735DDCF2F926A
:108B00003F924F925F926F927F928F929F92AF921D
:108B1000CF92DF92EF92FF920F931F93CF93DF9349
:108B200000D01F92CDB7DEB74C011B01CA01B901BD
:108B3000E982FA820B831C8320E030E04AE754E4A8
:108B40000F9437350F9468332B013C0120E030E05F
:108B50004AE754E4F10160817181828193810F942D
:108B600037350F9468338B010419150920E030E084
:108B70004AE754E469817A818B819C810F9437356F
:108B80000F9468339B012419350984E5E82E85E4A8
:108B9000F82EA201B101C4010E9452650F900F90FE
:108BA0000F900F90DF91CF911F910F91FF90EF9059
:108BB000DF90CF90AF909F908F907F906F905F905D
:108BC0004F903F902F900895AF92CF92DF92EF9207
:108BD000FF920F931F93CF93DF9361E081E00E9498
:108BE0005766D0915306C0E0D11119C0809152064A
:108BF000811104C00E940F6A8111C4C080911E02BD
:108C0000882309F4B6C081E090915206911180E06A
:108C100004E024E04EE95AE26C2FB4D9AAC0D13066
:108C2000E1F480915206813021F40E940F6A811193
:108C3000B1C080911E02882309F49BC011E080918D
:108C40005206813009F010E08091C7130E94F88627
:108C500000E09C0148E85AE289C0D23009F58091D1
:108C60005206823021F40E940F6A8111B0C08091B7
:108C70001E02882309F47DC011E0809152068230E3
:108C800009F010E06091C8137091C9138091CA1364
:108C90009091CB1311DF00E09C0144E85AE266C0DA
:108CA000D33009F580915206833021F40E940F6A77
:108CB0008111A6C080911E02882309F45AC011E0D8
:108CC00080915206833009F010E06091CC137091CE
:108CD000CD138091CE139091CF13EEDE00E09C0176
:108CE00040E85AE243C0D43001F580915206843006
:108CF00021F40E940F6A81119CC080911E0288237A
:108D0000C1F111E080915206843009F010E06091C9
:108D1000D0137091D1138091D2139091D313CCDEE4
:108D200000E09C014CE75AE221C0D53011F580915A
:108D30005206853021F40E940F6A811193C0809100
:108D40001E028823B1F011E080915206853009F0AF
:108D500010E06091790270917A0280917B0290918B
:108D60007C02AADE00E09C0148E65AE26C2F812FCB
:108D70003DD9CF5FDF5FC53009F036CF86E0809305
:108D8000510688C00E94DA6580911F06882309F485
:108D900035CF80C081E00E94046A0091C71310E0C3
:108DA000A12CC12CD12C4EE4E42E45E4F42E2FEF5F
:108DB00030E040E050E067EC73E183E99AE20E9422
:108DC000526580911F06882309F433CF63C081E088
:108DD0000E94046AA12CC12CD12C16E6E12EFE2C97
:108DE0000EE111E420E030E0A90168EC73E186E8CF
:108DF0009AE285DE80911F06882309F438CF4AC0A5
:108E000081E00E94046AA12CC12CD12C16E6E12E2F
:108E1000FE2C0EE111E420E030E0A9016CEC73E1DE
:108E200082E89AE26CDE80911F06882309F442CF23
:108E300031C081E00E94046AA12CC12CD12C16E61D
:108E4000E12EFE2C0EE111E420E030E0A90160EDFE
:108E500073E18EE79AE253DE80911F06882309F4BE
:108E60004CCF18C081E00E94046AA12CC12CD12CE7
:108E700016E6E12EFE2C0EE111E420E030E0A9011F
:108E800069E772E082E79AE23ADE80911F06882362
:108E900009F455CFDF91CF911F910F91FF90EF9083
:108EA000DF90CF90AF900895CF93DF93EC01072E22
:108EB000000C880B990B0F949B3320E030E048ECBA
:108EC00052E40F9437350F946D33688379838A8326
:108ED0009B83DF91CF910895CF93DF93EC01072E11
:108EE000000C880B990B0F949B332AE037ED43E27B
:108EF0005CE30F943735688379838A839B83DF91A2
:108F0000CF910895CF93DF93EC01072E000C880BCF
:108F1000990B0F949B33688379838A839B83DF91BA
:108F2000CF910895CF93DF93EC01072E000C880BAF
:108F3000990B0F949B3320E030E048EC52E40F94FF
:108F40003735688379838A839B83DF91CF91089536
:108F5000CF93DF93EC01072E000C880B990B0F9435
:108F60009B332AE037ED43E25CE30F9437356883A7
:108F700079838A839B83DF91CF910895CF93DF9389
:108F8000EC01072E000C880B990B0F949B332AE001
:108F900037ED43E25CE30F943735688379838A8346
:108FA0009B83DF91CF91089564E577E483EC98E4A7
:108FB0000C94EF656CE677E48DE198E40C94EF6532
:108FC00062E877E483EA98E40C94EF6562E977E479
:108FD0008EE398E40C94EF6568EA77E48FE598E413
:108FE0000C94EF656EEB77E48CEF97E40C94EF65EF
:108FF0000C94BDE90C9404EACF93DF9300D01F9248
:10900000CDB7DEB7BC01990F880B990B0F949B333A
:109010002AE037ED43E25CE30F94373569837A83C6
:109020008B839C83CE0101960E94A48B0F900F909E
:109030000F900F90DF91CF910895CF93DF9300D0E1
:109040001F92CDB7DEB7BC01990F880B990B0F9417
:109050009B332AE037ED43E25CE30F9437356983B5
:109060007A838B839C83CE0101960E94EC870F90BC
:109070000F900F900F90DF91CF910895CF93DF93D2
:1090800000D01F92CDB7DEB7BC01990F880B990BAA
:109090000F949B3320E030E048EC52E40F943735D6
:1090A00069837A838B839C83CE0101960E944B8ACD
:1090B0000F900F900F900F90DF91CF910895CF9365
:1090C000DF9300D01F92CDB7DEB7BC01990F880B9C
:1090D000990B0F949B332AE037ED43E25CE30F9446
:1090E000373569837A838B839C83CE0101960E94F6
:1090F000038B0F900F900F900F90DF91CF910895F9
:10910000CF92DF92EF92FF926B017C0120E030E082
:10911000A9010F94F93287FD05C020E030E040E05E
:109120005FE304C020E030E040E05FEBC701B60140
:109130000F9420320F946833CB01FF90EF90DF90B3
:10914000CF900C944D87BC01990F880B990B0F940D
:109150009B33D6CFCF93DF9300D01F92CDB7DEB72E
:109160000F946D330F94993369837A838B839C8337
:10917000CE0101960E944B8A0F900F900F900F9096
:10918000DF91CF910895BC01990F880B990B0F9433
:109190009B3320E030E048EC52E40F943735DACFCF
:1091A0000F931F93CF93DF9361E081E00E94576696
:1091B000C0915306D0E0C1111AC0809152068111AE
:1091C00004C00E940F6A8111E8C080911E028823AA
:1091D00009F461C081E090915206911180E004E0B1
:1091E00024E048EE5AE26D2F0E94C23F54C0C130C5
:1091F000D9F480915206813021F40E940F6A8111C6
:10920000D4C080911E02882309F445C081E090916A
:109210005206913009F080E003E02EE34FED5AE270
:109220006D2F0E94C23F37C0C230D1F480915206E8
:10923000823021F40E940F6A8111C0C080911E0209
:10924000882349F181E090915206923009F080E044
:1092500003E02EE342ED5AE26D2F0E94C23F1BC095
:10926000C330C9F480915206833021F40E940F6A02
:109270008111ADC080911E02882369F081E0909138
:109280005206933009F080E003E02EE34DEC5AE201
:109290006D2F0E94C23F0E94976581111DC0C4308E
:1092A000E9F480915206843021F40E940F6A811102
:1092B00097C080911E02882309F49BC081E09091A1
:1092C0005206943009F080E003E02EE344EC5AE2C9
:1092D0006D2F0E94C23F8DC014E001C015E0C11384
:1092E0001BC0809152068C1304C00E940F6A81112A
:1092F00082C080911E02882371F081E09091520615
:109300009C1380E003E02EE34BEB5AE26D2F0E94AA
:10931000C23F1C2F01C01C2F81E0810FC81318C051
:10932000809152068C1304C00E940F6A81116CC098
:1093300080911E02882361F081E0909152069C1377
:1093400080E003E02EE34CEA5AE26D2F0E94C23F18
:1093500082E0810FC81318C0809152068C1304C09C
:109360000E940F6A811159C080911E02882361F00A
:1093700081E0909152069C1380E003E02EE343EAE3
:109380005AE26D2F0E94C23FDF5FCF5FD53009F0F8
:1093900012CF1D5F1093510648C00E94DA6580917C
:1093A0001F06882309F411CF40C08CE09DE408DA41
:1093B00080911F06882309F424CF37C08AEA90E5FC
:1093C000FFD980911F06882309F438CF2EC084ED81
:1093D0009EE4F6D980911F06882309F44BCF25C05F
:1093E0008EE593E5EDD980911F06882309F461CFBE
:1093F0001CC015E091CF84EE95E4E2D980911F0660
:10940000882309F476CF11C085E89AE4D9D98091F0
:109410001F06882309F48CCF08C085EE9BE4D0D9C1
:1094200080911F06882309F49FCFDF91CF911F9170
:109430000F9108952F923F924F925F926F927F9279
:109440008F929F92AF92CF92DF92EF92FF920F9303
:109450001F93CF93DF9300D01F92CDB7DEB74C019F
:109460001B01E982FA820B831C83CA01B9010F94A4
:1094700099332AE037ED43E25CE30F9437350F94DC
:1094800068332B013C01F1016081718182819381FC
:109490000F9499332AE037ED43E25CE30F943735BC
:1094A0000F9468338B010419150969817A818B81C6
:1094B0009C810F9499332AE037ED43E25CE30F94EB
:1094C00037350F9468339B012419350984EDE82E54
:1094D00087E4F82EA201B101C4010E9452650F90E9
:1094E0000F900F900F90DF91CF911F910F91FF90F0
:1094F000EF90DF90CF90AF909F908F907F906F9084
:109500005F904F903F902F900895AF92CF92DF924F
:10951000EF92FF920F931F93CF93DF9361E081E06F
:109520000E945766D0915306C0E0D1111AC08091B5
:109530005206811104C00E940F6A811194C080916B
:109540001E02882309F486C081E090915206911191
:1095500080E004E024E046EE5CE26C2F0E94C23F13
:1095600079C0D13039F580915206813021F40E94C2
:109570000F6A811180C080911E02882309F46AC09D
:1095800011E080915206813009F010E06091E40C06
:109590007091E50C8091E60C9091E70C0F94993353
:1095A000D9DD00E09C0140EE5CE26C2F812F0E942F
:1095B000F63F50C0D23039F580915206823021F406
:1095C0000E940F6A811171C080911E02882309F4E4
:1095D00041C011E080915206823009F010E06091A4
:1095E000E80C7091E90C8091EA0C9091EB0C0F94CF
:1095F0009933B0DD00E09C014CED5CE26C2F812FD3
:109600000E94F63F27C0D33029F58091520683305F
:1096100021F40E940F6A811162C080911E0288238A
:10962000C9F011E080915206833009F010E060919A
:10963000EC0C7091ED0C8091EE0C9091EF0C0F946E
:10964000993388DD00E09C0148ED5CE26C2F812FAE
:109650000E94F63FCF5FDF5FC53009F066CF84E040
:109660008093510655C00E94DA6580911F068823B9
:1096700009F465CF4DC0A12C48E6C42E49EBD42E89
:1096800010EDE12E17E0F12E00E010E024E630E0CE
:1096900040E050E064EE7CE083EE9CE2CBDE809123
:1096A0001F06882309F467CF33C0A12C28E6C22EF9
:1096B00029EBD22E10EDE12E17E0F12E00E010E0A4
:1096C00024E630E040E050E068EE7CE08EED9CE285
:1096D000B1DE80911F06882309F476CF19C0A12C32
:1096E00088E6C82E89EBD82E10EDE12E17E0F12E7A
:1096F00000E010E024E630E040E050E06CEE7CE07A
:109700008AED9CE297DE80911F06882309F485CFBD
:10971000DF91CF911F910F91FF90EF90DF90CF904D
:10972000AF9008952F923F924F925F926F927F92E7
:109730008F929F92AF92CF92DF92EF92FF920F9310
:109740001F93CF93DF9300D01F92CDB7DEB74C01AC
:109750001B01E982FA820B831C83CA01B9010F94B1
:1097600068332B013C01F101608171818281938119
:109770000F9468338B010419150969817A818B81F3
:109780009C810F9468339B012419350980EEE82EE3
:1097900087E4F82EA201B101C4010E9452650F9026
:1097A0000F900F900F90DF91CF911F910F91FF902D
:1097B000EF90DF90CF90AF909F908F907F906F90C1
:1097C0005F904F903F902F9008959F92AF92BF92DD
:1097D000CF92DF92EF92FF920F931F93CF93DF937D
:1097E00000D01F92CDB7DEB761E081E00E945766DE
:1097F00090905306B12C91101AC08091520681119D
:1098000004C00E940F6A811198C080911E028823B3
:1098100009F48AC081E090915206911180E004E041
:1098200024E046EC5CE26B2D0E94C23F7DC081E0EB
:1098300098122CC080915206813021F40E940F6A48
:10984000811183C080911E02882309F46DC011E04C
:1098500080915206813009F010E08091450D909181
:10986000460DA091470DB091480D89839A83AB8333
:10987000BC83CE0101960E94EC8700E09C0142EB84
:109880005CE26B2D812F0E94F63F4EC082E0981261
:1098900025C080915206823021F40E940F6A811106
:1098A0007CC080911E02882309F43EC011E08091A3
:1098B0005206823009F010E06091C00B7091C10B2C
:1098C0008091C20B9091C30B1BDC00E09C014EE920
:1098D0005CE26B2D812F0E94F63F26C083E0981238
:1098E00023C080915206833021F40E940F6A8111B7
:1098F0006CC080911E028823B9F011E0809152065D
:10990000833009F010E06091C40B7091C50B809119
:10991000C60B9091C70BF4DB00E09C014EE85CE2C3
:109920006B2D812F0E94F63FB394939485E0B8127B
:1099300062CF84E0809351065FC00E94DA65809117
:109940001F06882309F461CF57C020E030E048ECBF
:1099500052E46091450D7091460D8091470D9091B4
:10996000480D0F9437350F946833A12CC12CD12C9E
:109970002AEDE22E27E4F22E8B012FEF3FE740E0A5
:1099800050E065E47DE08CEB9CE20E9452658091A2
:109990001F06882309F456CF2FC081E00E94046A75
:1099A000A12CC12CD12CE12CF12C08E413E420E0F3
:1099B00030E0A90160EC7BE088EA9CE2B3DE8091B4
:1099C0001F06882309F46DCF17C081E00E94046A46
:1099D000A12CC12CD12CE12CF12C08E413E420E0C3
:1099E00030E0A90164EC7BE086E99CE29BDE80919B
:1099F0001F06882309F47DCF0F900F900F900F90D2
:109A0000DF91CF911F910F91FF90EF90DF90CF905A
:109A1000BF90AF909F900895AF92CF92DF92EF9258
:109A2000FF920F931F93CF93DF9361E081E00E9439
:109A30005766D0915306C0E0D1111AC080915206EA
:109A4000811104C00E940F6A811103C180911E021E
:109A5000882309F4F5C081E090915206911180E0CD
:109A600004E024E04CE75CE26C2F0E94C23FE8C0B7
:109A7000D13029F580915206813021F40E940F6A7D
:109A80008111EFC080911E02882309F4D9C011E032
:109A900080915206813009F010E06091F70D7091CD
:109AA000F80D8091F90D9091FA0D2ADB00E09C01F0
:109AB0004EE65CE26C2F812F0E94F63FC1C0D2308F
:109AC00029F580915206823021F40E940F6A81119B
:109AD000E2C080911E02882309F4B2C011E0809197
:109AE0005206823009F010E06091FB0D7091FC0D80
:109AF0008091FD0D9091FE0D03DB00E09C0140E69E
:109B00005CE26C2F812F0E94F63F9AC0D33029F57A
:109B100080915206833021F40E940F6A8111D5C0D2
:109B200080911E02882309F48BC011E080915206B7
:109B3000833009F010E06091FF0D7091000E80916C
:109B4000010E9091020EDCDA00E09C0142E55CE23D
:109B50006C2F812F0E94F63F73C0D43029F580917D
:109B60005206843021F40E940F6A8111C8C080918E
:109B70001E02882309F464C011E0809152068430EB
:109B800009F010E06091030E7091040E8091050EB3
:109B90009091060EB5DA00E09C0144E45CE26C2F83
:109BA000812F0E94F63F4CC0D53029F58091520696
:109BB000853021F40E940F6A8111BBC080911E0282
:109BC000882309F43DC011E080915206853009F0E8
:109BD00010E06091130E7091140E8091150E90910B
:109BE000160E8EDA00E09C014AE35CE26C2F812FB6
:109BF0000E94F63F25C0D63019F580915206863076
:109C000021F40E940F6A8111ADC080911E02882349
:109C1000B9F011E080915206863009F010E06091B1
:109C2000170E7091180E8091190E90911A0E68DA25
:109C300000E09C0146E25CE26C2F812F0E94F63F1F
:109C4000CF5FDF5FC53009F0F7CE87E08093510624
:109C5000A1C00E94DA6580911F06882309F4F6CE20
:109C600099C081E00E94046AA12CC12CD12CE12C66
:109C700010ECF12E09E714E420E030E040E85FE367
:109C800067EF7DE085E79CE24DDD80911F0688232C
:109C900009F4F8CE7FC081E00E94046AA12CC12C97
:109CA000D12CE12C10ECF12E09E714E420E030E097
:109CB00040E85FE36BEF7DE087E69CE233DD809177
:109CC0001F06882309F405CF65C081E00E94046A5D
:109CD000A12CC12CD12CE12C10ECF12E09E714E4BD
:109CE00020E030E040E85FE36FEF7DE089E59CE253
:109CF00019DD80911F06882309F412CF4BC081E043
:109D00000E94046AA12CC12CD12CE12C10ECF12E64
:109D100009E714E420E030E040E85FE363E07EE040
:109D20008BE49CE2FFDC80911F06882309F41FCF9F
:109D300031C081E00E94046AA12CC12CD12CE12CFD
:109D400010ECF12E09E714E420E030E0A90163E112
:109D50007EE08FE39CE2E6DC80911F06882309F415
:109D60002DCF18C081E00E94046AA12CC12CD12CF7
:109D7000E12C10ECF12E09E714E420E030E0A90119
:109D800067E17EE080E39CE2CDDC80911F068823C2
:109D900009F43BCFDF91CF911F910F91FF90EF908E
:109DA000DF90CF90AF9008959F92AF92BF92CF92E5
:109DB000DF92EF92FF920F931F93CF93DF9300D028
:109DC0001F92CDB7DEB761E081E00E9457669090A8
:109DD0005306B12C91101AC080915206811104C013
:109DE0000E940F6A8111BFC080911E02882309F46E
:109DF000B2C081E090915206911180E004E024E02D
:109E000048E95BE26B2D0E94C23FA5C081E0981239
:109E100025C080915206813021F40E940F6A811181
:109E2000AAC080911E02882309F495C011E0809198
:109E30005206813009F010E06091A30D7091A40DDD
:109E40008091A50D9091A60D5BD900E09C0148E89A
:109E50005BE26B2D812F0E94F63F7DC082E098125D
:109E600025C080915206823021F40E940F6A811130
:109E70009CC080911E02882309F46DC011E080917E
:109E80005206823009F010E06091A70D7091A80D84
:109E90008091A90D9091AA0D33D900E09C0148E76B
:109EA0005BE26B2D812F0E94F63F55C083E0981234
:109EB0002CC080915206833021F40E940F6A8111D8
:109EC0008EC080911E02882309F445C011E0809164
:109ED0005206833009F010E08091AB0D9091AC0DEB
:109EE000A091AD0DB091AE0D89839A83AB83BC83F5
:109EF000CE0101960E94038B00E09C0148E65BE2E4
:109F00006B2D812F0E94F63F26C084E0981223C05B
:109F100080915206843021F40E940F6A81118CC016
:109F200080911E028823B9F011E08091520684309E
:109F300009F010E06091AF0D7091B00D8091B10DFE
:109F40009091B20DDDD800E09C0148E55BE26B2DFD
:109F5000812F0E94F63FB394939485E0B8123ACFD4
:109F6000B092510682C00E94DA6580911F06882354
:109F700009F43ACF7AC081E00E94046AA12CC12C76
:109F8000D12CE12C10E8F12E07E714E420E030E0BA
:109F900040E85FE363EA7DE080E99BE2C3DB809118
:109FA0001F06882309F43DCF60C081E00E94046A47
:109FB000A12CC12CD12CE12C10E8F12E07E714E4E0
:109FC00020E030E040E85FE367EA7DE080E89BE284
:109FD000A9DB80911F06882309F44BCF46C081E09E
:109FE0000E94046A20E030E048EC52E46091AB0D3E
:109FF0007091AC0D8091AD0D9091AE0D0F943735F1
:10A000000F9468338B010A501109A12CC12CD12C5B
:10A010009CEEE92E97E4F92E25EF3FE74AE050E069
:10A020006BEA7DE080E79BE20E94526580911F060B
:10A03000882309F446CF19C081E00E94046AA12C4C
:10A04000C12CD12CE12C10E8F12E07E714E420E01C
:10A0500030E040E85FE36FEA7DE080E69BE262DBB0
:10A0600080911F06882309F45BCF0F900F900F900B
:10A070000F90DF91CF911F910F91FF90EF90DF90A4
:10A08000CF90BF90AF909F9008952F923F924F92A4
:10A090005F926F927F928F929F92AF92CF92DF9258
:10A0A000EF92FF920F931F93CF93DF9300D01F92F5
:10A0B000CDB7DEB74C011B01CA01B901E982FA82B2
:10A0C0000B831C832AE037ED43E25CE30F943735C2
:10A0D0000F9468332B013C012AE037ED43E25CE347
:10A0E000F10160817181828193810F9437350F94E2
:10A0F00068338B01041915092AE037ED43E25CE36C
:10A1000069817A818B819C810F9437350F946833F4
:10A110009B012419350986EEE82E87E4F82EA2016A
:10A12000B101C4010E9452650F900F900F900F90E3
:10A13000DF91CF911F910F91FF90EF90DF90CF9023
:10A14000AF909F908F907F906F905F904F903F90D7
:10A150002F9008959F92AF92BF92CF92DF92EF928D
:10A16000FF920F931F93CF93DF9300D01F92CDB731
:10A17000DEB761E081E00E94576690905306B12CF3
:10A1800091101AC080915206811104C00E940F6A7A
:10A19000811152C180911E02882309F444C181E0DB
:10A1A00090915206911180E004E024E044E15CE2E9
:10A1B0006B2D0E94C23F37C181E098122CC0809164
:10A1C0005206813021F40E940F6A81113DC18091B5
:10A1D0001E02882309F427C111E0809152068130C4
:10A1E00009F010E08091070E9091080EA091090EE1
:10A1F000B0910A0E89839A83AB83BC83CE0101960A
:10A200000E944B8A00E09C0148E05CE26B2D812FAC
:10A210000E94F63F08C182E098122CC0809152063D
:10A22000823021F40E940F6A811128C180911E02A0
:10A23000882309F4F8C011E080915206823009F0B9
:10A2400010E080910B0E90910C0EA0910D0EB0912C
:10A250000E0E89839A83AB83BC83CE0101960E9444
:10A260004B8A00E09C0144EF5BE26B2D812F0E9442
:10A27000F63FD9C083E098122CC0809152068330FB
:10A2800021F40E940F6A811113C180911E0288235C
:10A2900009F4C9C011E080915206833009F010E042
:10A2A00080910F0E9091100EA091110EB091120E90
:10A2B00089839A83AB83BC83CE0101960E944B8A2B
:10A2C00000E09C0142EE5BE26B2D812F0E94F63F85
:10A2D000AAC084E0981228C080915206843021F4EC
:10A2E0000E940F6A8111FEC080911E02882309F42A
:10A2F0009AC011E080915206843009F010E060911C
:10A30000D30D7091D40D8091D50D9091D60D0F94F1
:10A3100099330E94AA4800E09C0144ED5BE26B2D5A
:10A32000812F0E94F63F7FC085E0981228C080915F
:10A330005206853021F40E940F6A8111F1C080918C
:10A340001E02882309F46FC011E080915206853007
:10A3500009F010E06091D70D7091D80D8091D90D62
:10A360009091DA0D0F9499330E94AA4800E09C0165
:10A3700046EC5BE26B2D812F0E94F63F54C086E0D5
:10A38000981228C080915206863021F40E940F6AEC
:10A390008111E4C080911E02882309F444C011E0B9
:10A3A00080915206863009F010E06091DB0D7091CB
:10A3B000DC0D8091DD0D9091DE0D0F9499330E949C
:10A3C000AA4800E09C0148EB5BE26B2D812F0E94C4
:10A3D000F63F29C087E0981226C080915206873048
:10A3E00021F40E940F6A8111D7C080911E02882338
:10A3F000D1F011E080915206873009F010E06091B1
:10A40000DF0D7091E00D8091E10D9091E20D0F94C0
:10A4100099330E94AA4800E09C014AEA5BE26B2D56
:10A42000812F0E94F63FB394939485E0B812A8CE92
:10A4300088E080935106CDC00E94DA6580911F06A6
:10A44000882309F4A7CEC5C081E00E94046AA12C2C
:10A45000C12CD12CE12C1CE5F12E01EC17E420E0FD
:10A4600030E040E251E467E07EE08EE09CE20DDE09
:10A4700080911F06882309F4AACEABC081E00E9418
:10A48000046AA12CC12CD12CE12C1CE5F12E01EC8D
:10A4900017E420E030E048EC52E46BE07EE08EEF21
:10A4A0009BE2F3DD80911F06882309F4BFCE91C0A3
:10A4B00081E00E94046AA12CC12CD12CE12C1CE566
:10A4C000F12E01EC17E420E030E048EC52E46FE0BC
:10A4D0007EE08BEE9BE2D9DD80911F06882309F494
:10A4E000D4CE77C081E00E94046AA12C68EFC62E0A
:10A4F00067E4D62E18EBE12E12E8F12E01E010E011
:10A5000024E630E040E050E063ED7DE08BED9BE23F
:10A510000E941A4A80911F06882309F4E5CE59C08B
:10A5200081E00E94046AA12C48EFC42E47E4D42E97
:10A5300018EBE12E12E8F12E01E010E024E630E005
:10A5400040E050E067ED7DE08DEC9BE20E941A4A0E
:10A5500080911F06882309F4F2CE3BC081E00E945F
:10A56000046AA12C28EFC22E27E4D22E18EBE12E8C
:10A5700012E8F12E01E010E02AE030E040E050E087
:10A580006BED7DE08FEB9BE20E941A4A80911F06E3
:10A59000882309F4FFCE1DC081E00E94046AA12C2B
:10A5A00088EFC82E87E4D82E18EBE12E12E8F12EA2
:10A5B00001E010E024E630E040E050E06FED7DE0A7
:10A5C00081EB9BE20E941A4A80911F06882309F4BE
:10A5D0000CCF0F900F900F900F90DF91CF911F91A4
:10A5E0000F91FF90EF90DF90CF90BF90AF909F9032
:10A5F00008952F923F924F925F926F927F928F9227
:10A600009F92AF92CF92DF92EF92FF920F931F93A0
:10A61000CF93DF9300D01F92CDB7DEB74C011B0163
:10A62000CA01B901E982FA820B831C8320E030E081
:10A6300048EC52E40F9437350F9468332B013C01FA
:10A6400020E030E048EC52E4F101608171818281C8
:10A6500093810F9437350F9468338B0104191509D2
:10A6600020E030E048EC52E469817A818B819C8162
:10A670000F9437350F9468339B012419350982EF05
:10A68000E82E87E4F82EA201B101C4010E945265B0
:10A690000F900F900F900F90DF91CF911F910F911E
:10A6A000FF90EF90DF90CF90AF909F908F907F9032
:10A6B0006F905F904F903F902F9008959F92AF9230
:10A6C000BF92CF92DF92EF92FF920F931F93CF939F
:10A6D000DF9300D01F92CDB7DEB761E081E00E942A
:10A6E000576690905306B12C91101AC08091520673
:10A6F000811104C00E940F6A8111D4C080911E0292
:10A70000882309F4C7C081E090915206911180E03E
:10A7100004E024E046E45BE26B2D0E94C23FBAC035
:10A7200081E098122CC080915206813021F40E9461
:10A730000F6A8111BFC080911E02882309F4AAC04C
:10A7400011E080915206813009F010E08091E70D10
:10A750009091E80DA091E90DB091EA0D89839A835B
:10A76000AB83BC83CE0101960E94A48B00E09C01C8
:10A7700042E35BE26B2D812F0E94F63F8BC082E0AB
:10A7800098122CC080915206823021F40E940F6AE8
:10A790008111ACC080911E02882309F47BC011E0B6
:10A7A00080915206823009F010E08091EB0D90917B
:10A7B000EC0DA091ED0DB091EE0D89839A83AB83E2
:10A7C000BC83CE0101960E94A48B00E09C014EE167
:10A7D0005BE26B2D812F0E94F63F5CC083E09812F4
:10A7E0002CC080915206833021F40E940F6A81119F
:10A7F00099C080911E02882309F44CC011E0809119
:10A800005206833009F010E08091EF0D9091F00D29
:10A81000A091F10DB091F20D89839A83AB83BC8333
:10A82000CE0101960E94A48B00E09C014AE05BE20D
:10A830006B2D812F0E94F63F2DC084E098122AC014
:10A8400080915206843021F40E940F6A811186C0E3
:10A8500080911E028823F1F011E08091520684302D
:10A8600009F010E08091F30D9091F40DA091F50D99
:10A87000B091F60D89839A83AB83BC83CE01019698
:10A880000E94A48B00E09C0146EF5AE26B2D812FC1
:10A890000E94F63FB394939485E0B81225CFB0920E
:10A8A000510677C00E94DA6580911F06882309F45B
:10A8B00025CF6FC081E00E94046AA12C6AEFC62EEA
:10A8C00067E4D62EE12C1CE3F12E0CE116E420E027
:10A8D00030E040EA50E467EE7DE08CE39BE289DE05
:10A8E00080911F06882309F426CF53C081E00E947F
:10A8F000046AA12C4AEFC42E47E4D42EE12C1CE3B9
:10A90000F12E0CE116E420E030E040EA50E46BEE7A
:10A910007DE088E29BE26DDE80911F06882309F4CA
:10A9200039CF37C081E00E94046AA12C2AEFC22EE1
:10A9300027E4D22EE12C1CE3F12E0CE116E420E0FA
:10A9400030E040EA50E46FEE7DE084E19BE251DECE
:10A9500080911F06882309F44CCF1BC081E00E9420
:10A96000046AA12C8AEFC82E87E4D82EE12C1CE3C0
:10A97000F12E0CE116E420E030E040EA50E463EF11
:10A980007DE080E09BE235DE80911F06882309F49C
:10A990005FCF0F900F900F900F90DF91CF911F918D
:10A9A0000F91FF90EF90DF90CF90BF90AF909F906E
:10A9B00008950F93CF93DF9361E081E00E94576683
:10A9C000D0915306C0E0D1111AC080915206811176
:10A9D00004C00E940F6A81118BC080911E028823DF
:10A9E00009F47EC081E090915206911180E004E06C
:10A9F00024E04CE55DE26C2F0E94C23F71C0D13073
:10AA0000D9F480915206813021F40E940F6A81119D
:10AA100077C080911E02882309F462C081E0909182
:10AA20005206913009F080E003E02EE345E55DE257
:10AA30006C2F0E94C23F54C0D230D9F4809152068C
:10AA4000823021F40E940F6A811164C080911E023D
:10AA5000882309F445C081E090915206923009F0B4
:10AA600080E003E02EE34EE45DE26C2F0E94C23FE3
:10AA700037C0D330D1F480915206833021F40E9444
:10AA80000F6A811151C080911E02882349F181E033
:10AA900090915206933009F080E003E02EE347E402
:10AAA0005DE26C2F0E94C23F1BC0D430C9F480917C
:10AAB0005206843021F40E940F6A81113FC08091B8
:10AAC0001E02882369F081E090915206943009F0CB
:10AAD00080E003E02EE34DE35DE26C2F0E94C23F75
:10AAE000CF5FDF5FC53009F06ECFC09351062FC036
:10AAF0000E94DA6580911F06882309F46ECF27C073
:10AB000088E399E50E94E04380911F06882309F4B9
:10AB100080CF1DC08DE399E50E94E04380911F0620
:10AB2000882309F493CF13C082E499E50E94E0439F
:10AB300080911F06882309F4A6CF09C087E499E510
:10AB40000E94E04380911F06882309F4B8CFDF916B
:10AB5000CF910F910895CF92DF92EF92FF92CF9312
:10AB6000C82F0E94BC2B6B017C0124EA30E74DE723
:10AB70005FE360916A0670916B0680916C0690911C
:10AB80006D060F94F93287FD05C04AEF50E060E092
:10AB900070E003C040E050E0BA01C40ED51EE61ECE
:10ABA000F71EC0926606D0926706E0926806F092A1
:10ABB0006906C0931F02CF91FF90EF90DF90CF9076
:10ABC00008952F923F924F925F926F927F928F9251
:10ABD0009F92AF92BF92CF92DF92EF92FF921F931C
:10ABE000CF93DF93CDB7DEB728970FB6F894DEBFCB
:10ABF0000FBECDBF1C01162F0E940F6A882329F0BB
:10AC0000109281060E94DA65DAC0209179063091AF
:10AC10007A063E832D83232B09F49DC0E4E01E9F1A
:10AC2000C001112498878F83FC01EE59FD4F80806D
:10AC30009180A280B38020E030E04AE754E4C5016F
:10AC4000B4010F941F322B013C0120E030E04AE7B1
:10AC500054E4C501B4010F9420326B017C01809152
:10AC600057028823B9F1113029F198F0123091F58B
:10AC700040904F02509050026090510270905202EA
:10AC8000C0905302D0905402E0905502F0905602CA
:10AC900021C040903F02509040026090410270906D
:10ACA0004202C0904302D0904402E0904502F090EE
:10ACB000460210C0409047025090480260904902FE
:10ACC00070904A02C0904B02D0904C02E0904D022E
:10ACD000F0904E022D813E81B901330F880B990B04
:10ACE0000F949B3320916A0630916B0640916C065D
:10ACF00050916D060F9437359B01AC01C501B4012D
:10AD00000F942032EF81F885EE59FD4F5F0160838B
:10AD10007183828393832D813E8137FF0CC0A30111
:10AD200092010F94F93287FF11C0F50140825182E0
:10AD3000628273820BC0A70196010F94FC3418162F
:10AD40002CF4F501C082D182E282F382812F03DFED
:10AD500081E080931E0210927A061092790680910B
:10AD60001E02882361F124E0129FF0011124EE59A4
:10AD7000FD4F80819181A281B38189839A83AB83C6
:10AD8000BC832DEC3CEC4CEC5DE360916A06709169
:10AD90006B0680916C0690916D060F94FC3487FDD4
:10ADA00005C0CE0101960E948A8805C060E2CE01EE
:10ADB00001960E940289BC01C1010E945740289659
:10ADC0000FB6F894DEBF0FBECDBFDF91CF911F91BC
:10ADD000FF90EF90DF90CF90BF90AF909F908F90BB
:10ADE0007F906F905F904F903F902F90089560E01C
:10ADF00084ED9DE2E6CE61E08DEC9DE2E2CE62E084
:10AE000086EC9DE2DECECF93DF9300D01F92CDB7CC
:10AE1000DEB70E940F6A882329F0109281060E94F3
:10AE2000DA6557C06091790670917A0661157105EF
:10AE300069F1072E000C880B990B0F949B3320911E
:10AE40006A0630916B0640916C0650916D060F9426
:10AE500037359B01AC0160916E0270916F02809159
:10AE60007002909171020F94203260936E02709381
:10AE70006F02809370029093710283E06CDE81E038
:10AE800080931E0210927A061092790680911E021B
:10AE90008823F9F0209102063091030640910406C0
:10AEA0005091050660916E0270916F028091700260
:10AEB000909171020F941F3269837A838B839C83F4
:10AEC000CE0101960E948A88BC0185E69DE20E941F
:10AED00057400F900F900F900F90DF91CF910895F2
:10AEE00021E02093810660936A0670936B0680933D
:10AEF0006C0690936D0620E040E060E070E0809189
:10AF00000006909101060C94AE6560E070E080E26E
:10AF100091E4E6CF60E070E080E89FE3E1CF6DEC84
:10AF20007CEC8CEC9DE3DCCFFF920F931F93CF93CF
:10AF3000DF93F82E709301066093000661E081E0D4
:10AF40000E945766D0915306C0E091E081E0F81668
:10AF500059F1F81628F082E0F81609F449C06CC0DF
:10AF6000D111D3C0992389F08091520618166CF044
:10AF70002091790630917A062F5F3F4F30937A0601
:10AF8000209379068F5F8093520680911E0288235A
:10AF900009F42CC100E010E021E041E06FEB7DE21C
:10AFA0008C2F0E945F3F22C1D111AFC0992389F03D
:10AFB0008091520618166CF02091790630917A062D
:10AFC0002F5F3F4F30937A06209379068F5F8093EF
:10AFD000520680911E02882309F408C100E010E0A7
:10AFE00021E041E068EB7DE28C2F0E945F3FFEC0D4
:10AFF000D1118BC0992389F08091520618166CF0FC
:10B000002091790630917A062F5F3F4F30937A0670
:10B01000209379068F5F8093520680911E028823C9
:10B0200009F4E4C000E010E021E041E061EB7DE2E2
:10B030008C2F0E945F3FDAC040916E0250916F02E8
:10B040006091700270917102409302065093030662
:10B050006093040670930506D11122C0992389F0EC
:10B060008091520618166CF02091790630917A067C
:10B070002F5F3F4F30937A06209379068F5F80933E
:10B08000520680911E02882309F4E8C000E010E017
:10B0900021E041E067EA7DE28C2F0E945F3FDEC045
:10B0A00083E0F81232C06091550C7091560C80917B
:10B0B000570C9091580C20911F0C211126C00F9411
:10B0C000683320912D0230912E0262177307ECF441
:10B0D000D130C9F480915206813021F40E940F6A68
:10B0E00081118EC080911E02882369F081E09091C9
:10B0F0005206913009F080E004E024E047E95DE287
:10B100006C2F0E94C23F82E072C0D130D9F480918E
:10B110005206813021F40E940F6A811179C080911A
:10B120001E02882309F462C081E09091520691309A
:10B1300009F080E004E024E04DE85DE26C2F0E941D
:10B14000C23F54C0D230D9F480915206823021F4EB
:10B150000E940F6A811164C080911E02882309F445
:10B1600045C081E090915206923009F080E003E002
:10B170002EE343E85DE26C2F0E94C23F37C0D3301C
:10B18000D1F480915206833021F40E940F6A81111C
:10B1900051C080911E02882349F181E090915206AE
:10B1A000933009F080E003E02EE34AE75DE26C2F84
:10B1B0000E94C23F1BC0D430C9F480915206843033
:10B1C00021F40E940F6A81113FC080911E028823E2
:10B1D00069F081E090915206943009F080E003E03C
:10B1E0002EE34FE65DE26C2F0E94C23F85E0CF5F09
:10B1F000DF5F90E0C53009F0A9CE8093510632C0E0
:10B200000E94DA6580911F06882309F46BCF2AC05B
:10B210000E94DA6580911F06882309F480CF22C03E
:10B2200085E897E50E94E04380911F06882309F492
:10B2300093CF18C08AE897E50E94E04380911F06EB
:10B24000882309F4A6CF0EC08FE897E50E94E0435B
:10B2500080911F06882309F4B8CF04C083E0F81258
:10B26000C5CF21CFDF91CF911F910F91FF9008950E
:10B270004FEF67EF76E580E057CE4FEF6BEF76E567
:10B2800081E052CE4FEF6FEF76E582E04DCE4FEF8B
:10B2900063E077E583E048CE0F93CF93DF9361E0DF
:10B2A00081E00E945766D0915306C0E0D1111AC0C8
:10B2B00080915206811104C00E940F6A8111A9C0B9
:10B2C00080911E02882309F49BC081E09091520670
:10B2D000911180E004E024E048E35DE26C2F0E94DD
:10B2E000C23F8EC0D130D9F480915206813021F412
:10B2F0000E940F6A811195C080911E02882309F473
:10B300007FC081E090915206913009F080E003E027
:10B310002EE34EE25DE26C2F0E94C23F71C0D2303C
:10B32000D9F480915206823021F40E940F6A811173
:10B3300082C080911E02882309F462C081E090914E
:10B340005206923009F080E000E22EE340E25DE236
:10B350006C2F0E94C23F54C0D330D9F48091520662
:10B36000833021F40E940F6A81116FC080911E0208
:10B37000882309F445C081E090915206933009F08A
:10B3800080E000E22EE342E15DE26C2F0E94C23FCA
:10B3900037C0D430D1F480915206843021F40E9419
:10B3A0000F6A81115CC080911E02882349F181E0FF
:10B3B00090915206943009F080E000E22EE343E0E1
:10B3C0005DE26C2F0E94C23F1BC0D530C9F4809152
:10B3D0005206853021F40E940F6A81114AC0809183
:10B3E0001E02882369F081E090915206953009F0A1
:10B3F00080E000E22EE34EEE5CE26C2F0E94C23F42
:10B40000CF5FDF5FC53009F051CF86E080935106F2
:10B4100039C00E94DA6580911F06882309F450CF55
:10B4200031C089ED94E50E94E04380911F06882396
:10B4300009F462CF27C08AE29DE20E9450658091A4
:10B440001F06882309F475CF1DC08FE19DE20E947D
:10B45000506580911F06882309F488CF13C088E9BE
:10B4600093E00E94506580911F06882309F49BCFCA
:10B4700009C08FEF9CE20E94506580911F068823CF
:10B4800009F4ADCFDF91CF910F910895FC01718345
:10B490006083089566E47AE583ED9AE50C94EF65A0
:10B4A0000F931F93CF93DF9361E081E00E94576673
:10B4B000C0915306D0E081E0C11122C0882389F0F9
:10B4C0008091520618166CF02091790630917A0618
:10B4D0002F5F3F4F30937A06209379068F5F8093DA
:10B4E000520680911E02882309F441C000E010E05A
:10B4F00020E041E06EE37FE28D2F0E945F3F37C086
:10B50000C130D1F480915206813021F40E940F6A3B
:10B51000811137C080911E02882349F181E090910A
:10B520005206913009F080E000E22EE343E35FE24F
:10B530006D2F0E94C23F1BC0C230C9F480915206D9
:10B54000823021F40E940F6A811122C080911E0274
:10B55000882369F081E090915206923009F080E0F2
:10B5600000E22EE34FE15FE26D2F0E94C23FDF5FFA
:10B57000CF5F80E0D53009F09FCF83E08093510604
:10B580000DC0C093C80B80911F06882319F206C016
:10B59000C093C80B80911F068823C1F2DF91CF9121
:10B5A0001F910F9108950C944D87EF92FF920F9386
:10B5B0001F93CF93DF93CDB7DEB72B970FB6F894D9
:10B5C000DEBF0FBECDBF7C0140910706842F042E45
:10B5D000000C990B20910806223051F0233019F00D
:10B5E0002DE63FE20AC047FF06C029E73FE205C05B
:10B5F0002BE83FE202C022E83FE29F934F933F9344
:10B600002F938E010F5F1F4F1F930F930F944C3B8F
:10B6100040912B0250912C024F50510997010F90ED
:10B620000F900F900F900F900F904E155F050CF438
:10B630009A0130935A0C2093590C80E00E942D9F60
:10B64000C8010E944C672B960FB6F894DEBF0FBE60
:10B65000CDBFDF91CF911F910F91FF90EF90089593
:10B66000E091070687E1E802F0011124EF5AF34F59
:10B67000808591859ACFAF92BF92CF92DF92EF9261
:10B68000FF920F931F93CF93DF93B82E80930806FA
:10B690006093070661E081E00E945766D0915306EF
:10B6A000C0E081E0D1112EC0882389F0809152063C
:10B6B00018166CF02091790630917A062F5F3F4F73
:10B6C00030937A06209379068F5F8093520680919B
:10B6D0001E02882309F494C022E0B21649F033E038
:10B6E000B31203C06FE47FE205C06FE37FE202C0E4
:10B6F0006FE57FE200E010E021E041E08C2F0E9446
:10B700005F3F7EC0D130D9F480915206813021F460
:10B710000E940F6A81117DC080911E02882309F466
:10B720006FC081E090915206913009F080E004E012
:10B7300024E04AEC5FE26C2F0E94C23F61C0D2302D
:10B74000D9F480915206823021F40E940F6A81114F
:10B7500068C080911E02882309F452C081E0909154
:10B760005206923009F080E000E22EE34EEB5FE2F9
:10B770006C2F0E94C23F44C0D330D1F48091520656
:10B78000833021F40E940F6A811156C080911E02FD
:10B790008823B1F181E090915206933009F080E066
:10B7A00000E22EE342EB5FE26C2F0E94C23F28C012
:10B7B000D43031F580915206843021F40E940F6A12
:10B7C000811145C080911E028823D1F011E0809143
:10B7D0005206843009F010E02091070637E1230378
:10B7E000F0011124EF5AF34F808591850E944D8717
:10B7F00000E09C0144E95FE26C2F812F0E94F63F3C
:10B80000CF5FDF5F80E0C53009F04CCFC0935106B9
:10B8100046C00E94DA6580911F06882309F47CCF18
:10B820003EC080910F0690911006BFDE80911F06EA
:10B83000882309F48ECF33C08091110690911206AF
:10B84000B4DE80911F06882309F4A0CF28C081E0D0
:10B850000E94046A6091070627E16203B001112487
:10B86000FB01EF5AF34F0085118508571109675AFC
:10B87000734FA12C80E3C82E8BE5D82E9AE4E92ED5
:10B880009AE5F92E2AEA30E048E750E083EA9FE2A1
:10B890000E94526580911F06882309F493CFDF919F
:10B8A000CF911F910F91FF90EF90DF90CF90BF90BD
:10B8B000AF90089560E081E0DECE8F929F92AF92CC
:10B8C000BF92CF92DF92EF92FF920F931F93CF938D
:10B8D000DF934C015B016A0160E085E00E945766DE
:10B8E000D0915306F12C82E0E82ED1111AC080913C
:10B8F0001E02882321F180912102823041F08330A1
:10B9000019F464EF7EE205C062EE7EE202C064E0FC
:10B910007FE200E010E021E041E08F2D0E945F3FD8
:10B920000EC0D13061F480911E02882341F000E006
:10B9300010E020E041E0B4018F2D0E945F3FA11490
:10B94000B10481F0D23081F480911E02882309F481
:10B950006EC000E010E020E041E0B5018F2D0E94B4
:10B960005F3F65C0C2E001C0C3E0C114D10491F0E3
:10B97000DC130FC080911E02882351F000E010E01C
:10B9800020E041E0B6018F2D0E945F3FCD2F01C026
:10B99000CD2FCF5F21E030E0A114B10411F420E0FD
:10B9A00030E081E090E0C114D10411F480E090E037
:10B9B000820F931F029781F0DC130DC080911E024D
:10B9C000882349F000E010E020E041E06DE17FE2F3
:10B9D0008F2D0E945F3FCF5FDC1314C080911E0249
:10B9E000882371F000E010E021E040E062E17FE2B6
:10B9F0008F2D0E945F3F609106068F2D0E94F93EB9
:10BA0000E0921E02F394DF5F85E0F8126ECFCF5F05
:10BA1000C0935106DF91CF911F910F91FF90EF904E
:10BA2000DF90CF90BF90AF909F908F900895C3E02C
:10BA3000C114D10409F0ADCFADCF40E050E060E0DB
:10BA400070E087ED9EE239CF4EEC5EE26EEB7EE277
:10BA500085EB9EE232CF40E050E065EA7EE28CE981
:10BA60009EE22BCF40E050E06DE87EE28EE79EE262
:10BA700024CF40E050E06FE67EE282E69EE21DCFFA
:10BA800046E55EE265E47EE285E39EE216CF40E0B5
:10BA900050E067E27EE28EE19EE20FCF40E050E0B0
:10BAA0006EE07EE281E09EE208CF40E050E064EF8D
:10BAB0007DE283EF9DE201CF40E050E064EE7DE265
:10BAC0008BED9DE2FACE6111609321024093060650
:10BAD000082E000C990BAA0BBB0B8C309105A0F51E
:10BAE000FC018827EA56FF4F8F4F0D94813684E280
:10BAF0009DE51FC08BE29DE51CC08EE49DE519C04D
:10BB000080E49DE516C087E49DE513C08CE59DE5C6
:10BB100010C085E59DE50DC089E39DE50AC082E37F
:10BB20009DE507C01092C80B80E59AE502C08DE143
:10BB30009DE5009749F021E02093810620E040E058
:10BB400060E070E00C94AE650C94D36580916E0655
:10BB5000882321F0109281060E94DA650C94863EBB
:10BB60009091EA0893FB882780F993FF06C081E053
:10BB700090911A07911101C080E00895F1DF8823A8
:10BB800039F08091EA0882FB882780F991E08927C3
:10BB9000089540E061E080E096DF88E990E30F944B
:10BBA000EA210C940ED9EADF882321F084E990E39E
:10BBB0000F94EA210C94EA99109290161092810247
:10BBC0008091EA0880628093EA080E94F2996FEF00
:10BBD00086E890E30E94FC6BE6C70F93CF93DF9358
:10BBE00061E081E00E945766D0915306C0E08C2F3F
:10BBF0008D0FC9F480915206811104C00E940F6A12
:10BC0000811133C080911E02882341F181E090911F
:10BC10005206911180E004E024E041E850E36C2FEB
:10BC20000E94C23F1BC08130C9F48091520681300E
:10BC300021F40E940F6A81111EC080911E02882388
:10BC400069F081E090915206913009F080E000E2C5
:10BC50002EE346E750E36C2F0E94C23FCF5FC53012
:10BC600031F682E0809351060BC0A4D780911F0665
:10BC7000882341F205C0A0DF80911F068823E9F2E6
:10BC8000DF91CF910F910895EF92FF920F931F9341
:10BC9000CF93DF9361E081E00E945766C091530625
:10BCA00010E0C11118C080915206811104C00E9499
:10BCB0000F6A81118BC180911E02882361F081E09F
:10BCC00090915206911180E004E024E04AE650E3AE
:10BCD000612F0E94C23F8091EA0882FBDD27D0F9E4
:10BCE00082FD06C0D1E090918316913009F0D0E03A
:10BCF00083FBEE24E0F883FF03C032DFF82E01C09F
:10BD0000F12CDD2309F458C0C130D9F480915206DA
:10BD1000813021F40E940F6A81115FC180911E025F
:10BD2000882309F46BC181E090915206913009F0AB
:10BD300080E000E22EE34EE550E3612F0E94C23F17
:10BD40005DC1C230D9F480915206823021F40E9444
:10BD50000F6A811149C180911E02882309F44EC1E6
:10BD600081E090915206923009F080E003E02EE3EA
:10BD700043E550E3612F0E94C23F40C1C33009F048
:10BD800047C080915206833021F40E940F6A8111CE
:10BD900037C180911E02882309F430C181E090915F
:10BDA0005206933009F080E003E02EE34EE450E3C6
:10BDB000612F0E94C23F22C180918316823029F0F8
:10BDC000DDDE811102C0D1E004C0C13009F422C11E
:10BDD000D2E0CD131BC0809152068C1304C00E9488
:10BDE0000F6A811139C180911E02882371F081E0B0
:10BDF000909152069C1380E003E02EE348E350E369
:10BE0000612F0E94C23FDC2F01C0DC2FDF5F01C029
:10BE1000D4E0CD131BC0809152068C1304C00E9445
:10BE20000F6A811123C180911E02882371F081E085
:10BE3000909152069C1380E003E02EE34CE250E325
:10BE4000612F0E94C23FDC2F01C0DC2F81E08D0FEB
:10BE5000C81318C0809152068C1304C00E940F6A48
:10BE600081110EC180911E02882361F081E09091C2
:10BE700052069C1380E003E02EE34EE150E3612F75
:10BE80000E94C23F82E08D0F4091590C50915A0C94
:10BE900090911F0C911107C020912D0230912E021C
:10BEA00042175307DCF0C81333C0809152068C133D
:10BEB00004C00E940F6A8111EDC080911E02882388
:10BEC00039F181E0909152069C1380E000E22EE36C
:10BED00046E050E3612F0E94C23F1AC0C81318C049
:10BEE000809152068C1304C00E940F6A8111DBC03E
:10BEF00080911E02882361F081E0909152069C138C
:10BF000080E003E02EE346EF5FE2612F0E94C23F34
:10BF1000DD5FCD1318C0809152068C1304C00E94BF
:10BF20000F6A8111CAC080911E02882361F081E0EE
:10BF3000909152069C1380E003E02EE348EE5FE20E
:10BF4000612F0E94C23F91E09D0FEE20E9F0F110B9
:10BF500035C0C91331C0809152068C1304C00E94B1
:10BF60000F6A8111B4C080911E02882329F181E0FB
:10BF7000909152069C1380E003E02EE34AED5FE2CD
:10BF8000612F0E94C23F18C0C91316C0809152068B
:10BF90008C1302C00E940F6A80911E02882361F0F8
:10BFA00081E0909152069C1380E000E22EE34FEC7A
:10BFB0005FE2612F0E94C23F92E09D0F1F5FCF5F43
:10BFC000153009F06ECE909351068AC0F3D580915A
:10BFD0001F06882309F46FCE83C0DBDD80911F0626
:10BFE000882309F49BCE7CC08DEE9DE50E94E04342
:10BFF00080911F06882309F4AECE72C0D4E026CF0C
:10C000008AE391E60E94E04380911F06882309F4A9
:10C01000C0CE66C080915206813021F40E940F6A22
:10C02000811112C080911E028823A1F081E09091BD
:10C030005206913009F080E000E22EE341E450E343
:10C04000612F0E94C23F06C0AEDD80911F0688238B
:10C0500049F346C0D2E0DACE8CE499E50E94E04391
:10C0600080911F06882309F4BECE3AC080E193E692
:10C070000E94E04380911F06882309F4D4CE30C08B
:10C080008FE394E60E94E04380911F06882309F421
:10C09000E9CE26C086E190E303D580911F06882370
:10C0A00009F40BCF1DC08AE59CE50E94E043809116
:10C0B0001F06882309F41CCF13C086EA9DE50E9461
:10C0C000E04380911F06882309F42DCF09C089E43D
:10C0D00094E40E94E04380911F06882309F443CF33
:10C0E000DF91CF911F910F91FF90EF900895609194
:10C0F0004F0C70E080E00C94699A60917602709128
:10C100007702072E000C880B990B0F949B332AE0C3
:10C1100037ED43E25CE30F9437356093720270931E
:10C12000730280937402909375020895FC016083FA
:10C13000089580E00C942D9F66E970E681EA90E610
:10C140004EC50C942787EF92FF920F931F93CF93C6
:10C15000DF9300D01F92CDB7DEB7082F7B010E947E
:10C160000F6A882321F01092810624D53FC04091A8
:10C17000790650917A064115510571F010927A06B0
:10C180001092790681E080931E02052E000C660B4A
:10C19000770B802F0E940A9580911E02882331F12F
:10C1A00084E0089F800111240D54124F6091B20B5E
:10C1B0007091B30B072E000C880B990B0F949B33D7
:10C1C0009B01AC01F80160817181828193810F94A0
:10C1D000373569837A838B839C8360E2CE01019635
:10C1E0000E949A89BC01C7010E9457400F900F908E
:10C1F0000F900F90DF91CF911F910F91FF90EF90D3
:10C20000089567E171E380E09ECF6CE071E381E027
:10C210009ACF20E040E060E070E0A0D481E080931D
:10C2200081061092B30B1092B20B089581E091E653
:10C23000F0CF85E091E6EDCFAF92CF92DF92EF9213
:10C24000FF920F931F936801DB01ED91FC918F0129
:10C25000041B150B241B350BAE2CEAE4EE2EEAE58D
:10C26000FE2E20D41F910F91FF90EF90DF90CF9082
:10C27000AF900895AF92CF92DF92EF92FF920F931B
:10C280001F93CF93DF9361E081E011D5D0915306E6
:10C29000C0E0D1111AC080915206811104C00E94E1
:10C2A0000F6A81111EC180911E02882309F410C1FA
:10C2B00081E090915206911180E004E024E047E093
:10C2C00051E36C2F0E94C23F03C1D13011F5809120
:10C2D0005206813021F40E940F6A811109C18091B8
:10C2E0001E02882309F4F4C011E0809152068130C7
:10C2F00009F010E080915C0290915D020E944D87F0
:10C3000000E09C014BEF50E36C2F812F0E94F63F21
:10C31000DFC0D23011F580915206823021F40E94A4
:10C320000F6A8111F7C080911E02882309F4D0C0E2
:10C3300011E080915206823009F010E08091590C92
:10C3400090915A0C0E944D8700E09C014DEE50E305
:10C350006C2F812F0E94F63FBBC0D33011F5809126
:10C360005206833021F40E940F6A8111E7C0809148
:10C370001E02882309F4ACC011E08091520683307C
:10C3800009F010E08091350C9091360C0E944D8799
:10C3900000E09C0145EE50E36C2F812F0E94F63F98
:10C3A00097C0D43001F580915206843021F40E9468
:10C3B0000F6A8111D7C080911E02882309F488C0BA
:10C3C00011E080915206843009F010E080914F0C0A
:10C3D0000E94278700E09C0141ED50E36C2F812FE4
:10C3E0000E94F63F75C0D53011F580915206853018
:10C3F00021F40E940F6A8111D2C080911E0288230D
:10C4000009F466C011E080915206853009F010E011
:10C4100080917602909177020E944D8700E09C0106
:10C4200047EC50E36C2F812F0E94F63F51C0D6306D
:10C43000D1F480915206863019F4F1D78111C1C030
:10C4400080911E02882309F443C081E09091520636
:10C45000963009F080E003E02EE34CEB50E36C2FC4
:10C460000E94C23F35C0D730C9F480915206873050
:10C4700019F4D5D78111AFC080911E02882341F1F4
:10C4800081E090915206973009F080E003E02EE3BE
:10C4900041EB50E36C2F0E94C23F1AC0D830C1F468
:10C4A00080915206883019F4BAD781119EC08091CC
:10C4B0001E02882369F081E090915206983009F0BD
:10C4C00080E003E02EE342EA50E36C2F0E94C23F7B
:10C4D000CF5FDF5FC53009F0DCCE89E08093510685
:10C4E0008DC068D380911F06882309F4DCCE86C0F6
:10C4F000E12C00E010E027EE33E04AE050E06CE58C
:10C5000072E081E091E398DE80911F06882309F4B0
:10C51000E6CE74C081E078D7E12C09E910E622E28A
:10C5200031E040E050E069E57CE084EF90E384DEB8
:10C5300080911F06882309F4F6CE60C081E064D79D
:10C54000E12C0AE71FE92CE830E040E050E065E329
:10C550007CE089EE90E370DE80911F06882309F469
:10C5600006CF4CC081E050D700914F0C10E0A12CB9
:10C5700087E7C82E80E6D82E9CE9E92E90E6F92EB2
:10C580002FEF30E040E050E06FE47CE08BED90E393
:10C5900089D280911F06882309F40DCF2FC0E12C8A
:10C5A0000DE710E627EE33E04AE050E066E772E080
:10C5B0008CEC90E341DE80911F06882309F41DCFA7
:10C5C0001DC086E191E60E94E04380911F0688230A
:10C5D00009F436CF13C089E191E60E94E0438091CF
:10C5E0001F06882309F448CF09C08DEB96E60E9408
:10C5F000E04380911F06882309F459CFDF91CF9142
:10C600001F910F91FF90EF90DF90CF90AF90089522
:10C6100060E070E080E00E94699A0E94C79FC3C2F8
:10C62000AF92CF92DF92EF92FF920F931F93CF932F
:10C63000DF9361E081E03BD3D0915306C0E0D1119C
:10C6400019C080915206811103C0E9D68111A7C09B
:10C6500080911E02882309F471C081E090915206F6
:10C66000911180E004E024E045E551E36C2F0E9445
:10C67000C23F64C0D13009F580915206813019F46F
:10C68000CED6811193C080911E02882309F456C032
:10C6900011E080915206813009F010E08091590C30
:10C6A00090915A0C0E944D8700E09C0147E451E3B1
:10C6B0006C2F812F0E94F63F41C0D23001F580914E
:10C6C0005206823019F4ABD681118EC080911E02C1
:10C6D0008823A1F111E080915206823009F010E028
:10C6E0008091350C9091360C0E944D8700E09C01A2
:10C6F0004FE351E36C2F812F0E94F63F1FC0D330D0
:10C70000E9F480915206833019F489D681118AC0E8
:10C7100080911E02882391F011E0809152068330AF
:10C7200009F010E080914F0C0E94F88600E09C0117
:10C730004BE251E36C2F812F0E94F63F8091590C00
:10C7400090915A0C2091350C3091360C232B11F41A
:10C75000892BE1F0D430C1F480915206843019F471
:10C760005ED681117CC080911E02882369F081E031
:10C7700090915206943009F080E000E22EE342E20C
:10C7800051E36C2F0E94C23F85E001C084E0CF5F7F
:10C79000DF5FC53009F053CF8093510666C00AD2DF
:10C7A00080911F06882309F453CF5FC081E02CD607
:10C7B0000091590C10915A0CA12C49E9C42E40E665
:10C7C000D42E5AE4E52E5AE5F52E22E231E040E07F
:10C7D00050E069E57CE08EE491E364D180911F062E
:10C7E000882309F450CF41C081E00ED60091350C6A
:10C7F0001091360CA12C2AE7C22E2FE9D22E3AE452
:10C80000E32E3AE5F32E2CE830E040E050E065E31B
:10C810007CE083E491E346D180911F06882309F4EC
:10C8200055CF23C081E0F0D500914F0C10E0A12C32
:10C8300087E7C82E80E6D82E9EE4E92E95E4F92EEF
:10C840002FEF30E040E050E06FE47CE085E391E3DF
:10C8500029D180911F06882309F45ACF06C0D8DE5B
:10C8600080911F06882309F47ECFDF91CF911F911D
:10C870000F91FF90EF90DF90CF90AF9008950F93BE
:10C880001F93CF93DF9361E081E011D2D0915306E3
:10C89000C0E0D11116C080915206811103C0BFD5EE
:10C8A00081119AC080911E02882309F43CC081E066
:10C8B00090915206911180E004E024E049EA51E3AE
:10C8C0002FC0D130B1F480915206813019F4A7D530
:10C8D000811189C080911E02882329F181E0909105
:10C8E0005206913009F080E003E02EE347E951E37E
:10C8F00017C0D230C1F480915206823019F48FD51E
:10C9000081117BC080911E02882369F081E09091A3
:10C910005206923009F080E003E02EE348E851E34C
:10C920006C2F0E94C23F03D1182FD330D1F48091D5
:10C930005206833019F473D5811169C080911E02AB
:10C94000882309F476C081E090915206933009F073
:10C9500080E000E22EE349E751E36C2F0E94C23FE2
:10C9600068C0811168C0D430B1F48091520684301F
:10C9700019F455D5811152C080911E02882319F1F6
:10C9800081E090915206943009F080E000E22EE3BD
:10C990004BE651E315C0D530B1F480915206853095
:10C9A00009F443C080911E02882369F081E09091D0
:10C9B0005206953009F080E000E22EE34AE551E3AB
:10C9C0006C2F0E94C23F86E0CF5FDF5FC53009F069
:10C9D00060CF809351063AC0EDD080911F06882326
:10C9E00009F460CF33C080ED98E40E94E043809169
:10C9F0001F06882309F46ECF29C08DEB96E60E94AE
:10CA0000E04380911F06882309F47CCF1FC04CD2DD
:10CA100080911F06882309F491CF18C048D28091D5
:10CA20001F06882309F4A8CF11C0F9D4811105C0CD
:10CA3000B9CF112341F284E0C7CF0E9410BF81E03B
:10CA400088D180911F06882309F4ACCFDF91CF9164
:10CA50001F910F910895E0912006E63000F581E0E6
:10CA60008E0F809320068091790690917A06A0E03F
:10CA7000B0E0309153062091510648E0E49FF00168
:10CA80001124EF5DF94F4091740650917506518362
:10CA9000408382839383A483B58336832783089559
:10CAA0000D94EA214F925F926F927F928F929F92A4
:10CAB000AF92CF92DF92EF92FF920F931F93CF939B
:10CAC000DF933C014B01EA012901C5DF83E080933C
:10CAD0001E0270921E0660921D0690921C068092A5
:10CAE0001B06D0931A06C09319065092180640925E
:10CAF000170610937A0600937906F0927506E09275
:10CB00007406D0921606C0921506A0921406DF9104
:10CB1000CF911F910F91FF90EF90DF90CF90AF904A
:10CB20009F908F907F906F905F904F90089580912D
:10CB3000210E90911E0E891B8F7071F49091EA085E
:10CB400092FB882780F992FD08C081E090918316BE
:10CB5000913019F080E0089581E00895E091740625
:10CB6000F0917506E817F907E9F090937506809340
:10CB7000740670937A066093790640935306209367
:10CB800051068F56994621F4109281061092200684
:10CB90000E94F83E82E080931E0281E080931F068F
:10CBA00010927C06089520E040E060E070E08FE69F
:10CBB00099E6D4CFE0912006EE2381F0E150E09396
:10CBC000200688E0E89FF0011124EF5DF94F2781EE
:10CBD000468160E070E080819181C0CFE4CFCF9347
:10CBE000DF93FC01EB018091790690917A0697FF23
:10CBF00004C010927A06109279062091170630919F
:10CC000018068091790690917A062817390724F43E
:10CC100030937A062093790680911E02882391F042
:10CC20002091190630911A068091790690917A0622
:10CC3000820F931F1995BC0180911D0690911E06CD
:10CC40000E94574080916E06811108C080911406A1
:10CC5000882351F180911E02882331F180911B06B7
:10CC600090911C06009761F06091190670911A0668
:10CC70002091790630917A06620F731FFE01199593
:10CC8000E0911506F0911606309741F08091140658
:10CC9000811103C080916E0681111995C0D388233C
:10CCA00019F0DF91CF9186CFDF91CF910895282F92
:10CCB000109273068091790690917A06813090489F
:10CCC00020F010927A061092790680917B068823D4
:10CCD00031F0809179068093520610921F06809160
:10CCE00051061816BCF4082E000C990B821B9109F2
:10CCF00020915206022E000C330B2817390754F0EE
:10CD000097FF02C080E090E08093520690937A06ED
:10CD100080937906809152066623C1F09091530664
:10CD2000891714F48093530620915306022E000CA9
:10CD3000330B2C5F3F4F482F082E000C550B241748
:10CD4000350734F484508093530608958093530636
:10CD50000895882361F063E972E084E690E00F941F
:10CD6000042D6AEB72E084E690E00D94042D68EBEC
:10CD700071E084E190E00D94042D8F929F92AF9228
:10CD8000BF92CF92DF92EF92FF9249D3882369F04E
:10CD90000E946DBB10928106FF90EF90DF90CF90C4
:10CDA000BF90AF909F908F9005CF81E080938106D8
:10CDB000C0907906D0907A06C114D10409F444C019
:10CDC00010927A06109279060D2C000CEE08FF08DE
:10CDD000C701B6010F949B332091BB0D3091BC0D60
:10CDE0004091BD0D5091BE0D0F9437352091F30C3D
:10CDF0003091F40C4091F50C5091F60C0F942032C8
:10CE00004B015C0120E030E040E050EC0F94FC343A
:10CE100087FD1AC020E030E040EA50E4C501B401CB
:10CE20000F94F932181684F0B701A60182E00E942F
:10CE30000A958092F30C9092F40CA092F50CB092AB
:10CE4000F60C82E080931E0280911E028823D9F0A6
:10CE500083EF9CE00E94EC87BC018EEA91E30E9484
:10CE600057406091F30C7091F40C8091F50C909107
:10CE7000F60CFF90EF90DF90CF90BF90AF909F9017
:10CE80008F900C949841FF90EF90DF90CF90BF90DF
:10CE9000AF909F908F90089521E0209313060F94F8
:10CEA000EF211092130608950E94A8BB52CF0E9452
:10CEB00032C94FCFEF92FF920F931F93E091790603
:10CEC000F0917A06309759F0A1E01E161F060CF07B
:10CED000A0E0FA01A08310927A0610927906FA0176
:10CEE00040810E942A411F910F91FF90EF90089579
:10CEF000FC0180810895FC01849108954F925F9216
:10CF00006F927F928F929F92AF92BF92CF92DF9259
:10CF1000EF92FF920F931F93CF93DF936C017B01EE
:10CF20005A012901672B31F088248394912CC0E0A9
:10CF3000D0E019C0F8011182108227C03701680CB7
:10CF4000791C76946794E3012197A201BE01C60182
:10CF5000F50119951816190654F0892BC9F04301EB
:10CF6000FFEF8F1A9F0AE814F90440F702C07E0110
:10CF7000FACFCE15DF0530F4CE0102968816990659
:10CF800020F02196F801D183C0838FEF9FEF05C079
:10CF9000F801D183C08380E090E0DF91CF911F91B1
:10CFA0000F91FF90EF90DF90CF90BF90AF909F9048
:10CFB0008F907F906F905F904F9008958F929F9287
:10CFC000AF92BF92CF92DF92EF92FF920F931F9397
:10CFD000CF93DF93EC016B017A01FB01199587FD7B
:10CFE00006C0082F10E020E030E0219620C1982FE5
:10CFF000907E903CC1F4082F0F7110E020E030E0EB
:10D000004801590186E0880C991CAA1CBB1C8A9512
:10D01000D1F7CE010196F60119958F739501840120
:10D02000082B229604C1982F907F903E19F58F709F
:10D03000882E912CA12CB12C16E0880C991CAA1CCE
:10D04000BB1C1A95D1F7CE010196F60119958F7385
:10D05000882A06E0880C991CAA1CBB1C0A95D1F7EB
:10D06000CE010296F60119958F7395018401082B64
:10D070002396DDC0982F987F903F81F58770882E8A
:10D08000912CA12CB12CF6E0880C991CAA1CBB1C7D
:10D09000FA95D1F7CE010196F60119958F73882A7A
:10D0A000A6E0880C991CAA1CBB1CAA95D1F7CE013E
:10D0B0000296F60119958F73882AB6E0880C991CA0
:10D0C000AA1CBB1CBA95D1F7CE010396F60119959F
:10D0D0008F7395018401082B2496A9C0982F9C7FFB
:10D0E000983FE9F58370882E912CA12CB12C56E045
:10D0F000880C991CAA1CBB1C5A95D1F7CE0101962D
:10D10000F60119958F73882A66E0880C991CAA1C71
:10D11000BB1C6A95D1F7CE010296F60119958F7363
:10D12000882A76E0880C991CAA1CBB1C7A95D1F73A
:10D13000CE010396F60119958F73882AE6E0880CD4
:10D14000991CAA1CBB1CEA95D1F7CE010496F601E6
:10D1500019958F7395018401082B259668C0982F27
:10D160009E7F9C3F09F04AC08170882E912CA12C93
:10D17000B12C86E0880C991CAA1CBB1C8A95D1F79F
:10D18000CE010196F60119958F73882A96E0880CD6
:10D19000991CAA1CBB1C9A95D1F7CE010296F601E8
:10D1A00019958F73882A26E0880C991CAA1CBB1C31
:10D1B0002A95D1F7CE010396F60119958F73882A27
:10D1C00036E0880C991CAA1CBB1C3A95D1F7CE01FD
:10D1D0000496F60119958F73882A46E0880C991CED
:10D1E000AA1CBB1C4A95D1F7CE010596F6011995EC
:10D1F0008F7395018401082B269619C0982F907C77
:10D20000903849F4082F007C003871F42196CE0143
:10D21000F6011995F7CF082F0E7F0D3F28F02196C4
:10D22000CE01F6011995F7CF00E010E09801E11466
:10D23000F10429F0F7010083118322833383CE01A7
:10D24000DF91CF911F910F91FF90EF90DF90CF90E2
:10D25000BF90AF909F908F9008951F93CF93DF93CF
:10D2600000D01F92CDB7DEB710E0AE014F5F5F4F29
:10D2700068E777E6A3DE49815A816B817C81452B83
:10D28000462B472B11F01F5FF0CF812F0F900F908F
:10D290000F900F90DF91CF911F9108951F93CF931F
:10D2A000DF9300D01F92CDB7DEB710E0AE014F5F25
:10D2B0005F4F6BE777E682DE49815A816B817C8123
:10D2C000452B462B472B11F01F5FF0CF812F0F907E
:10D2D0000F900F900F90DF91CF911F9108951092B2
:10D2E000730680916E0610926E06882349F020E046
:10D2F00040E060E070E084E49EE530DC0C94C43EE5
:10D3000020915C0230915D024091790650917A063D
:10D31000C901840F951F2436310551F4473051055A
:10D3200014F006972CC04A3F5F4F34F5069627C08D
:10D330002436310524F485369105F4F404C084368E
:10D34000910524F419C08A3091053CF0883E43E0F1
:10D3500094072CF087EE93E002C08AE090E0281753
:10D36000390741F090935D0280935C0210927A0637
:10D37000109279060C94083784E690E0E7CF8A3063
:10D38000910524F78AE090E0EDCFCF93DF931F92D1
:10D39000CDB7DEB780919B08811103C08DED98E079
:10D3A0002FC0211103C08BE998E02AC08DE0815085
:10D3B00048F0440F411DE82FF0E0E352F74F908111
:10D3C0004927F5CF809165068417A9F0409365063B
:10D3D0008BE998E0698341DF90E06981861B9109C0
:10D3E00097FF02C080E090E0809376061092770667
:10D3F00088E0809320028091770690E08556974FD1
:10D400000F90DF91CF9108958093730610926F066D
:10D410001092700610927106109272060895809113
:10D420006E0610926E060895DF92EF92FF920F93B0
:10D430001F93CF93DF9300D01F92CDB7DEB7082F95
:10D440006115710559F1E62ED72E15E18CE0F82E05
:10D45000153159F411E0100F6F2DF09E600D11245D
:10D4600080E00E947B36012F10E0AE014F5F5F4FDE
:10D4700068E777E68E2D9D2DA1DDE82ED92E6981F6
:10D480007A818B819C81611571058105910531F04F
:10D490004FEF5FEF0E9480361F5FDACF0F900F9043
:10D4A0000F900F90DF91CF911F910F91FF90EF9010
:10D4B000DF900895CF92DF92EF92FF920F931F9328
:10D4C0000E94BC2B009161061091620620916306B8
:10D4D000309164066B017C01C01AD10AE20AF30A9A
:10D4E000F7FC13C020916006209520936006DC01B4
:10D4F000CB018A549C4FAF4FBF4F809361069093EE
:10D500006206A0936306B093640681E09091600682
:10D51000911101C080E01F910F91FF90EF90DF907B
:10D52000CF900895CF9393E090931E0281111092B3
:10D5300083060E94BC2BDC01CB018C509E4FAF4F69
:10D54000BF4F80937D0690937E06A0937F06B09395
:10D55000800668E873E182E090E00F94042DC6E055
:10D56000C15049F00F94992C62E070E080E090E0A7
:10D570000E94ED2BF5CFCF910895AF92BF92CF923D
:10D58000DF92EF920F931F93CF93DF9300D01F9200
:10D59000CDB7DEB780911F028F3F09F444C00E94CF
:10D5A000BC2B0091660610916706209168063091A9
:10D5B0006906DC01CB01801B910BA20BB30BB7FDFD
:10D5C00032C090911E0E8091210E8F5F8F70981740
:10D5D00051F1E0911F0284E0E802F0011124E25FC2
:10D5E000FB4F20E030E040E752E4608171818281AE
:10D5F00093810F94003369837A838B839C83A12C5E
:10D60000B12C6501E12C8E010F5F1F4F2EE632E039
:10D610004AE652E066E672E082E692E00E94D8E7CF
:10D620008FEF80931F020F900F900F900F90DF915C
:10D63000CF911F910F91EF90DF90CF90BF90AF905F
:10D6400008950F931F930E94BC2B00917D061091AB
:10D650007E0620917F0630918006DC01CB01801B85
:10D66000910BA20BB30BB7FD11C08091030181FB9D
:10D67000992790F981E089279091030192FF8260B8
:10D680009091000196FF84608093830680918306C9
:10D6900081709091830691FD826090915406891764
:10D6A00041F18130A9F028F0823041F0833059F007
:10D6B0001EC0913089F09230A9F019C0992361F011
:10D6C000933081F014C0913069F0923081F404C03D
:10D6D000992341F0933059F49091780691509093AA
:10D6E000780605C0909178069F5F909378068093A6
:10D6F00054061F910F910895CF93DF930E94C43E6B
:10D70000E4E0F1E080818D7F8083C5E0D1E0888115
:10D710008095827043E051E0DA018C9380818B7FA9
:10D7200080838881809584708C9321E031E0D901D9
:10D730008C918F7B8C938091020180958074809373
:10D74000000180818E7F8083888180958170FA01BD
:10D75000808382E08093820674DF10927806DF91E6
:10D76000CF91089581E090918506911101C080E0EC
:10D770000895CF93DF9320919B0621111EC0FC01D9
:10D7800001900020E9F73197EF01C81BD90BC63192
:10D79000D10534F031972081207C2038D9F3F4CFA3
:10D7A000BC01DD27AE0185E896E00F94323BCB57F4
:10D7B000D94F188283E080931E02DF91CF910895A4
:10D7C000CF93DF93CDB7DEB78E8190919B068917FB
:10D7D00080F080939B069E01275F3F4F4F815885C5
:10D7E00065E170E085E896E00F947B3B83E08093F1
:10D7F0001E02DF91CF9108950F931F93CF93DF9374
:10D800008C0167FF03C010929B0660E080919B062D
:10D8100090E0262F062E000C330B281739070CF149
:10D8200060939B06C8010F94943AF801E80FF91F22
:10D83000EF01C01BD10BC631D10534F03197849173
:10D84000807C8038D9F3F4CFDD27AE01B80185E8BC
:10D8500096E00F94B53ACB57D94F188283E0809366
:10D860001E02DF91CF911F910F9108954F925F9209
:10D870006F927F928F929F92AF92BF92CF92DF92E0
:10D88000EF92FF920F931F9378DEDBDE8091830689
:10D8900082FF15C080915F06811113C091E09093C3
:10D8A0005F0620919016211103C0809113068927ED
:10D8B00080936E061092901681E034DE02C01092C2
:10D8C0005F06809103018095817010918206811717
:10D8D000B9F080938206882309F4BCC164EF71E03B
:10D8E00080E090E00E94B4860E94DB77123009F05D
:10D8F000ACC10E94AB7883E080931E020E94C43EBC
:10D900000E94BC2B6B017C0180915B0690915C06B0
:10D91000A0915D06B0915E06A7019601281B390B08
:10D920004A0B5B0B57FF05C080917C06882309F4E6
:10D9300026C2D701C6018C599F4FAF4FBF4F80936E
:10D940005B0690935C06A0935D06B0935E066091C3
:10D950007806062E000C770B77FF03C07195619552
:10D960007109062E000C770B880B990B0F949B33D3
:10D970002B013C0120E030E040E050E40F94FC3407
:10D9800087FF05C080916E0681117DC08DC080919A
:10D990007306882309F456C080906F069090700635
:10D9A000A0907106B090720681149104A104B10494
:10D9B000E1F120E030E040E05FE3C301B2010F9409
:10D9C00037352B013C01C701B601681979098A096D
:10D9D0009B090F9499339B01AC01C301B2010F94D1
:10D9E000003320E030E04AE754E40F9437354B0130
:10D9F0005C0120E030E040EA52E40F94FC3487FF01
:10DA00000FC020E030E040EF51E4C501B4010F94B5
:10DA1000FC3487FD0AC02AE030E040E050E009C055
:10DA200024E630E040E050E004C021E030E040E097
:10DA300050E0C0926F06D0927006E0927106F092AC
:10DA4000720604C021E030E040E050E0A09178068A
:10DA50000091790610917A060A2E000CBB0B0F94E8
:10DA6000A83622E030E040E050E00F946536DA015D
:10DA7000C901800F911FA11DB11D90937A0680935B
:10DA8000790610927806D701C6018856954CAF4F9B
:10DA9000BF4F8093570690935806A0935906B093B2
:10DAA0005A0681E080931E0220917406309175061B
:10DAB00049E62F36340741F480912002882309F487
:10DAC000DCC08150809320022954344451F5809168
:10DAD0002002882321F081508093200222C084E01C
:10DAE00080932002809177068F5F809377069091D4
:10DAF0007606981728F4109277068CE0809320021F
:10DB000081E080931E02D701C6018856954CAF4F25
:10DB1000BF4F8093570690935806A0935906B09331
:10DB20005A0680916F0081FB222720F981FF05C0F2
:10DB300080916F008D7F80936F008091310D909167
:10DB4000320DA091330DB091340D222329F0209194
:10DB50006F00226020936F003AE0B695A7959795E5
:10DB600087953A95D1F7009721E0A207B10520F0FB
:10DB70008FEF9FEFA0E0B0E09695879520911E0271
:10DB8000211105C030917C063111F5C051C00097BC
:10DB900041F040915506509156064817590708F034
:10DBA00047C080917C06811117C0223008F075C0F3
:10DBB0008091FE04811107C081E08093FE0485EC12
:10DBC00094E00E94843085EC94E00E94BB3081E0B8
:10DBD00080937B0680937C0683E00E94043E61E094
:10DBE00085EC94E00E94E430E0917406F0917506B3
:10DBF000199510927B0680917C0681115AC0109273
:10DC00006E060E94BC2BDC01CB018C199D09AE096C
:10DC1000BF09009155061091560620E030E0081724
:10DC200019072A073B0720F4909356068093550660
:10DC300080917406909175068F56994609F45FC0DD
:10DC40008091810681115BC085C060E087EF91E320
:10DC5000D3DD51CEA7D5123009F44DCE60E08AEE67
:10DC600091E3CADD80917406909175068F569946AE
:10DC700009F441CE0E94D3653ECE8CE08093200211
:10DC80008091550690915606019790935606809381
:10DC9000550681E080931E0217CF243030F02430E7
:10DCA00009F086CF10921E0283CF81E080931E027E
:10DCB0007FCF85EC94E00E94BF3091E0811101C0DC
:10DCC00090E090937C06992309F499CF0E94BC2B95
:10DCD000DC01CB018C199D09AE09BF09C090550626
:10DCE000D0905606E12CF12CC816D906EA06FB06A0
:10DCF00008F045C0909356068093550640C048E909
:10DD0000C40E4AE3D41EE11CF11CC0925706D09207
:10DD10005806E0925906F0925A0680917C068111CD
:10DD20002EC080911E02813091F0833041F51F9109
:10DD30000F91FF90EF90DF90CF90BF90AF909F90AA
:10DD40008F907F906F905F904F900C94F83E109260
:10DD50001E0215C08091570690915806A091590651
:10DD6000B0915A06C81AD90AEA0AFB0AF7FCD5CFBD
:10DD70000E94D365D2CF009709F42ECF0ACF1F910E
:10DD80000F91FF90EF90DF90CF90BF90AF909F905A
:10DD90008F907F906F905F904F90089561E02CDDA1
:10DDA0000C94D365CF93DF931F921F92CDB7DEB74C
:10DDB00089839A83A1DC89819A81F0DF0F900F908B
:10DDC000DF91CF910C94C93E8091EA0882FD05C095
:10DDD00080918316823061F410C080919B0881117C
:10DDE00003C08DED98E002C08BE998E061E0C1CC02
:10DDF000813031F08DEB91E305C08DED91E302C0F0
:10DE000081ED91E36FEFF8CC8091EA0882FF09C0C1
:10DE100083FF04C080911A07811106C020E020937F
:10DE200084068091840608958091A5069091A606A7
:10DE3000A091A706B091A8060097A105B10571F3BE
:10DE4000BC01CD016D597F4F8F4F9F4F24E630E0CD
:10DE500040E050E00F9443366091A1067091A20615
:10DE60008091A3069091A4060F944336D8CF8FE6F5
:10DE700099E69093750680937406089561E0FC011D
:10DE800080810E94E12D8FEF0C944B94CF93DF9310
:10DE9000EC018A810E940C9460E08881DF91CF912F
:10DEA0000C94E12D8F929F92AF92BF92EF92FF92CE
:10DEB0000F931F93CF93DF93EC018B017A010E94A4
:10DEC000BC2B4B015C012CE2820E21E0921EA11CB6
:10DED000B11C0E9425948B838F3F61F40E94BC2B60
:10DEE000DC01CB0188199909AA09BB09B7FDF1CF5B
:10DEF00081E10DC08E3F51F4B701C8010E942C94FE
:10DF00000E9425940E94259411E003C08FE089832C
:10DF100010E0CE01B3DF812FDF91CF911F910F91E0
:10DF2000FF90EF90BF90AF909F908F900895CF9209
:10DF3000DF92EF92FF926A017B010E94BC2BC60E1A
:10DF4000D71EE81EF91E0E9425948F3F61F00E94A3
:10DF5000BC2BDC01CB018C199D09AE09BF09B7FDB3
:10DF6000F2CF80E001C081E0FF90EF90DF90CF9092
:10DF70000895EF92FF921F93CF93DF9300D01F92EB
:10DF8000CDB7DEB77C01162F29833A834B835C83A0
:10DF90007DDF48E552E060E070E0C701C8DF812F17
:10DFA00080640E944B948C810E944B948B810E94D0
:10DFB0004B948A810E944B9489810E944B94112337
:10DFC00011F087E801C085E90E944B941C3011F4E0
:10DFD0000E94259410E00E942594F701838387FF17
:10DFE00004C01F3F11F01F5FF6CF0F900F900F90EE
:10DFF0000F90DF91CF911F91FF90EF9008958F9236
:10E000009F92AF92BF92CF92DF92EF92FF920F93C7
:10E010001F93CF93DF93EC01162F1C821982488344
:10E020000E94BC2B6B017C0120EDC20E27E0D21EAA
:10E03000E11CF11CA89561E088810E94E12D61E05E
:10E0400088810E94A52D0E941D9485E08A830E94EC
:10E050000C940AE08FEF0E944B940150D9F7A895D9
:10E0600020E030E0A90160E0CE0183DF8B838130C6
:10E0700061F00E94BC2BDC01CB018C199D09AE091B
:10E08000BF09B7FDEDCF81E055C0A8952AEA31E080
:10E0900040E050E068E0CE016CDF853011F481E0B3
:10E0A00009C004E00E9425948B830150D9F78A3A75
:10E0B00051F482E08C83A8958C81823081F0812C90
:10E0C000912C540111C00E94BC2BDC01CB018C1996
:10E0D0009D09AE09BF09B7FDD9CF82E02BC0812CC5
:10E0E000912CA12C80E4B82E20E030E0A90167E358
:10E0F000CE013FDFA501940169E2CE013ADF8B83B7
:10E10000882361F00E94BC2BDC01CB018C199D0996
:10E11000AE09BF09B7FDE8CF8AE00CC08C81823020
:10E12000D1F420E030E0A9016AE3CE0122DF8823A8
:10E1300029F088E08983CE01A1DE16C00E942594D3
:10E14000807C803C11F483E08C830E9425940E94A3
:10E1500025940E942594CE0191DE173018F41A837D
:10E1600081E003C088E1898380E0DF91CF911F9136
:10E170000F91FF90EF90DF90CF90BF90AF909F9066
:10E180008F9008950F931F93CF93DF93EC01890134
:10E190008C81833039F089E0440F551F661F771F4B
:10E1A0008A95D1F79A01AB0161E1CE01E2DE8111DE
:10E1B00009C040E052E0B801CE01DF91CF911F913C
:10E1C0000F9170CE84E08983CE0158DE80E0DF912C
:10E1D000CF911F910F910895CF93DF93EC01862F7C
:10E1E000BA010E9450948FEF0E944B948FEF0E94CF
:10E1F0004B940E9425948B83982F9F71953031F01A
:10E2000083E18983CE013ADE80E001C081E0DF91C5
:10E21000CF9108950F931F93CF93DF93EC01890162
:10E220008C81833039F089E0440F551F661F771FBA
:10E230008A95D1F79A01AB0168E1CE019ADE81118E
:10E240001EC0A8016EEFCE01C7DF8823E1F048E5CC
:10E2500052E060E070E0CE016ADE882371F020E0D9
:10E2600030E0A9016DE0CE0184DE81110AC00E9478
:10E270002594811106C011E007C087E103C086E044
:10E2800001C086E1898310E0CE01F8DD812FDF91A6
:10E29000CF911F910F910895CF93DF931F92CDB728
:10E2A000DEB72091921630919316CE01019621157A
:10E2B000310519F0821B930B02C0885996410F90CB
:10E2C000DF91CF910895FC01238121110C940582E7
:10E2D00008958091EA08847F8B7F8093EA081092EA
:10E2E000A1061092A2061092A3061092A406109204
:10E2F000A5061092A6061092A7061092A8061092E4
:10E300001607109255078EE091E0E6E5F7E0DF0191
:10E310009C011D9221503040E1F78FEF80939A08C5
:10E320000895FC0120E03EE2DB014C91403241F0D7
:10E33000283011F430833196DB014C9140833196C3
:10E340002F5F6F5F7F4F2B3079F7108208952F92E8
:10E350003F924F925F926F927F928F929F92AF9275
:10E36000BF92CF92DF92EF92FF920F931F93CF93C2
:10E37000DF93CDB7DEB7C356D1090FB6F894DEBF31
:10E380000FBECDBF8C015B014A014DB65EB6312C8C
:10E390007E0187E5E80EF11C9BE1292E4BE958E050
:10E3A000BE016F5F7F4FC5010E94758018160CF08B
:10E3B00005C18C85282F2871203109F074C09091F7
:10E3C000A0069150923008F46EC06DB67EB6BE01C4
:10E3D0006F5F7F4FC701A5DF0115110521F0F8011F
:10E3E0008081811173C021E081E090E0F70101900C
:10E3F0000020E9F73197EE19FF09E80FF91F32966F
:10E400008DB79EB78E1B9F0B0FB6F8949EBF0FBEA5
:10E410008DBFEDB7FEB731966F01211102C0B80173
:10E4200002C06EE174E0C6010F941D3BB701C60146
:10E430000F94073B6EE174E0C6010F94073B1CAEDE
:10E440001FAE21E0A701B501CE01CC960E94018448
:10E4500081110DC08091A006811109C00E94498DD3
:10E4600083EF93E30E943B8DC7010E94E292FE017D
:10E47000FC96DE019196822D01900D928A95E1F72E
:10E4800040E050E0BE016F5D7F4FC60160DFCE010E
:10E49000819619DFCE01CC9616DF0FB6F8947EBEBA
:10E4A0000FBE6DBE7BCF9981992309F487C0953E3D
:10E4B00009F474CF9E3209F471CF90919B089E327B
:10E4C00009F46CCF8A7009F069CF0AC0F801019095
:10E4D0000020E9F73197CF01801B910B20E086CF18
:10E4E00081E0203109F080E09091EA0880FB94F906
:10E4F0009093EA08811108C08985873409F04ECFCE
:10E500008A858E3709F44ACF8091A006813021F0A8
:10E5100068F08230B9F142CF80919E0690919F06BB
:10E52000019690939F0680939E0638CFBE016F5F41
:10E530007F4F8DED98E0F5DE0115110511F06801B2
:10E5400005C08DEDC82E88E0D82E08C0F601819157
:10E550006F018823B1F30E948B92F8CFF60181916D
:10E560006F01882319F00E948B92F8CF80E20E94FD
:10E570008B926D8D7E8D8F8D98A14AE050E00E9428
:10E5800098930CCFBE016F5F7F4F8DED98E0C9DE91
:10E590008114910441F06DED78E0C4010F94F43AD8
:10E5A000892B51F40BC0832D90E020919C06309173
:10E5B0009D068217930711F03394F0CE0FB6F894AE
:10E5C0005EBE0FBE4DBECD59DF4F0FB6F894DEBF15
:10E5D0000FBECDBFDF91CF911F910F91FF90EF90B4
:10E5E000DF90CF90BF90AF909F908F907F906F9073
:10E5F0005F904F903F902F900895CF93DF93CDB7CA
:10E60000DEB76B970FB6F894DEBF0FBECDBF10928A
:10E61000A00640E050E0BA018FE798E00E94248114
:10E620008BE1EFE7F8E0DE01119601900D928A95FB
:10E63000E1F740E050E0BE016F5F7F4F80E090E087
:10E6400086DECE0101963FDE6B960FB6F894DEBFF4
:10E650000FBECDBFDF91CF9108950F931F93CF933E
:10E66000DF93CDB7DEB72D970FB6F894DEBF0FBEA0
:10E67000CDBF80911A07882391F0BE016F5F7F4F55
:10E6800087E197E00E94977E8E010F5F1F4FF80190
:10E6900081918F01882339F00E948B92F8CF89EE07
:10E6A00093E30E943B8D8AE00E948B922D960FB6D9
:10E6B000F894DEBF0FBECDBFDF91CF911F910F91B8
:10E6C0000895CF92DF92EF92FF920F931F93CF9313
:10E6D000DF93CDB7DEB7EDB6FEB6DC010D900020BE
:10E6E000E9F79D01281B390B2C5F3F4F4DB75EB7F3
:10E6F000421B530B0FB6F8945EBF0FBE4DBF0DB754
:10E700001EB70F5F1F4F9F938F9383EA93E39F93EF
:10E710008F931F930F930F944C3B680154E0C50EE9
:10E72000D11C0F900F900F900F900F900F90F6014B
:10E730008081882349F0082E000C990B0F94783AB9
:10E74000F60181936F01F3CFC8010F94EF218FE998
:10E7500093E30F94EA210FB6F894FEBE0FBEEDBE10
:10E76000DF91CF911F910F91FF90EF90DF90CF90AD
:10E7700008958091EA0883FF03C084608093EA08CB
:10E7800008951092BF0B8091EA088F7D8B7F809354
:10E79000EA080E94B05D882321F087E197E00C949D
:10E7A00005820895EEDF8091EA08877F8093EA086A
:10E7B00008950F931F93CF93DF938B01EA01DB0141
:10E7C0006D917C910E94977ED801ED91FC91908192
:10E7D000888191110EC08936B0F48FE28083F801F0
:10E7E0008081918101969183808388818F5F888366
:10E7F0000AC0893680F73196D801ED93FC93888161
:10E800008F5F8883E1CFDF91CF911F910F910895A2
:10E810000F931F93CF93DF9300D0CDB7DEB79C014A
:10E820002F5F3F4F3B832A832FE2FC01208381E04F
:10E83000898310E00BE180915507181770F4019F50
:10E84000C0011124AE014F5F5F4FBE016E5F7F4F6D
:10E850008A5A984FAEDF1F5FEECF89818B3570F4F7
:10E86000AE014F5F5F4FBE016E5F7F4F87E197E064
:10E87000A0DF8A819B8101979B838A83EA81FB8148
:10E8800010820F900F900F90DF91CF911F910F91F9
:10E8900008958091EA0882FF1FC087E692E30E94F4
:10E8A0003B8D6091A1067091A2068091A306909184
:10E8B000A4064AE050E00E948D938FE20E948B9262
:10E8C0006091A5067091A6068091A7069091A80672
:10E8D0004AE050E00C94989386E592E30C943B8DCB
:10E8E000EF92FF920F931F93CF93DF938C01FC0164
:10E8F00001900020E9F73197EF01C81BD90B109266
:10E9000017076EE470E00F94123B7C01009729F426
:10E91000FE013197E00FF11F0EC060E270E00F942E
:10E92000123B8C010F5F1F4F6AE270E0C7010F942A
:10E93000123BFC0131978DE081838AE08283138250
:10E94000B80187E197E00E94948680911707882399
:10E9500061F00E944C8D8FE392E3DF91CF911F9184
:10E960000F91FF90EF900C943B8DDF91CF911F9111
:10E970000F91FF90EF90089587E197E00E94BA8190
:10E9800087E197E00E9405828091EA088D7F8E7F63
:10E990008093EA081092A1061092A2061092A30694
:10E9A0001092A40681E08093B00B08950F931F93FB
:10E9B000CF93DF93CDB7DEB76B970FB6F894DEBF7A
:10E9C0000FBECDBF8B0122E02093A00690939D0641
:10E9D00080939C0640E050E0BA0184E698E00E94F3
:10E9E00024818BE1E4E6F8E0DE01119601900D92BE
:10E9F0008A95E1F7A801BE016F5F7F4F80E090E04C
:10EA0000A6DCCE0101965FDC6B960FB6F894DEBFF4
:10EA10000FBECDBFDF91CF911F910F910895CF937E
:10EA2000DF93CDB7DEB76B970FB6F894DEBF0FBE9E
:10EA3000CDBF81E08093A00610929F0610929E06A3
:10EA400040E050E0BA0184E698E00E9424818BE126
:10EA5000E4E6F8E0DE01119601900D928A95E1F767
:10EA600040E050E0BE016F5F7F4F80E090E06FDCE0
:10EA7000CE01019628DC80919E0690919F066B96B0
:10EA80000FB6F894DEBF0FBECDBFDF91CF910895D2
:10EA90002F923F924F925F926F927F928F929F92AE
:10EAA000AF92BF92CF92DF92EF92FF920F931F939C
:10EAB000CF93DF93CDB7DEB76C970FB6F894DEBF78
:10EAC0000FBECDBF5C014C8F2DB63EB619821C82A5
:10EAD000FB0180819E012F5F3F4F49018F3239F04A
:10EAE00084E698E0F501918380838B0160C08FE715
:10EAF00098E0F501918380838B010F5F1F4F011513
:10EB0000110509F454C04DB65EB66FE270E0C8015D
:10EB10000F94123B3C010817190708F048C07C010C
:10EB2000E01AF10AFF24C70101962DB73EB7281B52
:10EB3000390B0FB6F8943EBF0FBE2DBF8DB79EB7F1
:10EB400001966C01A701B8010F94323BF601EE0D5E
:10EB5000FF1D10823C8D332319F0C6010E94E29202
:10EB6000F5016081718121E0A601C4010E94018448
:10EB7000811111C0B60182E292E30E944F8D8FE1B4
:10EB800092E30E943B8D0FB6F8945EBE0FBE4DBE61
:10EB900000E010E00CC0F5019182808283010F5FDC
:10EBA0001F4F0FB6F8945EBE0FBE4DBEA8CFC40176
:10EBB0008ADBC8010FB6F8943EBE0FBE2DBE6C9620
:10EBC0000FB6F894DEBF0FBECDBFDF91CF911F917E
:10EBD0000F91FF90EF90DF90CF90BF90AF909F90FC
:10EBE0008F907F906F905F904F903F902F900895FF
:10EBF0000F931F93CF93DF931F921F92CDB7DEB772
:10EC00002091EA0823FF28C0BC0140E0CE01019614
:10EC10003FDF8C01009701F1BC0189819A810E943C
:10EC2000DB84B801882381F084E992E30E944F8D50
:10EC30008AE00E948B921092A1061092A206109276
:10EC4000A3061092A40608C08CE792E30E944F8DA1
:10EC500089E792E30E943B8D0F900F90DF91CF9157
:10EC60001F910F910895EF92FF920F931F93CF93EF
:10EC7000DF9300D0CDB7DEB72091EA0823FF09C1AA
:10EC8000F42EE62E8C010E94B05D882309F451C059
:10EC9000FF2009F45BC080911607882359F00E9479
:10ECA0004C8D8AE593E30E943B8D80E090E00F94C9
:10ECB0004730EFC089EA96E0ABDDE091160784E0CB
:10ECC000E89FF0011124EE5EF84F8091A10690912B
:10ECD000A206A091A306B091A40680839183A2838B
:10ECE000B3830E94498DB80181E493E30E944F8D64
:10ECF0008091160799E6899FB00111246755794FD5
:10ED000086E393E30E944F8D4091A1065091A206A5
:10ED10006091A3067091A40680E393E30E94B08DF6
:10ED20008AE00E948B92809116078F5F809316076E
:10ED300025C0FF2039F00E94498D80E293E30E94B4
:10ED40003B8D1CC01092160722E001C021E02B83EE
:10ED50000E94498D8BE193E30E943B8D2B812130F2
:10ED600009F494C08FE093E30E943B8DB80187E0E3
:10ED700093E30E944F8D8AE00E948B9202DD40E077
:10ED8000B801CE01019684DE8C01009709F481C0A0
:10ED900069817A81EE2009F44FC021E0AC0187E15E
:10EDA00097E00E940184882309F43EC080912807DF
:10EDB00090912907A0912A07B0912B078093A5066F
:10EDC0009093A606A093A706B093A8061092A1065A
:10EDD0001092A2061092A3061092A406B80189EF21
:10EDE00092E30E944F8D4091A5065091A606609136
:10EDF000A7067091A80681EF92E30E94B08D8AE089
:10EE00000E948B9282EE92E30E943B8DB80180E0DB
:10EE100090E0CCDD80919B08811102C0C80102C046
:10EE20008BE998E060E02FC0B8018EEC92E30E947D
:10EE30004F8D8BEC92E30FC026E5AC0187E197E0A4
:10EE40000E94018481110AC0B80187EB92E30E94FD
:10EE50004F8D84EB92E30E943B8D1BC08091EA08AA
:10EE600081608093EA08B80180E090E09FDD109215
:10EE7000B00BB80182EA92E30E944F8D8AE00E94B3
:10EE80008B9260E0C8010E94B96B03C085E193E3F7
:10EE90006BCF0F900F900F90DF91CF911F910F913B
:10EEA000FF90EF9008952091EA0822602093EA08ED
:10EEB00040E060E0D8CE0F931F93CF93DF93CDB7A0
:10EEC000DEB76B970FB6F894DEBF0FBECDBF8C01D7
:10EED00019821C8280916708811103C06FE778E076
:10EEE00002C064E678E021E0A801CE0101960E940C
:10EEF00001848823F1F08BE1FE013196A4E6B8E0AD
:10EF000001900D928A95E1F7A0915507AA30D8F4A7
:10EF100081E08A0F809355078BE18A9FD0011124ED
:10EF2000AA5AB84FE4E6F8E001900D928A95E1F70D
:10EF30000AC00E94498DB80189E092E30E944F8D7A
:10EF40008AE00E948B92CE010196BDD96B960FB6D6
:10EF5000F894DEBF0FBECDBFDF91CF911F910F910F
:10EF60000895809155078823C9F0815080935507F3
:10EF7000882359F090E001972BE1289FF001299F09
:10EF8000F00D1124EA5AF84F02C0EFE7F8E08BE1E8
:10EF9000A4E6B8E001900D928A95E1F780915507BB
:10EFA00008958BE1EFE7F8E0A4E6B8E001900D9258
:10EFB0008A95E1F708958091EA08877F8093EA08AF
:10EFC00080918208882321F08FE798E00E940582D3
:10EFD00045E360E080E597E012D8811105C00E940A
:10EFE000498D8BED93E32AC041E060E577E082E351
:10EFF00097E07DD481110DC040E060E577E082E3C9
:10F0000097E075D4811105C00E944C8D87EC93E385
:10F0100015C062E377E08FE798E0E5D6811105C07F
:10F020000E944C8D86EB93E309C08091EA088860CA
:10F030008093EA080E94498D8AEA93E30E943B8DFF
:10F04000B0DF83E080931E020895AF92BF92CF920B
:10F05000DF92EF92FF921F93CF93DF93CDB7DEB78E
:10F06000A8970FB6F894DEBF0FBECDBF80919A0867
:10F0700087FD61C08091EA0882FD5DC083FF9BDF50
:10F080008091EA0883FF54C080919A08082E000CF2
:10F09000990BC0969F938F9386E392E39F938F93F0
:10F0A0006E0181E2C80ED11CDF92CF920F944C3BCF
:10F0B00040E050E0BA018FE798E00E9424810F9071
:10F0C0000F900F900F900F900F90FE0131967F01DF
:10F0D00040E050E0B7018FE798E00E947580181675
:10F0E0003CF5F70101900020E9F731971E2F1E191A
:10F0F000115068F05701A10EB11C17FDBA94F5012B
:10F10000808190E00F94783AF5018083F1CF8A8571
:10F110008E37F1F245E050E0B601C7010F94243B71
:10F12000892BB1F6C601CDDA80919A088F5F01C0B4
:10F130008FEF80939A08A8960FB6F894DEBF0FBEA3
:10F14000CDBFDF91CF911F91FF90EF90DF90CF90D7
:10F15000BF90AF90089510929A0823CF60CC0E9480
:10F160000ED987E197E00E940582809116078823D7
:10F1700029F181508093160729E6829FC00111244E
:10F1800041E061E08755994F6EDDE091160784E01C
:10F19000E89FF0011124EE5EF84F408151816281B9
:10F1A00073814093A1065093A2066093A3067093C7
:10F1B000A40687E197E00E942481DBCAE2DA0E947C
:10F1C000E8D80F944B2D0F94902D6D337105810568
:10F1D000910520F085E092E30F94EA2110928406D5
:10F1E0000C94E46E10927F081092820810926408CA
:10F1F0001092670880E090E0FC01EA5AF84F108214
:10F2000013824B968E3021E09207B1F789E180930B
:10F210005107109254071092490710921707109245
:10F220001A070895CF93DF9387E197E04CD8C4E69F
:10F23000D8E06B97CE0147D887E0C635D807C9F725
:10F2400084E698E040D88FE798E0DF91CF913BC803
:10F25000CF938091EF088823B9F14091F20A509141
:10F26000F30A6091F40A7091F50A22EF38E0809178
:10F27000F0089091F1080E940A71C82F811102C014
:10F28000C0E023C04091EB085091EC086091ED087C
:10F290007091EE08411551056105710591F022EF5D
:10F2A00038E08091F0089091F1080E940A7188235B
:10F2B00039F31092EB081092EC081092ED081092BE
:10F2C000EE081092EF0801C0C1E08C2FCF91089595
:10F2D000CF92DF92EF92FF92CF936B017C01C42F0C
:10F2E0008091F20A9091F30AA091F40AB091F50A84
:10F2F0008C159D05AE05BF05C9F0AADF811102C0BE
:10F3000080E018C022EF38E0B701A6018091F00834
:10F310009091F1080E94C270882391F3C092F20A82
:10F32000D092F30AE092F40AF092F50A81E0C1115A
:10F330008093EF08CF91FF90EF90DF90CF900895EA
:10F34000CF92DF92EF92FF920F931F93CF93DF93B1
:10F35000FC0181859285A385B4850196A11DB11D0F
:10F3600084179507A607B70710F480E060C0878967
:10F37000803149F4BB27A72F962F852FC388D488C7
:10F38000E588F6880FC0803281F783899489A58942
:10F39000B6896A017B01C7E0F694E794D794C794D5
:10F3A000CA95D1F78C0D9D1DAE1DBF1DE9016A01E7
:10F3B0007B018F014091F20A5091F30A6091F40AA7
:10F3C0007091F50A84179507A607B70731F040E05A
:10F3D000BC01CD017DDF882341F2F80187898031AE
:10F3E00079F4B701A601552766277727440F551FE3
:10F3F000FA01EE50F74F80819181A0E0B0E012C099
:10F40000B701A6014F77552766277727440F551F69
:10F41000440F551FFA01EE50F74F80819181A28170
:10F42000B381BF7088839983AA83BB8381E0DF9116
:10F43000CF911F910F91FF90EF90DF90CF900895A3
:10F440004F925F926F927F92AF92BF92CF92DF9274
:10F45000EF92FF920F931F93CF93DF9300D01F92F1
:10F46000CDB7DEB78C0149835A836B837C83590106
:10F47000C12CD12C7601412C82E0582E612C712CAC
:10F4800049815A816B817C819E012F5F3F4FC8016A
:10F4900057DF882341F1D301C201F801058404C07C
:10F4A000880F991FAA1FBB1F0A94D2F7C80ED91E36
:10F4B000EA1EFB1E49815A816B817C8187898031DC
:10F4C00039F481E0483F5F4F6105710538F4D8CFCA
:10F4D00081E0483F5F4F6F4F7F4090F2F501C0825F
:10F4E000D182E282F3820F900F900F900F90DF9104
:10F4F000CF911F910F91FF90EF90DF90CF90BF9031
:10F50000AF907F906F905F904F9008954F925F9271
:10F510006F927F928F929F92AF92BF92CF92DF9223
:10F52000EF92FF920F931F93CF93DF93EC016A0149
:10F530007B0128013901423051056105710510F444
:10F5400080E064C089859A85AB85BC850196A11D44
:10F55000B11D84179507A607B70790F38F898031EF
:10F5600049F48D2C9E2CAF2CBB248B899C89AD89B2
:10F57000BE890FC0803221F78B889C88AD88BE88F9
:10F58000DB01CA0157E0B695A795979587955A95DF
:10F59000D1F7880E991EAA1EBB1E41E0C501B40119
:10F5A00097DE882369F29F89903161F4DD24EE248F
:10F5B000FF249601220F331FF901EE50F74F5182BD
:10F5C000408211C0E894C7F8DD24EE24FF249601A0
:10F5D000220F331F220F331FF901EE50F74F4082E5
:10F5E0005182628273829A89923080F04D815E816D
:10F5F0006F817885840E951EA61EB71E8092EB083B
:10F600009092EC08A092ED08B092EE08DF91CF91B5
:10F610001F910F91FF90EF90DF90CF90BF90AF9030
:10F620009F908F907F906F905F904F9008952F9252
:10F630003F924F925F926F927F928F929F92AF9282
:10F64000BF92CF92DF92EF92FF920F931F93CF93CF
:10F65000DF93CDB7DEB72F970FB6F894DEBF0FBE9E
:10F66000CDBF1C014D835E836F8378873B872A87DC
:10F67000FC0181859285A385B4858C019D010F5F76
:10F680001F4F2F4F3F4F0C871D872E873F87AA851F
:10F69000BB85CD90DD90ED90FC90C114D104E104C8
:10F6A000F10431F0BFEFCB1ADB0AEB0AFB0A10C002
:10F6B000F101C080D180E280F380F1E0F9870D8113
:10F6C0001E812F813885013011052105310509F092
:10F6D000198646015701412C512C3201F1018185D7
:10F6E0009285A385B485481659066A067B0608F0FC
:10F6F0004EC00C851D852E853F85081519052A05E8
:10F700003B0550F482E0882E912CA12CB12C92E084
:10F71000C92ED12CE12CF12C9E012F5F3F4FB5015A
:10F72000A401C1010DDE882391F149815A816B81C9
:10F730007C81D501C4010196A11DB11D452B462B2D
:10F74000472B19F06C017D010FC0AC01BD014C19B4
:10F750005D096E097F090D811E812F813885401753
:10F7600051076207730741F01FEF411A510A610AFE
:10F77000710A4C015D01B2CF0FEF1FEF2FEF3FE099
:10F78000B501A401C101C2DE8D83811113C01D82A8
:10F790003DC02401350121E0421A51086108710879
:10F7A00095018401B301A201C101B0DE882379F380
:10F7B00053014201C814D904EA04FB0450F3AA859A
:10F7C000BB854D915D916D917C9141155105610510
:10F7D0007105A9F4EA85FB85C082D182E282F382B9
:10F7E000F985FF2399F00FEFC01AD00AE00AF00A5A
:10F7F000D101CD92DD92ED92FC92139707C0970153
:10F800008601C10183DE8111E5CFC1CF8D812F96A5
:10F810000FB6F894DEBF0FBECDBFDF91CF911F9121
:10F820000F91FF90EF90DF90CF90BF90AF909F909F
:10F830008F907F906F905F904F903F902F900895A2
:10F84000AF92BF92CF92DF92EF92FF920F931F93EE
:10F85000CF93DF9300D01F92CDB7DEB75C016A0172
:10F860007B0182E090E0A0E0B0E0F501808391832D
:10F87000A283B3839E012F5F3F4FB701A601C5014D
:10F880005FDD882321F100E010E09801B701A601B7
:10F89000C5013CDE8823D9F0C980DA80EB80FC808A
:10F8A000F5018789803149F481E0F8EFCF16FFEF49
:10F8B000DF06E104F10460F4DDCF81E098EFC916C2
:10F8C0009FEFD906E9069FE0F90610F4D3CF80E058
:10F8D0000F900F900F900F90DF91CF911F910F918C
:10F8E000FF90EF90DF90CF90BF90AF9008954F9230
:10F8F0005F926F927F928F929F92AF92BF92FF9290
:10F900000F931F93CF93DF93EC01142F7093F108A3
:10F910006093F0081F8A82E090E0A0E0B0E0888366
:10F920009983AA83BB831092EF081092EB08109280
:10F93000EC081092ED081092EE088FEF9FEFDC01BB
:10F940008093F20A9093F30AA093F40AB093F50A15
:10F95000442371F1453008F0E0C040E060E070E021
:10F96000CB01B6DC882309F4D8C020E1129FA001A6
:10F9700011244E51574FFA01E254FE4F80818F7788
:10F9800009F0CBC03C9680819181A281B3818436FD
:10F990009105A105B10508F4C0C03497808091801D
:10F9A000A280B38081149104A104B10421F4B5C0F4
:10F9B000812C912C540140E0C501B40189DCF82E62
:10F9C000882309F4AAC08091FD089091FE08811552
:10F9D000924009F0A2C090910209992309F49DC0B8
:10F9E0002091000930910109232B09F496C08091E0
:10F9F000FF08882309F491C09A8B8C831D8690E0C0
:10FA000061E070E02D85E22FAB01022E02C0440FB1
:10FA1000551F0A94E2F78417950731F031E0320F51
:10FA20003D87283078F379C0209108093091090981
:10FA30002115310519F040E050E008C02091160969
:10FA40003091170940911809509119092D833E836F
:10FA50004F83588780910009909101092401350155
:10FA6000480E591E611C711C4B8A5C8A6D8A7E8A05
:10FA70000091030910910409198F088FA0910209C0
:10FA8000B0E00F949E36460E571E681E791E4A8EB1
:10FA90005B8E6C8E7D8E85E0000F111F8A95E1F7DD
:10FAA00001501E4F012F11270695400E511E611C5B
:10FAB000711C4E865F86688A798A2091050930918B
:10FAC00006092115310521F0890120E030E008C048
:10FAD0000091120910911309209114093091150910
:10FAE000B501A4014419550966097709400F511F52
:10FAF000621F731F04C07695679557954795EA95E1
:10FB0000D2F749875A876B877C87453F8FE0580734
:10FB10006105710520F48CE08F8BF12C15C0453FF9
:10FB20005F4F6105710510F480E10DC080911E09E1
:10FB300090911F09A0912009B09121098A8F9B8F74
:10FB4000AC8FBD8F80E28F8B8F2DDF91CF911F9176
:10FB50000F91FF90BF90AF909F908F907F906F908C
:10FB60005F904F900895CF93DF93EC019C012C5F41
:10FB70003F4F41E050E060E070E0898D9A8D57DDA5
:10FB8000882399F04D895E896F89788D452B462BA6
:10FB9000472B59F44C815D816E817F814D8B5E8B4B
:10FBA0006F8B788F998190689983DF91CF910895B9
:10FBB000CF92DF92EF92FF920F931F93CF93DF9339
:10FBC000DC0151964D915D916D917C915497403E31
:10FBD0005F4F6F41710510F010E067C0EC01C3DFAB
:10FBE0008823D1F335DB182F8823B1F3E98DFA8D03
:10FBF0008C819D81AE81BF810297A109B1090584E5
:10FC000004C0880F991FAA1FBB1F0A94D2F7C6848D
:10FC1000D784E088F188C80ED91EEA1EFB1E81E059
:10FC20008093EF08C092F20AD092F30AE092F40AAD
:10FC3000F092F50A80E092E0E2EFF8E0DF019C014B
:10FC40001D9221503040E1F701E0E98DFA8D848169
:10FC5000081798F422EF38E0B701A601400F511DB4
:10FC6000611D711D8091F0089091F1080E940A7148
:10FC7000882309F4B1CF0F5FE8CF40E052E060E0A5
:10FC800070E0058404C0440F551F661F771F0A9457
:10FC9000D2F789899A89AB89BC89480F591F6A1F95
:10FCA0007B1F498B5A8B6B8B7C8B812FDF91CF9184
:10FCB0001F910F91FF90EF90DF90CF900895CF9319
:10FCC000DF93EC0141E0611101C040E06C857D856E
:10FCD0008E859F85FDDA882341F0888920E2829F06
:10FCE000C00111248E50974F02C080E090E0DF9158
:10FCF000CF910895FC0120E090E08EE23081303217
:10FD000069F0283029F4DB01A90FB11D8C939F5FA6
:10FD1000DB01A90FB11D30813C939F5F2F5F3196AE
:10FD20002B3061F7FB01E90FF11D10820895CF938D
:10FD3000DF93FC012381211102C080E010C022501A
:10FD4000223028F48FE2FB018083118207C0EB018F
:10FD500060E0B5DF009789F3BE01CCDF81E0DF9181
:10FD6000CF9108952BE030E22150FB01E20FF11D0D
:10FD700030832111F9CFDC0197E03A2FEB2F8D91E1
:10FD800081110AC0DA013C931196EC9381E0FB01EA
:10FD90009081903239F525C08F32A1F38E3229F44B
:10FDA0009A30F9F028E09AE0E8CFE7E0F4E3349104
:10FDB000332321F031963813FACF13C0921788F00D
:10FDC000813278F08F3769F031E0320FFB01E20FBA
:10FDD000F11D2FE9280F2A3108F480528083232F48
:10FDE000CCCF80E008950F931F93CF93DF93FC0156
:10FDF0002381222311F080E043C08B01EC01FB0141
:10FE00008789803131F18032B1F783E08B83F8014B
:10FE1000428D538D648D758D4D8B5E8B6F8B788F7E
:10FE20009E012F5E3F4FC8010BDB882321F31A8F01
:10FE3000098F81E08983188619861A861B861C82A1
:10FE40001D821E821F82188A1C861D861E861F86A2
:10FE500017C082E08B831D8A1E8A1F8A188EFB01C1
:10FE6000808D918DA0E0B0E025E0880F991FAA1F3A
:10FE7000BB1F2A95D1F7898B9A8BAB8BBC8BD7CFC5
:10FE8000DF91CF911F910F9108952F923F924F9242
:10FE90005F926F927F928F929F92AF92BF92CF921A
:10FEA000DF92EF92FF920F931F93CF93DF9300D0D7
:10FEB0001F92CDB7DEB79C838B834B015A01DC01C7
:10FEC00013968C91811103C08FEF9FEFE1C0EB81FE
:10FED000FC81818180FFF8CFEB81FC81818992894F
:10FEE000A389B4894085518562857385841B950BF0
:10FEF000A60BB70BA50160E070E084179507A60775
:10FF0000B70708F45C0175018B819C8104969A8384
:10FF10008983612C92E0792EE114F10409F48AC0FE
:10FF2000AB81BC8118964D915D916D917C911B9731
:10FF30006A01B1E0DB22EB81FC8123811A012B01F4
:10FF400089E056944794379427948A95D1F7818D08
:10FF5000928D223061F4FC01828D938DA48DB58D3C
:10FF6000BC01CD01620D731D841D951D49C0DC01CE
:10FF700014961C9111501221C114D104F9F41111DD
:10FF80001DC0452B462B472B59F4EB81FC818589FD
:10FF90009689A789B08D84839583A683B7830EC085
:10FFA000AB81BC8114964D915D916D917C911797B9
:10FFB00029813A81C5D9882309F486CFEB81FC8158
:10FFC000218D328D84819581A681B7810297A10907
:10FFD000B109F901058404C0880F991FAA1FBB1F2E
:10FFE0000A94D2F74685578560897189840F951FD9
:10FFF000A61FB71FBC01CD01610F711D811D911D91
:020000021000EC
:1000000093012C193D0987012E153F0508F489013C
:100010000115F2E01F0779F52091F20A3091F30AF9
:100020004091F40A5091F50A621773078407950707
:1000300019F421C0C5012CC09401AB01BC01809111
:10004000F0089091F1080E94C270882309F43CCF17
:10005000800E911EEB81FC8180859185A285B38500
:10006000800F911FA11DB11D80879187A287B38743
:10007000E01AF10A51CF40E02BD9882309F424CFAC
:10008000B6016E50774FA801C4010F94EB3AE0CF50
:100090000F900F900F900F90DF91CF911F910F91C4
:1000A000FF90EF90DF90CF90BF90AF909F908F9098
:1000B0007F906F905F904F903F902F900895CF93D7
:1000C000DF931F92CDB7DEB741E050E0BE016F5F16
:1000D0007F4FDBDE019719F4898190E002C08FEF3A
:1000E0009FEF0F90DF91CF910895DF92EF92FF92F3
:1000F0000F931F93CF93DF93FC012381223060F095
:1001000000851185228533850F711127222733271A
:10011000012B022B032B11F08FEF5DC04115510510
:1001200011F0FA0110827A01EB018C018DE0D82EDA
:1001300040E250E0BE01C801A8DE8032910539F0EE
:1001400021E0892B09F420E0822F819544C0288189
:100150002223C9F1253E11F02E3231F4E114F104CD
:1001600039F3F7011082E4CFE114F10441F13B854A
:100170003F733F3021F54A8D5B8D452B01F52F7183
:100180003FEF320F3530D8F430E021503109D29EA4
:10019000C001D39E900D1124D701A80FB91FFE01F5
:1001A00020E0AD01253088F431813D932F5F3296F8
:1001B0002D30C1F7288126FF02C0FA0115862B8554
:1001C00023FDB6CF08C080E006C02B3010F4348188
:1001D000ECCF3681EACFDF91CF911F910F91FF9045
:1001E000EF90DF9008951F93CF93DF93FC0123815D
:1001F000223018F480E090E023C0EC014085518566
:100200006285738585E076956795579547958A95BC
:10021000D1F7142F1F70CF0152DF97FDEBCF8885E8
:100220009985AA85BB854F96A11DB11D88879987A1
:10023000AA87BB87F0E21F9FC00111248E50974F01
:10024000DF91CF911F9108958F929F92AF92BF92AD
:10025000CF92DF92EF92FF920F931F93CF93DF9392
:10026000EC018B81811102C080E077C009891A8975
:100270002B893C890417150726073707A8F36A015D
:100280007B01823029F4C886D986EA86FB860DC0B8
:10029000C114D104E104F10451F4188619861A86B8
:1002A0001B861C821D821E821F8281E056C08884AC
:1002B0009984AA84BB84E98DFA8D258530E0275F77
:1002C0003F4FB501A4014150510961097109022E46
:1002D00004C076956795579547950A94D2F7D7014C
:1002E000C6010197A109B10904C0B695A7959795D4
:1002F00087952A95D2F784179507A607B70720F0A8
:1003000089288A288B2849F44D895E896F89788DE0
:100310004C835D836E837F8304C0841B950BA60B87
:10032000B70B4C015D018E010C5F1F4F81149104CE
:10033000A104B10409F4A7CF4C815D816E817F8156
:100340009801898D9A8D0E94A07991E0891A91086F
:10035000A108B1088111EACF87CFDF91CF911F911A
:100360000F91FF90EF90DF90CF90BF90AF909F9054
:100370008F9008950F931F93CF93DF93EC018B81A0
:100380008823D9F1898187FF32C061E0CE0197DCF3
:100390008C01009791F1FC018081853E71F18B8188
:1003A000823040F489899A89AB89BC89848F958F82
:1003B000A68FB78F8D899E89AF89B88DF801938FED
:1003C000828FB58BA48BE091F60AF091F70A3097F3
:1003D00059F0B8016A5E7F4FC80148961995F80137
:1003E000808D918D938B828B89818F778983DF912B
:1003F000CF911F910F910C94287981E0888380E040
:10040000DF91CF911F910F910895CF93DF93EC016E
:10041000B1DF1B82DF91CF9108954F925F926F926F
:100420007F928F929F92AF92BF92EF92FF920F9323
:100430001F93CF93DF9300D01F92CDB7DEB7FC019F
:1004400083818130E1F4818181FF19C081899289A2
:10045000A389B48984179507A607B70780F0892B6D
:100460008A2B8B2B09F474C04A015B017F01408405
:10047000518462847384CF01E7DE811102C080E081
:1004800068C0F701818D928D81149104A104B1049B
:1004900069F4458956896789708DD2D9882379F3A3
:1004A000F701158A168A178A108E39C0F701448120
:1004B0005581668177819E012F5F3F4F0E94A07911
:1004C0008823E9F249815A816B817C81F701818D12
:1004D000928DFC012789203139F4483FFFEF5F07F7
:1004E00061057105E0F407C0483F2FEF520762072E
:1004F0002FE07207A0F4A4D9882309F4C0CFF70134
:1005000044815581668177810FEF1FEF2FEF3FE028
:10051000818D928D0E94867A882309F4B0CFF701ED
:10052000818A928AA38AB48A818180688183C70183
:1005300021DF882309F4A3CFB501A401481459048D
:100540006A047B0410F4B301A201C7017DDE01C07F
:1005500081E00F900F900F900F90DF91CF911F913E
:100560000F91FF90EF90BF90AF909F908F907F90F2
:100570006F905F904F9008951F93CF93DF93EC019E
:10058000142F80E2689FF00111249F012E50374FF5
:10059000D9011B968C91817121F0842F827109F011
:1005A00057C08091F20A9091F30AA091F40AB09199
:1005B000F50A8C879D87AE87BF87688BEE50F74F13
:1005C0004489558960E070E0BA01552744274D8B76
:1005D0005E8B6F8B788F828D938DA0E0B0E0482B7F
:1005E000592B6A2B7B2B4D8B5E8B6F8B788FD901B0
:1005F0001B968C91887151F4848D958DA68DB78D45
:10060000898B9A8BAB8BBC8B81E00CC0803101F560
:100610009E012F5E3F4F898D9A8D0E94207A8823FC
:10062000B9F084E08B83812F8F7089831C821D82B7
:100630001E821F82188619861A861B8614FF0BC01D
:1006400040E050E0BA01CE01E8DE811104C00FC0E5
:100650001B8280E00CC015FF09C049895A896B894B
:100660007C89CE01DF91CF911F91EECD81E0DF91AA
:10067000CF911F910895BF92CF92DF92EF92FF9298
:100680000F931F93CF93DF938C01EB016A01E22E4E
:10069000898D9A8DF801928F818F40E050E0BA01E8
:1006A000CE01D2DDF12C88859985AA85BB85498943
:1006B0005A896B897C8984179507A607B707C0F507
:1006C00025E0B695A795979587952A95D1F7F82FA8
:1006D000FF70BF2ECE0187DDDC01892B09F486C0B7
:1006E0008C91882319F0853EB9F47DC0F1100EC0BD
:1006F0004091F20A5091F30A6091F40A7091F50A60
:10070000F8014487558766877787B08A8C9188235C
:1007100069F0FF24F394C7CF4BE050E0BD01C60160
:100720000F94DE3A892B09F0BECF5AC0FF24F39410
:100730008E2D8274823409F059C0FF2049F0F801EF
:10074000B08861E0C801BBDAEC01892B69F44EC0C6
:100750008B81823009F44AC0CE012ADA882309F459
:1007600045C0C2EFD8E0B12C80E2FE0111928A951B
:10077000E9F78BE0F601DE0101900D928A95E1F731
:10078000E091F60AF091F70A309739F0BE01625F06
:100790007F4FCE014096199508C081E298E2998B6F
:1007A000888B80E098E09F878E87888999899B8BCA
:1007B0008A8B998F888F8E859F859F8B8E8B0E94C9
:1007C0002879882399F04E2D6B2DC801DF91CF91A8
:1007D0001F910F91FF90EF90DF90CF90BF90CCCE04
:1007E000E7FEF1CF03C0F11094CF82CF80E0DF911C
:1007F000CF911F910F91FF90EF90DF90CF90BF901E
:1008000008953F924F925F926F927F928F929F9244
:10081000AF92BF92CF92DF92EF92FF920F931F930E
:10082000CF93DF93CDB7DEB7C354D1090FB6F89499
:10083000DEBF0FBECDBF5C016B0124965FAF4EAF34
:100840002497522E1C8E1F8E19821C8261157105F1
:1008500011F410E074C0FC0183818111FACF249659
:10086000EEADFFAD249780818F32F1F4F6018381E4
:100870008250823058F0618D728DCE010196B3DACC
:10088000882339F38E010F5F1F4F01C08601249624
:10089000EEADFFAD249780818F3239F431962496E6
:1008A000FFAFEEAF2497F3CF8B017E01FCE1EF0E9B
:1008B000F11C3701CE0101964C014E2C3F2CAE01AC
:1008C0004E5B5F4FBE01695C7F4F24968EAD9FAD3E
:1008D000249748DA882309F4BCCF2496EEADFFAD07
:1008E000249780818F3231F431962496FFAFEEAF9A
:1008F0002497F3CF8823D9F021E0AE01495C5F4F04
:10090000B801C701B8DE882309F4A3CF0C151D0573
:1009100011F0C8017ADDE614F70431F0942D832D2F
:100920008701E92EF82ECBCF982D892DF9CF252DD3
:10093000AE01495C5F4FB801C5019DDE182FCE01A5
:1009400001960E946371CE014C960E946371812FC3
:10095000CD5BDF4F0FB6F894DEBF0FBECDBFDF918A
:10096000CF911F910F91FF90EF90DF90CF90BF90AC
:10097000AF909F908F907F906F905F904F903F903F
:100980000895CF93DF93EC0140E050E0BA0145DDDC
:10099000882369F061E0CE0192D9009741F025EEFD
:1009A000FC0120831B82DF91CF910C94287980E099
:1009B000DF91CF9108951F93CF93DF93CDB7DEB72B
:1009C0006B970FB6F894DEBF0FBECDBFAB01198297
:1009D0001C8222E0BC01CE01019613DF182F882370
:1009E00021F0CE010196CDDF182FCE0101960E9495
:1009F0006371812F6B960FB6F894DEBF0FBECDBF2B
:100A0000DF91CF911F9108952F923F924F925F9265
:100A10006F927F928F929F92AF92BF92CF92DF920E
:100A2000EF92FF920F931F93CF93DF9300D01F920B
:100A3000CDB7DEB78C014B013A01DC0113968C91E6
:100A400013978130C1F411968C9181FF14C082FFFD
:100A500018C0F8014189528963897489808591851C
:100A6000A285B38584179507A607B70751F0C8017B
:100A7000EBDB811106C081E0D8018C938FEF9FEFF3
:100A80003CC1530184C0D80159968D919C915A97CD
:100A9000FC0154805A946A017B0129E0F694E794A2
:100AA000D794C7942A95D1F75C207A01F1E0FF2210
:100AB000552009F478C080E092E08E199F09650105
:100AC0008A159B0508F46C01D80159962D913C912B
:100AD0005A9714968D919D910D90BC91A02D0297DF
:100AE000A109B109F901058404C0880F991FAA1F43
:100AF000BB1F0A94D2F74685578560897189840F98
:100B0000951FA61FB71F9C01AD01250D311D411D6D
:100B1000511D19012A01C11432E0D30609F08AC01F
:100B20008091F20A9091F30AA091F40AB091F50A2B
:100B300082159305A405B50569F41092EF088FEFAF
:100B40009FEFDC018093F20A9093F30AA093F40ADA
:100B5000B093F50A9401B201A1018091F00890913F
:100B6000F1080E940A71882309F485CFF801808575
:100B70009185A285B3858C0D9D1DA11DB11D80871A
:100B80009187A287B3878C0C9D1CAC18BD08D80137
:100B900018964D915D916D917C911B97A114B104B4
:100BA00009F071CF7DC0E114F10409F084CF1496EF
:100BB0004D915D916D917C9117974115510561059E
:100BC000710559F455968D919D910D90BC91A02D74
:100BD0000097A105B10541F521C09E012F5F3F4F50
:100BE0000E94A079882309F446CF89819A81AB813C
:100BF000BC81F801218D328DF9012789203139F42A
:100C0000883FFFEF9F07A105B10540F40DC0883F65
:100C10002FEF9207A2072FE0B20730F0C8010E9421
:100C2000B37D811148CF27CFF80184839583A683B4
:100C3000B78341CFE114F10419F5D80118964D910D
:100C40005D916D917C911B9751968D919D910D9029
:100C5000BC91A02D481759076A077B0788F00E94AE
:100C60002879882309F407CF81E08093EF08209248
:100C7000F20A3092F30A4092F40A5092F50A08C040
:100C800041E0C201B1010E946879882309F4F3CEE2
:100C9000A601B401C7018E50974F0F94EB3A66CF6F
:100CA0005196CD90DD90ED90FC90549711968C91DB
:100CB000C416D506E606F70640F4F801418B528BC0
:100CC000638B748B806881830DC02091F60A30910C
:100CD000F70A232B39F06114710421F08068D801E0
:100CE00011968C93F801818183FD02C0C30105C078
:100CF000C80140DB8111FACFBECE0F900F900F904C
:100D00000F90DF91CF911F910F91FF90EF90DF90A7
:100D1000CF90BF90AF909F908F907F906F905F909B
:100D20004F903F902F900895FB0101900020E9F72C
:100D30003197AF01461B570B67CECF93C82F0E9448
:100D4000FFACCC2351F024982C9A65E070E080E051
:100D500090E00E94ED2B149A03C0249A2C981498CA
:100D6000CF91089580E0E9CFCF92DF92EF92FF928A
:100D70006B017C0183E3C816D104E104F10470F037
:100D800082E3C81AD108E108F10862E370E080E06C
:100D900090E00E94ED2B0E943EA1ECCFC701B6016E
:100DA0000E94ED2BFF90EF90DF90CF900C943EA12E
:100DB000DC01FB01460F571FE417F507C1F08191D5
:100DC0002D913C911197382798E0B901660F771F54
:100DD00037FF06C09B0181E2282780E1382701C048
:100DE0009B01915091F711963C932E93E5CF089576
:100DF00024E6829FC001112481589F4F6FEF70E05D
:100E00000F943036262F6436710511F080E201C050
:100E100081E38093FB0A6A3071054CF03AE0822F3F
:100E2000632F0F9410360F941036905D01C090E23E
:100E30009093FC0A822F6AE00F941036905D909395
:100E4000FD0A85E28093FE0A8BEF9AE00895282F31
:100E5000843640F064E60F9410366AE00F94103642
:100E6000905D01C090E29093FC0A2A3048F03AE08D
:100E7000822F632F0F9410360F941036905D01C0AF
:100E800090E29093FD0A822F6AE00F941036905DF5
:100E90009093FE0A8CEF9AE008959C0197FD0EC096
:100EA0008436910584F064E670E00F943036CB010F
:100EB0006AE070E00F943036805D06C03195219570
:100EC00031098DE201C080E28093FC0A2A303105AD
:100ED00064F0EAE0F0E0C901BF010F943036CB01C5
:100EE000BF010F943036805D01C080E28093FD0A1F
:100EF000C9016AE070E00F943036805D8093FE0A8D
:100F00008CEF9AE00895AC01952F991F9927991FAE
:100F100029F022273327241B350B01C09A01483EB4
:100F20005340ACF0C90168EE73E00F943036CB014A
:100F3000EAE0F0E0BF010F943036805D8093FB0A59
:100F4000C90164E670E00F943036CB0112C024363C
:100F500031050CF1911102C080E201C08DE2809355
:100F6000FB0AC90164E670E00F943036CB01EAE079
:100F7000F0E0BF010F943036805D8093FC0AC90118
:100F8000BF010F943036CB01BF010F943036805D26
:100F90008093FD0A16C080E28093FB0A8093FC0ACE
:100FA0002A3031053CF091118DE28093FC0AEAE091
:100FB000F0E0E5CF911102C080E201C08DE28093A4
:100FC000FD0AC9016AE070E00F943036805D8093BD
:100FD000FE0A8BEF9AE008958F929F92AF92BF9294
:100FE000CF92DF92EF92FF92CF93FC01C080D1802D
:100FF000E280F38020E030E04AE754E4C701B60124
:101000000F9437354B015C0120E030E0A901C701A6
:10101000B6010F94F93287FD05C020E030E040EAC8
:1010200050E404C020E030E040EA50ECC501B401D7
:101030000F94203220E030E040E251E40F9400337E
:101040000F9468336B017C0197FD10C020E137E2FB
:1010500040E050E00F946536CA01B9012AE030E063
:1010600040E050E00F946536605D09C0F094E09474
:10107000D094C094C11CD11CE11CF11C6DE26093A2
:10108000F90AC701B60128EE33E040E050E00F94C2
:1010900065368AE0882E912CA12CB12CCA01B901A9
:1010A000A50194010F946536605D6093FA0AC7014B
:1010B000B60124E630E040E050E00F946536CA0106
:1010C000B901A50194010F946536605D6093FB0A38
:1010D0008EE28093FC0AC701B601A50194010F942A
:1010E0006536C62FCA01B901A50194010F94653672
:1010F000605D6093FD0AC05DC093FE0A89EF9AE0CF
:10110000CF91FF90EF90DF90CF90BF90AF909F90E6
:101110008F9008958F929F92AF92BF92CF92DF925D
:10112000EF92FF92FC01C080D180E280F38020E04A
:1011300030E048EC52E4C701B6010F9437354B015B
:101140005C0120E030E0A901C701B6010F94F9323B
:1011500087FD05C020E030E040EA50E404C020E014
:1011600030E040EA50ECC501B4010F94203220E099
:1011700030E040E251E40F9400330F9468339B0158
:1011800077FF06C022273327261B370B8DE201C0CD
:101190008BE28093F90AC90168EE73E00F94303650
:1011A000CB01EAE0F0E0BF010F943036805D809320
:1011B000FA0AC90164E670E00F943036CB01BF0132
:1011C0000F943036805D8093FB0AC901BF010F94F4
:1011D0003036282FCB01BF010F943036805D8093CD
:1011E000FC0A8EE28093FD0A205D2093FE0A89EFBF
:1011F0009AE0FF90EF90DF90CF90BF90AF909F90DC
:101200008F9008958F929F92AF92BF92CF92DF926C
:10121000EF92FF92CF93C62FFC01C080D180E28075
:10122000F38020E030E44CE156E4C701B6010F94AE
:1012300037354B015C0120E030E0A901C701B60160
:101240000F94F93287FD05C020E030E040EA50E419
:1012500004C020E030E040EA50ECC501B4010F9436
:10126000203220E030E040E251E40F9400330F944C
:1012700068336B017C01611571058105910561F091
:1012800097FF0CC0F094E094D094C094C11CD11C82
:10129000E11CF11C6DE203C060E201C06C2F6093A1
:1012A000F90AC701B60128EE33E040E050E00F94A0
:1012B00065368AE0882E912CA12CB12CCA01B90187
:1012C000A50194010F946536605D6093FA0A8EE281
:1012D0008093FB0AC701B60124E630E040E050E00D
:1012E0000F946536CA01B901A50194010F946536C2
:1012F000605D6093FC0AC701B601A50194010F94DB
:101300006536C62FCA01B901A50194010F9465364F
:10131000605D6093FD0AC05DC093FE0A89EF9AE0AC
:10132000CF91FF90EF90DF90CF90BF90AF909F90C4
:101330008F9008954F925F926F927F928F929F92BB
:10134000AF92BF92CF92DF92EF92FF92CF93B62EE1
:10135000FC01C080D180E280F38020E030E543ECE6
:1013600057E4C701B6010F9437352B013C0120E04B
:1013700030E0A901C701B6010F94F93287FD05C01D
:1013800020E030E040EA50E404C020E030E040EAF1
:1013900050ECC301B2010F94203220E030E040E273
:1013A00051E40F9400330F9468336B017C01611595
:1013B00071058105910561F097FF0CC0F094E094F0
:1013C000D094C094C11CD11CE11CF11C6DE203C07F
:1013D00060E201C06B2D6093F80AC701B60120E1FD
:1013E00037E240E050E00F9465368AE0882E912C79
:1013F000A12CB12CCA01B901A50194010F94653645
:10140000605D6093F90A8EE28093FA0AC701B60123
:1014100028EE33E040E050E00F946536CA01B90190
:10142000A50194010F946536605D6093FB0AC701C6
:10143000B60124E630E040E050E00F946536CA0182
:10144000B901A50194010F946536605D6093FC0AB3
:10145000C701B601A50194010F946536C62FCA01D4
:10146000B901A50194010F946536605D6093FD0A92
:10147000C05DC093FE0A88EF9AE0CF91FF90EF9095
:10148000DF90CF90BF90AF909F908F907F906F90A4
:101490005F904F9008958F929F92AF92BF92CF929C
:1014A000DF92EF92FF92FC01C080D180E280F38056
:1014B00020E030E0A901C701B6010F94F93287FF9F
:1014C00008C0C701B601905820E030E040E251E486
:1014D00006C020E030E040E251E4C701B6010F94BD
:1014E000373520E030E040EA50E40F94203220E02D
:1014F00030E040E251E40F9400330F9468336B0105
:101500007C016031F7E27F078105910584F020E1DD
:1015100037E240E050E00F946536CA01B9012AE095
:1015200030E040E050E00F946536605D01C060E25D
:101530006093FA0A88EEC81683E0D806E104F10445
:1015400094F0C701B60128EE33E040E050E00F947C
:101550006536CA01B9012AE030E040E050E00F945E
:101560006536605D01C060E26093FB0AE4E6CE167A
:10157000D104E104F10494F0C701B60124E630E09F
:1015800040E050E00F946536CA01B9012AE030E02E
:1015900040E050E00F946536605D01C060E260930A
:1015A000FC0AFAE0CF16D104E104F1049CF08AE0D1
:1015B000882E912CA12CB12CC701B601A501940154
:1015C0000F946536CA01B901A50194010F946536DF
:1015D000605D01C060E26093FD0AC701B6012AE0C8
:1015E00030E040E050E00F946536605D6093FE0AA5
:1015F0008AEF9AE0FF90EF90DF90CF90BF90AF908E
:101600009F908F9008958F929F92AF92BF92CF92AA
:10161000DF92EF92FF92CF93FC01C080D180E280F5
:10162000F38020E030E04AE754E4C701B6010F94AC
:1016300037354B015C0120E030E0A901C701B6015C
:101640000F94F93287FD05C020E030E040EA50E415
:1016500004C020E030E040EA50ECC501B4010F9432
:10166000203220E030E040E251E40F9400330F9448
:1016700068336B017C0197FF0AC0F094E094D0942A
:10168000C094C11CD11CE11CF11C8DE201C08BE295
:101690008093F80AC701B60120E137E240E050E04C
:1016A0000F9465368AE0882E912CA12CB12CCA01AA
:1016B000B901A50194010F946536605D6093F90A44
:1016C000C701B60128EE33E040E050E00F946536E4
:1016D000CA01B901A50194010F946536605D60935C
:1016E000FA0AC701B60124E630E040E050E00F946A
:1016F0006536CA01B901A50194010F946536605D94
:101700006093FB0A8EE28093FC0AC701B601A50133
:1017100094010F946536C62FCA01B901A501940141
:101720000F946536605D6093FD0AC05DC093FE0A4C
:1017300088EF9AE0CF91FF90EF90DF90CF90BF902D
:10174000AF909F908F9008958F929F92AF92BF928B
:10175000CF92DF92EF92FF92CF93FC01C080D180B5
:10176000E280F38020E030E0A901C701B6010F94C8
:10177000F93287FF08C0C701B601905820E030E079
:101780004AE754E406C020E030E04AE754E4C701E9
:10179000B6010F94373520E030E040EA50E40F9472
:1017A000203220E030E040E251E40F9400330F9407
:1017B00068336B017C01603AF6E87F07F1E08F0740
:1017C000910584F020EA36E841E050E00F94653658
:1017D000CA01B9012AE030E040E050E00F946536DC
:1017E000605D01C060E26093F80A80E1C81687E29C
:1017F000D806E104F10494F0C701B60120E137E214
:1018000040E050E00F946536CA01B9012AE030E0AB
:1018100040E050E00F946536605D01C060E2609387
:10182000F90AE8EECE16E3E0DE06E104F10494F0F6
:10183000C701B60128EE33E040E050E00F94653672
:10184000CA01B9012AE030E040E050E00F9465366B
:10185000605D01C060E26093FA0AC701B60124E648
:1018600030E040E050E00F9465368AE0882E912CFD
:10187000A12CB12CCA01B901A50194010F946536C0
:10188000605D6093FB0A8EE28093FC0AC701B6019B
:10189000A50194010F946536C62FCA01B901A501AF
:1018A00094010F946536605D6093FD0AC05DC0933E
:1018B000FE0A88EF9AE0CF91FF90EF90DF90CF90F3
:1018C000BF90AF909F908F9008958F929F92AF920C
:1018D000BF92CF92DF92EF92FF92FC01C080D18045
:1018E000E280F38020E030E04AE754E4C701B6012B
:1018F0000F9437354B015C0120E030E0A901C701AE
:10190000B6010F94F93287FD05C020E030E040EACF
:1019100050E404C020E030E040EA50ECC501B401DE
:101920000F94203220E030E040E251E40F94003385
:101930000F9468336B017C0197FF0AC0F094E09428
:10194000D094C094C11CD11CE11CF11C8DE201C0DB
:1019500080E28093F80AF0E1CF16F7E2DF06E104B7
:10196000F10494F0C701B60120E137E240E050E015
:101970000F946536CA01B9012AE030E040E050E03A
:101980000F946536605D01C060E26093F90A88EEED
:10199000C81683E0D806E104F10494F0C701B6014B
:1019A00028EE33E040E050E00F946536CA01B901FB
:1019B0002AE030E040E050E00F946536605D01C001
:1019C00060E26093FA0AC701B60124E630E040E025
:1019D00050E00F9465368AE0882E912CA12CB12C12
:1019E000CA01B901A50194010F946536605D609349
:1019F000FB0AC701B601A50194010F9465366B017E
:101A00007C01672B682B692B89F08EE28093FC0A9E
:101A1000CA01B901A50194010F946536605D609318
:101A2000FD0A80E38C0D8093FE0A1AC0CA01B90139
:101A3000A50194010F946536611571058105910525
:101A400039F02EE22093FC0A605D6093FD0A05C028
:101A500080E28093FD0A8093FC0A80E28093FE0A74
:101A600088EF9AE0FF90EF90DF90CF90BF90AF901B
:101A70009F908F900895CF93DF93FC018491EF01A5
:101A80002196882319F047D5FE01F8CFDF91CF9139
:101A900008958EE194E3EFCF84E294E3ECCF0F93CB
:101AA0001F93CF93DF931F921F92CDB7DEB7698349
:101AB0007A83E1DF6981062F7A81172FF8018191FE
:101AC0008F01882311F027D5F9CF0F900F90DF9168
:101AD000CF911F910F910895CF93DF93EB01CBDF4F
:101AE0006AE070E0CE01DF91CF9108C6CF92DF921D
:101AF000EF92FF926A017B01BEDF4AE050E0C7012E
:101B0000B601FF90EF90DF90CF90E7C5CF92DF92C4
:101B1000EF92FF926A017B01AEDF42E050E0C70125
:101B2000B601FF90EF90DF90CF9075C6CF92DF9215
:101B3000EF92FF926A017B019EDF42E050E0C70115
:101B4000B601FF90EF90DF90CF9065C6CF93DF9303
:101B5000EB0191DF6AE070E0CE01DF91CF91E3C548
:101B6000CF92DF92EF92FF926A017B0184DF4AE01D
:101B700050E0C701B601FF90EF90DF90CF90CDC548
:101B8000811103C087E194E302C08BE194E373CF3A
:101B9000F7DF8AE0C0C40C944C7181E0089581E0C5
:101BA00008958F929F92AF92BF92CF92DF92EF9261
:101BB000FF920F931F93CF93DF931F921F92CDB786
:101BC000DEB76C0159018B017B01E40EF51E0E1589
:101BD0001F0561F1F60180809180F80161918F010C
:101BE0006983C4016A830F94503E6A81681779F053
:101BF000C4010F94583EC4010F94503E9981891737
:101C000031F047DF8BE294E336DF81E010C041E042
